:020000040000FA
:100000000020040000000000FC0C0100FC0C0100BA
:10001000FC0C0100FC0C0100FC0C0100FC0C0100BC
:10002000FC0C0100FC0C0100FC0C0100FC0C0100AC
:10003000FC0C0100FC0C0100FC0C0100FC0C01009C
:10004000FC0C0100FC0C0100FC0C0100FC0C01008C
:10005000FC0C0100FC0C0100FC0C0100080C010070
:10006000FC0C0100FC0C0100FC0C0100FC0C01006C
:10007000FC0C0100FC0C0100FC0C0100FC0C01005C
:10008000FC0C0100FC0C0100FC0C0100FC0C01004C
:10009000FC0C0100FC0C0100FC0C0100FC0C01003C
:1000A000FC0C0100FC0C0100FC0C0100FC0C01002C
:1000B000FC0C0100FC0C0100FC0C0100FC0C01001C
:1000C000FC0C0100FC0C0100FC0C0100FC0C01000C
:1000D000FC0C0100FC0C0100FC0C0100FC0C0100FC
:1000E000FC0C0100FC0C0100FC0C0100FC0C0100EC
:1000F000FC0C0100FC0C0100FC0C0100FC0C0100DC
:10010000FC0C0100FC0C0100FC0C0100FC0C0100CB
:10011000FC0C0100FC0C0100FC0C0100FC0C0100BB
:10012000FC0C0100FC0C0100FC0C0100FC0C0100AB
:10013000FC0C0100FC0C0100FC0C0100FC0C01009B
:10014000FC0C0100FC0C0100FC0C0100FC0C01008B
:10015000FC0C0100FC0C0100FC0C0100FC0C01007B
:10016000FC0C0100FC0C0100FC0C0100FC0C01006B
:10017000FC0C0100FC0C0100FC0C0100FC0C01005B
:1001800082090100FC0C0100FC0C0100FC0C0100C8
:10019000FC0C0100FC0C0100FC0C0100FC0C01003B
:1001A000FC0C0100FC0C0100FC0C0100FC0C01002B
:1001B000FC0C0100FC0C0100FC0C0100FC0C01001B
:1001C000FC0C0100FC0C0100FC0C0100FC0C01000B
:1001D000FC0C0100FC0C0100FC0C0100FC0C0100FB
:1001E000FC0C0100FC0C0100FC0C0100FC0C0100EB
:1001F000FC0C0100FC0C0100FC0C0100FC0C0100DB
:10020000FFFFFF00FFFFFF00FC0C0100FC0C0100E2
:10021000FC0C0100FC0C0100FC0C0100FC0C0100BA
:10022000FC0C0100FC0C0100FC0C0100FC0C0100AA
:10023000FC0C0100FC0C0100FC0C0100FC0C01009A
:10024000FC0C0100FC0C0100FC0C0100FC0C01008A
:10025000FC0C0100FC0C0100FC0C0100080C01006E
:10026000FC0C0100FC0C0100FC0C0100FC0C01006A
:10027000FC0C0100FC0C0100FC0C0100FC0C01005A
:10028000FC0C0100FC0C0100FC0C0100FC0C01004A
:10029000FC0C0100FC0C0100FC0C0100FC0C01003A
:1002A000FC0C0100FC0C0100FC0C0100FC0C01002A
:1002B000FC0C0100FC0C0100FC0C0100FC0C01001A
:1002C000FC0C0100FC0C0100FC0C0100FC0C01000A
:1002D000FC0C0100FC0C0100FC0C0100FC0C0100FA
:1002E000FC0C0100FC0C0100FC0C0100FC0C0100EA
:1002F000FC0C0100FC0C0100FC0C0100FC0C0100DA
:10030000FC0C0100FC0C0100FC0C0100FC0C0100C9
:10031000FC0C0100FC0C0100FC0C0100FC0C0100B9
:10032000FC0C0100FC0C0100FC0C0100FC0C0100A9
:10033000FC0C0100FC0C0100FC0C0100FC0C010099
:10034000FC0C0100FC0C0100FC0C0100FC0C010089
:10035000FC0C0100FC0C0100FC0C0100FC0C010079
:10036000FC0C0100FC0C0100FC0C0100FC0C010069
:10037000FC0C0100FC0C0100FC0C0100FC0C010059
:1003800082090100FC0C0100FC0C0100FC0C0100C6
:10039000FC0C0100FC0C0100FC0C0100FC0C010039
:1003A000FC0C0100FC0C0100FC0C0100FC0C010029
:1003B000FC0C0100FC0C0100FC0C0100FC0C010019
:1003C000FC0C0100FC0C0100FC0C0100FC0C010009
:10400000CF6723000E7F24000E018800000000000F
:104010000C000700002E2F000100200011000700F7
:10402000000020000000E00002003200000002005A
:1040300000000000AC080200010000000040DA00AF
:104040000000FE004440A900004920000000E000FC
:104050000300320000002000A00188004440A800B6
:104060000000060091018800800078000000EB004D
:1040700015003700E280400032A0B4009101BA0080
:10408000E280400032A0B4009102BA00E280400019
:1040900032A0B4000002EB00472BDE00F507B200AF
:1040A000602CE10004003A000059EB008301E900B4
:1040B000FDFF3E00040037006128E10001003200EE
:1040C0000082EB00040007001101BA000200E000CA
:1040D000E8FF3A00000006003159BA008301E90008
:1040E0000C0032002159BA008301E90008003200B7
:1040F0000400E00003003A00E280400032A0B40077
:10410000F5FF370011D9BA008301E900FAFF3A0040
:104110008100E800E180400032A0B4000000060009
:10412000D6D90400000000002A0C040001000000A1
:104130003C0C040001000000520C040001000000CF
:10414000660C0400010000007A0C0400010000006D
:104150008E0C040001000000A20C0400010000000D
:10416000B00C040001000000E4C4040000000000E2
:104170007CC10400000000006EC1040000000000CB
:10418000C8C1040000000000B4C104000000000029
:10419000A8C10400000000009AC104000000000053
:1041A0008CC1040000000000F4C104000000000005
:1041B000DCC1040000000000D6C4040000000000C0
:1041C0002E91040000000000509104000000000047
:1041D000C28B040000000000628B0400000000009D
:1041E0006C91040000000000249004000000000016
:1041F0006A8C040000000000B68E0400000000007D
:104200001A90040000000000EA9104000000000081
:10421000D28B04000000000072AF04000000000018
:10422000D2AF040000000000F4AE04000000000063
:10423000A2AE0400000000003CB104000000000039
:1042400046B004000000000006B1040000000000B9
:1042500028B1040000000000E0B2040000000000EB
:1042600018B00400000000001698040000000000D0
:10427000E0970400000000004C98040000000000DB
:1042800086980400000000007A98040000000000F6
:10429000549B040000000000289904000000000066
:1042A000229B0400000000004C9B04000000000062
:1042B0004A9C040000000000AA98040000000000CE
:1042C00050E80400000000006AE80400000000005C
:1042D00040E804000000000036E804000000000090
:1042E000A8E80400000000009CE8040000000000B2
:1042F000CCE8040000000000C0E80400000000005A
:1043000090E8040000000000B4E804000000000091
:1043100084E8040000000000D4E90400000000006C
:104320000EE9040000000000BCE9040000000000E9
:104330000CEA040000000000D8E8040000000000BF
:1043400034FD040000000000F6FC04000000000042
:1043500072FD040000000000D0FC0400000000001A
:10436000C4FC040000000000D4FD040000000000B4
:10437000E0FD040000000000ECFD0400000000006F
:10438000F8FD040000000000BCFD04000000000077
:10439000C8FD040000000000B0FD040000000000A3
:1043A00048FE04000000000054FF0400000000006C
:1043B00074FF04000000000004FE04000000000080
:1043C00060E404000000000050E40400000000006D
:1043D00096E40400000000003AE40400000000003D
:1043E00048E4040000000000E2F9040000000000BE
:1043F000F6F9040000000000CAF904000000000003
:1044000064FA04000000000008FA04000000000044
:1044100016FA040000000000FC9C040000000000EC
:10442000CEFB040000000000D6CA0400000000001B
:1044300006CB04000000000030CC040000000000A7
:1044400024CB04000000000012CE04000000000095
:10445000E6C9040000000000BACA04000000000021
:10446000C8CA040000000000BACE0400000000002A
:10447000D00C040001000000C80C04000100000082
:10448000BC0C040001000000C20C0400010000008C
:10449000526104000000000022D704000000000068
:1044A00000D8040000000000F2D704000000000063
:1044B00080D804000000000072D804000000000052
:1044C000C8C0040000000000F8C0040000000000A4
:1044D0005A780400000000006A7804000000000020
:1044E00080780400000000008879040000000000CB
:1044F000F879040000000000487804000000000083
:104500001A7A0400000000002C7A04000000000069
:10451000747A040000000000E07A0400000000004B
:10452000027B040000000000467C04000000000044
:10453000A87C0400000000001A7D040000000000B8
:104540003E7D04000000000002790400000000002D
:10455000A07D040000000000BE7D040000000000FB
:10456000889FBE008A9FBE00010578000100E00020
:104570000400350008003C000000E000200032008C
:104580000500370060001000E080180002003B00CA
:1045900001F02C001A0037000004BE006011B800C2
:1045A0006B0920000982CF00020039000882CF0089
:1045B0000441B000694252000E00320008003B0086
:1045C00082817100610164008904D1000884D300F4
:1045D0008B05E8000442E800F9FF3A0005003700C7
:1045E0000804440089844C008B05E9000442E9007A
:1045F000FBFF3A00820207000AF0A70001F0A000CA
:104600004F05BE004F04BE0000000600F4FF2F005F
:10461000A1023700140020009F023700889FBE00CF
:104620008A9FBE008C1F7800B6020700BD023300CF
:1046300003866C006450E1002E0032006420E1002B
:10464000330032006150E1002F0032006120E100B0
:104650003100320085855500EB07B00009002000CD
:1046600008042000050037000804440089844C0039
:104670000A0031000603430087834B00000153000A
:1046800081815B00F8FF33000203BE000800A00038
:104690000804440089844C00F6FF3900C639DD0067
:1046A0008301730001003200130020008904D1004F
:1046B0000884D3000998A300050032000800A70071
:1046C0000300A0008904D1000884D3008B05E80012
:1046D0008904D1000884D3000001EB000281D200DC
:1046E0004702070001F0A1000CF0A70001F0A000B4
:1046F000950237006420E100970232000801BE00F5
:104700000200BE00F7FF37006120E1009202320094
:104710006000B800F3FF37000000200001F8270018
:10472000F0FF370003F0A200889FBE008A9FBE0002
:104730008C1F7800730207007A0233006450E10096
:104740004F0032006420E1005200320003826C000E
:1047500007003B000905D0000306D000820F54007B
:104760000C065D0002003900020032008901780069
:10477000030678008582550004003D000003FD001B
:104780008103FD008502EA008B854200840F7200E0
:1047900002003B0060001000E08018006011B800CB
:1047A0000005EB007A28E1000A00390006007800D5
:1047B000C75DDD00F707B200878075002D00370068
:1047C000828171000A017800610560008180D1005A
:1047D0000080D3008502E900F9FF3B000604400099
:1047E0008784480002003B0060041400E0841C0041
:1047F0000988A300070032008A817100828171005C
:10480000610164008904D1000884D3008B05E800AD
:10481000170037000978A30013003A000B00E000EE
:10482000130034008B05E9000804440089844C001F
:104830000A4474000978A3000D003A000B00E00060
:10484000070034008B05E9000804440089844C000B
:1048500001003A000B0020000978A300F7FF3200A6
:104860000001EB0002003700828171000A0178002C
:10487000E30107000CF0A70001F0A00032023700AE
:104880006420E10002003A00838F6C0032023300A2
:104890000801BE000200BE002B023700889FBE0048
:1048A0008A9FBE008C1F7800160207001D0233008D
:1048B00003866C006450E100240032006420E100B3
:1048C000270032006150E100220032006120E10047
:1048D000210032008B854200EB07B1000134B800A3
:1048E000003AB8000804420089844A00013AB8003E
:1048F0000030B8008880400009014A0004003300FD
:104900000000400081804800020149008B05E90059
:10491000C909DD008301700001003200130020008E
:10492000C814DE004814DD004709DE001200B200A2
:10493000C808DE0008847000B101070001F0A10082
:104940000CF0A70001F0A000FF0137006120E1009A
:10495000010232000801BE000200BE00F7FF37006E
:104960006150E100FCFF3A00FB0137000001BE008E
:10497000FC0107000470A70003F0A10003F8A300E6
:1049800013003A006509B10010003200090035003B
:104990006928E10002003500010028000000050040
:1049A00000004000818048008502E900FCFF3A00D9
:1049B00000000600F88F4200050035008100D1009C
:1049C0000080D3008502E800FCFF3A0000000600EA
:1049D0008000EB0000000500889FBE008A9FBE009B
:1049E000030578000300E000050035000B003C00E3
:1049F00000827000040271003000320007003700AE
:104A000060001000E080180060011900E0811900CA
:104A100002003B0001F02D00280037000004BE001A
:104A20000200BE006011B8006B0920009502200052
:104A30000182CF000A0039000541B1000082CF0099
:104A4000070039000541B1000982CF000400390098
:104A50000541B1000882CF00010039000541B100D5
:104A600005425200120032000A003B0082817100B0
:104A7000610164008100D1000080D3008984D300EB
:104A80000884D3008B05E8000442E800F7FF3A00F1
:104A9000070037000804440089844C0000004800E7
:104AA000818048008B05E9000442E900F9FF3A00E3
:104AB000530107000AF0A70001F0A0004F05BE0057
:104AC0004F04BE00000006000003BE00A501070061
:104AD0006011B8000470A70007F0A10007F8A30058
:104AE00017003A006509B1000D0032000D003500D5
:104AF000860220000628E10003003500030028009C
:104B00006000B800020005000000400081804800FD
:104B100002014900838149008502E900FAFF3A0059
:104B200000000600F88F4200050034008100D1002B
:104B30000080D3008502E800FCFF3A000000060078
:104B40006011B8008000EB0000000500881F7800AD
:104B5000000478005001BE004000BE000400400088
:104B6000858048000601490087814900009CBE00FD
:104B70000294BE000400E1000588E1000690E10017
:104B80000798E10002003100680044001008E800C6
:104B90004F04780000000600F4874700889FBE009D
:104BA0008A9FBE008C9FBE008E1F78000205BE004B
:104BB0000004BE00D4B79F00E5B79F00F6B79F0082
:104BC00087BF9F000000EB00C0B79F00B0B79F00F9
:104BD000A0B79F0090B79F0080B79F000D042000F2
:104BE000BFB097004FB09700000140000000E00008
:104BF0000F003D004F08DE0000007100C0B79F00AD
:104C00009E00070001003D0012002000A1000700E7
:104C100001003D0012002000A6000700B1000700BF
:104C2000B60007000F004000C8FF07002200370051
:104C30004F08DE0000067100CCB79F008F00070010
:104C400001003D00120020009200070001003D001D
:104C50001200200097000700A20007000FB2970083
:104C60009FB297002FB39700BFB39700A90007002A
:104C70000000520081805A0002015B0083815B00CA
:104C800080B79F0091B79F00A2B79F00B3B79F0066
:104C90000007EB009F0007000020E10001A8E100F1
:104CA00002B0E10003B8E100010031001E00200065
:104CB0000E005600C0B79F004FB297000400E000FE
:104CC0000700350010002000010020006011B8002E
:104CD00008047000898470000A0571008B857100DA
:104CE0008D06E900BEFF3A000400E00003003D002D
:104CF000820007000F00400094FF07004FA89700B4
:104D00000000E00004003A000FB497009FB4970041
:104D10002FB59700BFB59700940007004F077800A4
:104D20004F06BE004F05BE004F04BE004F01B1004C
:104D300000000600881F780018002000881F7800F7
:104D400095FF07008F87E9004F04780000000600F8
:104D5000801FEB0090FF07008F87E900000006002E
:104D6000889FBE008A9FBE008C1F78006E000700DF
:104D700007003D0073000700E00F5B00E08F5B0061
:104D800007003D00320007000006EB00040037007A
:104D90003400070002003D002A0007001C0020002C
:104DA00072000700E3FF07000203BE000002BE001E
:104DB0000C00E00001003200220007000400BE00E9
:104DC0000601BE004F0678004F05BE004F04BE002E
:104DD00000000600889FBE008A9FBE008C1F7800DE
:104DE0005100070005003D0056000700E00F5B0082
:104DF000E08F5B0006003D0004003700190007004B
:104E000003003D006000B8006011B800100007000A
:104E100056000700CEFF07000203BE000002BE00DE
:104E20000C00E00001003200060007000400BE0094
:104E30000601BE004F0678004F05BE004F04BE00BD
:104E4000000006006000B8006011B80000003700E4
:104E500004025000858258000603590087835900D8
:104E6000000006000006EB00E00F5200E08F5A0041
:104E7000E00F5B00E08F5B00000006000180400057
:104E800090B79F000001EB008FB097000100E00099
:104E9000000006000200700090B79F0001804000F3
:104EA00080B79F000001EB00FFA897000100E00021
:104EB000000006000200700080B79F0001804000E3
:104EC0006FAA9700CF20DE0001007000F0AF9F00B6
:104ED00004024200250007004F18DE0000027200A5
:104EE00000000600E4AF9F000804440089844C00E1
:104EF0000A054D008B854D00000006003FB297006B
:104F0000CFB297005FB39700EFB3970000FE2F007A
:104F1000000006003FB09700CFB097005FB1970048
:104F2000EFB19700000006000205BE000004BE00BD
:104F3000E00F5000E08F5800E00F5900E08F59005B
:104F4000000006006000B8006011B80008045000BE
:104F5000898458000A0559008B8559001C002000DF
:104F6000E00F5200E08F5A00000006000800BE006B
:104F70000A01BE00000006006022B8000602200000
:104F80000000D0008180D2000482D2008582D2004D
:104F90000000A0000202520083825A000300310088
:104FA0000202420083824A000000A1000603E900D9
:104FB000F3FF3A0000000600EFFF07000400BE0008
:104FC00000000600839F68000100E00002003D0031
:104FD00060001000E08018000300E00002003D00C7
:104FE00060011100E0811900E3FF07004F00E000BD
:104FF00002003B0060001000E08018000000060086
:1050000081002000618055000B003D000B00200056
:1050100061FE2F000100E1001D003400828171005B
:10502000610164008904D1000884D3000000E80015
:10503000FAFF3A0071002000610064000300700074
:10504000020060000900320061044400E0844C006A
:105050000988A500050032008B05E8006808E1001A
:1050600002003A008904D1000884D300F20F200026
:105070000258E10005003D00C75DDD00F907B20000
:105080008980750008007800000006000BF82700F2
:105090008B00780000000500889FBE008A9FBE003C
:1050A000841F7800170007004F00780011003300BC
:1050B000F0FF2F00838F6C0006003B0004056500A5
:1050C0000A00A7000800370009F0A6001000200021
:1050D00008003700820F5400838F5C000300390002
:1050E0001000200001003E000000200009F0A70091
:1050F0000000EA004F05BE004F04BE000000E000C3
:10510000000006000004BE00160007000003BE00F9
:105110000405BE000200BE0012000700844F7500A7
:10512000000006000200BE006450E10005003600E9
:105130006420E100020036000968A30001003A0083
:105140000800BE000160A0004F0678004F05BE00B9
:105150004F04BE0000000600F0FF2F00F1FF270003
:10516000F9FF3700C70ADE00F107B200F50FB20001
:1051700008003200E1CF4200020032000170A000BE
:1051800024000500810F70000100320004080500B2
:1051900044000500810F700002003A001400050071
:1051A0008502E9000000400081C04800FCFF3B0090
:1051B0000170A000240005008001EB000200370010
:1051C00061F079008301E800828F5100FCFF3A0012
:1051D000000006003E00000008200000080000005B
:1051E0001B5B0000440000001B5B0000004400004B
:1051F000001B00005B430000001B00005B3200004E
:105200004B0D000000430000000000001B5B00008D
:105210003244000000570000617200006E69000017
:105220006E6700003A2000006E6F000020760000DC
:105230006F6C00007461000067650000206F000063
:105240006E20000056700000756C00006C75000048
:1052500070200000706900006E000000203D00001A
:10526000200000005245000053450000540D00008E
:105270000A000000436C00007574000063680000C1
:10528000206500006E670000616700006564000033
:105290002121000021000000565200004547000077
:1052A000207400006F6F0000206C00006F7700001A
:1052B0002C20000069730000207400006865000065
:1052C000726500002061000020730000686F00001C
:1052D000727400003F000000436C00007574000011
:1052E000636800002064000069730000656E0000C0
:1052F0006761000067650000642100002121000053
:10530000002E0000203C0000002E000020000000C5
:10531000546F000020660000696E00006973000091
:10532000682000007365000074750000702C000098
:10533000207300007461000072740000207500008A
:10534000702000007468000065200000706F00008D
:105350007765000072200000737500007070000017
:105360006C6900006573000020770000697400001C
:1053700068200000636F00006D6D0000616E00002A
:105380006420000027570000270D00000A000000DD
:10539000200000000D0A0000280000007800000036
:1053A000293E0000004200007573000020500000FC
:1053B000697200006174000065200000763400000E
:1053C00000460000697200006D7700006172000005
:1053D00065200000763600002E3300002D620000AC
:1053E000657400006131000020720000323100005D
:1053F0003531000020000000202800003234000079
:10540000464A0000323500003647000042310000B5
:105410003036000020000000413300000041000051
:1054200035000000554E00004B0000002900000030
:1054300043460000473000003A20000000560000BC
:10544000707500003D350000562C00002000000063
:1054500056700000753D000033560000332C0000EC
:105460002000000049090000004F00000900000072
:1054700048090000004C000009000000456E0000D3
:105480007465000072200000726100007720000047
:10549000766100006C75000065200000666F0000FA
:1054A00072200000425200004700000057610000D7
:1054B000726E0000696E0000673A00002061000013
:1054C0006C720000656100006479000020610000DA
:1054D000207600006F6C00007461000067650000BA
:1054E000206F00006E20000056700000756C0000F8
:1054F0006C75000070200000706900006E000000F4
:105500004C450000540000004946000000540000D3
:10551000484500004E000000454C00005345000087
:10552000004700004F5400004F000000474F0000AC
:105530005355000042000000524500005455000041
:10554000524E000000520000454D00000050000087
:10555000524900004E540000004900004E50000027
:1055600055540000004600004F5200000054000057
:105570004F0000004E45000058540000005200004B
:105580004541000044000000444100005441000037
:10559000005300005441000052540000520000002B
:1055A00053540000415200005400000053540000C6
:1055B0004F50000052000000535400004F500000B4
:1055C00000530000454E000044000000524500001A
:1055D000434500004956000045000000434C0000D0
:1055E0004B0000004441000054000000424900000C
:1055F00054520000454100004400000041440000B6
:10560000430000004155000058500000494E000082
:10561000005000005355000000500000554C0000A1
:105620004C55000050000000444500004C41000073
:10563000590000004155000058000000465200008B
:10564000455100000044000055540000590000007E
:105650004D410000435200004F000000454E000045
:105660004400000000520000554E0000004C0000B5
:105670004953000054000000455800004954000000
:10568000004400004542000055470000004E000065
:105690004557000000000000120100000002000059
:1056A0000200000000080000D804000000FB000019
:1056B00002000000010200000301000009020000D6
:1056C00043000000020100000080000064090000A7
:1056D00004000000000100000202000001000000C0
:1056E0000524000000100000010400002402000056
:1056F000020500002406000000010000052400004F
:10570000010100000107000005810000030A0000FC
:10571000004000000904000001000000020A00002F
:105720000000000000070000050200000240000029
:105730000000000007050000820200004000000099
:105740000004000003090000042A000003440000D4
:1057500000610000006E00000067000000650000AE
:1057600000720000006F0000007500000073000070
:10577000002000000050000000720000006F0000D8
:1057800000740000006F0000007400000079000049
:10579000007000000065000000730000001E0000A3
:1057A00003420000007500000073000000200000AC
:1057B000005000000069000000720000006100005D
:1057C000007400000065000000200000005600008A
:1057D0000034000000200000001200000330000030
:1057E00000300000003000000030000000300000F9
:1057F0000030000000300000003100000000000018
:1058000042610000756400002064000065740000BF
:1058100065630000746900006F6E00002073000073
:10582000656C00006563000074650000642E000074
:105830002E0000002000000000000000000000001A
:10584000000000002C0100000000000058020000D1
:1058500000000000B004000000000000600900002B
:1058600000000000C01200000000000080250000C1
:10587000000000004038000000000000004B000065
:105880000000000080700000000000000096000092
:1058900000000000C0DA00000000000000E100008D
:1058A0000000000000C200000100000000F4000041
:1058B0000100000000E80000030000004152000069
:1058C000543100000000000000290000002000000A
:1058D0005700000020520000004E00006F770000CB
:1058E00020750000736900006E670000206F0000E3
:1058F0006E2D0000626F00006172000064200000E5
:1059000045450000505200004F4D00002049000066
:1059100032430000206900006E74000065720000D0
:105920006661000063650000004F00006E2D0000FE
:10593000626F0000617200006420000045450000B5
:10594000505200004F4D00002077000072690000A7
:105950007465000020700000726F00007465000024
:10596000637400002064000069730000616200003D
:105970006C65000064000000493200004331000003
:1059800000000000204800007A000000467200007D
:1059900065710000756500006E63000069650000B8
:1059A000732000003C200000314800007A200000F5
:1059B00061720000652000006E6F0000742000001E
:1059C00073750000707000006F7200007465000055
:1059D000642E000000000000306200000030000073
:1059E000303000002C00000030300000003000009B
:1059F0003132000033340000353600003738000003
:105A00003941000042430000444500004630000098
:105A100078000000436F0000756C0000646E0000A9
:105A200027740000206B00006565000070200000F6
:105A30007570000000000000535000004931000064
:105A40000000000029000000007500006E6B0000DF
:105A50006E6F0000776E0000206D00006F64000024
:105A600065000000504900004331000000000000C4
:105A70003A200000000000002E0000003157000016
:105A8000303100000000000042420000494F000099
:105A900031000000585300005631000000000000A3
:105AA000314100004C5300000042000050760000DD
:105AB000340000000808000008080000080000008A
:105AC00000000000524100005731000000000000BB
:105AD0004E4F0000454D0000530000000000000044
:105AE000290000000000000000000000200000006D
:105AF000000000002A00FA000000EB00700F980080
:105B00000000EB00109889000000EB00009889006D
:105B100000988100300798000000EB0020079800F3
:105B20000000EB00100798000000EB00B07F890038
:105B30000000EB00600798000000EB00209889004F
:105B40000000EB00500798000000EB00100F9800D9
:105B5000130037000000EB00700798000A003700C0
:105B60001E089000FE0090004500DD00010140008D
:105B7000613023000040EB0000F178007E009000CF
:105B80000000E800700798007E009000FF0F5000B2
:105B9000F3FF34001E0890000000E800100F98008A
:105BA0001E089000E40F5000EAFF34000000EB00F4
:105BB000309D8900B17F8100000320000088B9007A
:105BC0008102200080804000C0C62200008040008A
:105BD00098DB020000000000E17F8100002020002F
:105BE000008060000000E00004003200710020002E
:105BF00040652000E603020001000000A08E2A009C
:105C000098DB02000000000025043700309D810071
:105C10000000E0005F003200309D81000000E900DC
:105C2000309D89000000EB00700798001B003700D2
:105C300002988100309D8100FE0090004500DD004B
:105C40008100400060302300E14078000020230004
:105C500001717800309D8100FE0090004500DD005C
:105C60008100400060302300614078008EDF020038
:105C700000000000009881000000E8000098890002
:105C80007E0090000000E8007007980001988100F5
:105C9000F00F20000080600000988900309D810096
:105CA000FE0090004500DD008100400060302300D0
:105CB000614078000004E000DDFF3A000000EB00E6
:105CC000309D890033003700E05D230010407800EC
:105CD000644060000004E0002D003200B17F8100CC
:105CE000000320000088B900FA004000C0C622006E
:105CF0000080400010007800000001000000E0007B
:105D000023003200B17F8100000320000088B90029
:105D10008102200080804000C0C622000080400038
:105D200098DB020000000000A08E2A0098DB020031
:105D3000000000001198810000988100808F5000C1
:105D40001300320010988100700798000C00370093
:105D5000FE00900000202300614078008EDF0200EA
:105D600000000000FE009000F00F200000806000A6
:105D7000700798007E0090000000E800700798000F
:105D8000FE00900000988100808F5000F0FF3A00E4
:105D9000D3C2BF00C4DF0200000000000004E00026
:105DA000C9FF320002E00200000000000004E00031
:105DB0000300320016E0020000000000B8033700C4
:105DC000ECDF020000000000005798000E50900029
:105DD0000080FB006101B90012179800231798009A
:105DE000F0072000010020001E119000AE1190006D
:105DF000800F5100818F59003C033E001E1090001F
:105E0000AE109000006001002D033700E302370060
:105E10004D01370035033700D3003700FA02370051
:105E20006201370031033700770037002F03370056
:105E3000100337002D0337002C0337000D03370004
:105E400007023700290337006901370027033700AD
:105E500026033700250337002403370023033700C8
:105E60002203370021033700200337001F033700C8
:105E70001E033700F90037001C0337001B033700EF
:105E80001A033700190337001803370017033700C8
:105E900016033700150337001403370013033700C8
:105EA0001203370011033700100337000F033700C8
:105EB0000E0337000D0337000C0337000B033700C8
:105EC0000A033700090337000803370007033700C8
:105ED00006033700050337000403370003033700C8
:105EE000020337000103370000033700FF023700C9
:105EF000FE023700FD023700FC023700FB023700CC
:105F0000FA023700F9023700F8023700F7023700CB
:105F1000F6023700F5023700F4023700F3023700CB
:105F2000F2023700F1023700F0023700EF023700CB
:105F3000EE023700ED023700EC023700EB023700CB
:105F4000EA023700E9023700E8023700E7023700CB
:105F5000E6023700E5023700E4023700E3023700CB
:105F6000E2023700E1023700E0023700DF023700CB
:105F7000DE023700DD023700DC023700DB023700CB
:105F8000DA023700D9023700D8023700D7023700CB
:105F9000D6023700D5023700D4023700D3023700CB
:105FA000D2023700D1023700D0023700CF023700CB
:105FB000CE023700CD023700CC023700CB023700CB
:105FC000CA023700C9023700C8023700C7023700CB
:105FD000C6023700C5023700C4023700C3023700CB
:105FE000C2023700C1023700C0023700BF023700CB
:105FF000BE023700BD023700BC023700BB023700CB
:10600000BA02370058003700119881003E00900016
:10601000810F500050003200019881003E00900036
:10602000810F50000F003A00009881008000E900C5
:10603000F00F200000806000009889000298810025
:10604000012023000040EB0000F17800019881005E
:1060500031079800C08E2A0098DB02000000000083
:106060000F0337000000EB00100F98003E00900077
:106070008000E900F00F20000080600030079800E9
:10608000008F2A0098DB0200000000003E01900013
:10609000720798001D0037007E0190007E0090007E
:1060A0008000E80000202300E14078000020230069
:1060B00001717800FE00900000202300614078000C
:1060C0000004E000060032007E0090000120230062
:1060D00060C078008EDF020000000000030037007F
:1060E00000C2B3008EDF0200000000001E08900016
:1060F0000000E800100F98007E0090008000E8008B
:10610000F00F20000080600070079800FE009000F3
:1061100000988100808F5000DFFF3A0000988100D6
:106120008000E900F00F20000080600000988900E6
:10613000408F2A0098DB0200000000001E0890003B
:1061400030DE020000000000708F2A0098DB0200A1
:1061500000000000D202370070C0B3008EDF0200E2
:1061600000000000CE023700019881003E00900040
:10617000810F5000350032000000EB00100F980036
:10618000BE019000730798001D0037007E0190004B
:106190007E0090008000E80000202300E1407800AD
:1061A0000020230001717800FE00900000202300F1
:1061B000614078000004E000060032007E0090009C
:1061C0000120230060C078008EDF02000000000084
:1061D0000300370000C2B3008EDF020000000000A1
:1061E0001E0890000000E800100F98007E0090004C
:1061F0008000E800F00F2000008060007007980029
:10620000FE00900000988100808F5000DFFF3A0070
:10621000009881008000E900F00F200000806000FD
:1062200000988900408F2A0098DB020000000000DF
:106230001E08900030DE020000000000708F2A006F
:1062400098DB0200000000009502370070C0B30028
:106250008EDF02000000000091023700ECDF020038
:1062600000000000005798008E509000B0C5B300A9
:1062700080CF50008A023A00ECDF020000000000EC
:10628000005798000E5090000080FB000017980007
:10629000100420008E109000808F500054003200B7
:1062A000100420000E119000800F510009003C00E6
:1062B000100320008E119000808F510012003200D8
:1062C000400320008E109000808F50001600320096
:1062D00073023700300420000E119000800F51002F
:1062E00032003200300420008E119000808F510067
:1062F000DB003500400420008E109000808F50009D
:106300001100320066023700ECDF020000000000DE
:10631000005798008E509000E0C7B30080CF500027
:106320009E0132005E023700ECDF02000000000038
:10633000005798008E509000E0C7B30080CF500007
:10634000B1013200560237005E009000E40F5000A9
:1063500005003400D0EB0200000000000000EB005C
:10636000500798004E023700119881003E009000BF
:10637000810F5000090032003E0090008000E900CB
:10638000F00F20000080600030079800008F2A0086
:1063900098DB0200000000004102370070C0B3002B
:1063A0008EDF0200000000003D02370001988100EE
:1063B0003E009000810F5000090032003E00900026
:1063C0008000E800F00F2000008060003007980097
:1063D000908F2A0098DB0200000000003002370096
:1063E00070C0B3008EDF0200000000002C023700F6
:1063F0000000EB0010079800109881000000E900F1
:1064000080007800F00F2000008060007007980086
:10641000870037007E0090000120230060C07800D4
:106420000004E0007D003A007E0090008000E9005A
:10643000F00F200080806000002023006140780081
:106440000004E000750032001E0090000000E8002B
:10645000100798009E0090002E009000808F500042
:106460006E0036002E0090000000E8002007980023
:106470001198810000988100808F50001200320036
:106480000900370002988100012023000040EB0042
:1064900000F17800009881008000E900F00F2000F2
:1064A00000806000009889000198810010988100A8
:1064B000808F5000F3FF3A000298810001202300F2
:1064C0000040EB0000F178007E0090008000E900C1
:1064D000F00F200000806000100F980010003700BF
:1064E0001E0890000120230060C078000004E00036
:1064F00006003A001E0890008000E800F00F20001F
:106500000080600060079800090037001E089000B6
:106510008000E900F00F200000806000100F98005C
:106520009E08900000988100808F5000ECFF3A0098
:10653000D08F2A0098DB020000000000B17F8100AC
:10654000000320000088B900810220008080400004
:10655000C0C622000080400098DB0200000000005E
:10656000E17F810000202000008060000000E0004A
:10657000040032007100200040652000E6030200A4
:1065800001000000A08E2A0098DB0200000000003D
:106590006E019000120F9800150037009E089000C1
:1065A00000202300614078008EDF02000000000020
:1065B000029881009E08900000202300E1407800AE
:1065C0000020230001717800009881008000E8001D
:1065D000F00F200000806000009889001E089000E5
:1065E0008000E800F00F200000806000100F98008D
:1065F0009E0890007E009000808F5000E7FF3A00D8
:1066000002988100012023000040EB0000F1780097
:106610000398810033079800090037007E0090003E
:106620008000E900F00F20000080600070079800F3
:10663000FE00900000988100808F500075FF3A00A6
:10664000FE00900000988100808F500094013A0075
:1066500070C0B3008EDF0200000000009001370020
:106660000000EB0010079800109881000000E9007E
:1066700080007800F00F2000008060007007980014
:10668000880037007E0090000120230060C0780061
:106690000004E0007E003A007E0090008000E900E7
:1066A000F00F20008080600000202300614078000F
:1066B0000004E000760032001E0090000000E800B8
:1066C000100798002E0090008000E9001E00900046
:1066D000808F50006E003A002E0090000000E9000C
:1066E000200798001198810000988100808F500049
:1066F00012003200090037000298810001202300B7
:106700000040EB0000F17800009881008000E90073
:10671000F00F20000080600000988900019881003F
:1067200010988100808F5000F3FF3A00029881009A
:10673000012023000040EB0000F178007E00900073
:106740008000E900F00F200000806000100F98002A
:10675000100037001E0890000120230060C0780060
:106760000004E00006003A001E0890008000E800E7
:10677000F00F2000008060006007980009003700DB
:106780001E0890008000E900F00F200000806000EB
:10679000100F98009E08900000988100808F500094
:1067A000ECFF3A00D08F2A0098DB020000000000C6
:1067B000B17F8100000320000088B9008102200021
:1067C00080804000C0C622000080400098DB0200AC
:1067D00000000000E17F81000020200000806000B8
:1067E0000000E0000400320071002000406520003D
:1067F000E603020001000000A08E2A0098DB0200E0
:10680000000000006E009000100F98001500370087
:106810009E08900000202300614078008EDF020077
:1068200000000000029881009E08900000202300D4
:10683000E140780000202300017178000098810079
:106840008000E800F00F20000080600000988900C0
:106850001E0890008000E800F00F2000008060001B
:10686000100F98009E0890007E009000808F5000CE
:10687000E7FF3A0002988100012023000040EB006E
:1068800000F1780001988100310798000900370075
:106890007E0090008000E900F00F20000080600082
:1068A00070079800FE00900000988100808F5000D3
:1068B00074FF3A00FE00900000988100808F500025
:1068C000F7003A002E009000E10F50002F003A0030
:1068D000D08F2A0098DB020000000000B17F810009
:1068E000000320000088B900810220008080400061
:1068F000C0C622000080400098DB020000000000BB
:10690000E17F810000202000008060000000E000A6
:10691000040032007100200040652000E603020000
:1069200001000000A08E2A0098DB02000000000099
:106930000900370002988100012023000040EB008D
:1069400000F17800009881008000E900F00F20003D
:1069500000806000009889000198810010988100F3
:10696000808F5000F3FF3A0002988100012023003D
:106970000040EB0000F17800029881003207980097
:106980000000EB0020079800C500370070C0B3007E
:106990008EDF020000000000C10037001198810066
:1069A0003E009000810F50001300320011988100CA
:1069B0003E0090000100500080007800F00F2000A1
:1069C00000806000100F9800408F2A0098DB0200C2
:1069D000000000001E08900030DE020000000000F1
:1069E000708F2A0098DB02000000000013988100DD
:1069F00033079800AA00370070C0B3008EDF020092
:106A000000000000A6003700019881003E009000C1
:106A1000810F500013003200019881003E00900069
:106A20000080500080007800F00F2000008060009F
:106A3000100F9800408F2A0098DB02000000000031
:106A40001E08900030DE02000000000030902A0096
:106A500098DB0200000000000098810030079800D9
:106A60008F00370070C0B3008EDF0200000000000E
:106A70008B00370010002000700F98000000EB0022
:106A80002007980002988100012023000040EB00BD
:106A900000F17800009881008000E800F00F2000ED
:106AA00000806000009889000198810031079800FB
:106AB00050902A00C4DB020000000000780037007C
:106AC0005E0090000000E800500798005E00900013
:106AD000F40F500072003A00FCD0020000000000E9
:106AE0000000EB00500798000B023700009881006F
:106AF0008000E800F00F2000808060001098810086
:106B0000808F5000630032000E509000FF4F500005
:106B1000600036008E509000E0C7B30080CF500078
:106B20005C003E00019881003E009000808F500084
:106B300013003A000E5090008EDF020000000000AB
:106B4000029881008E50900000202300017178008F
:106B5000009881008000E800F00F200000806000B5
:106B60000098890002988100012023000040EB007A
:106B700000F1780002988100320798004800370041
:106B8000019881003E009000008050008000780055
:106B9000F00F200000806000100F9800408F2A0046
:106BA00098DB0200000000001E08900030DE0200AA
:106BB0000000000030902A0098DB02000000000076
:106BC0000098810070079800190037007E0090003F
:106BD0000001E800FE00900000202300E140780062
:106BE0000020230001717800FE00900000202300A7
:106BF000614078000004E000080032007E00900050
:106C00000120230060C078008EDF02000000000039
:106C100060902A0098DB0200000000007E009000D7
:106C20008000E900F00F20000080600070079800ED
:106C30007E0190003E0090008000E900F00F2000EF
:106C400000806000800F5100E0FF3A000E5090007D
:106C50008EDF0200000000003E0190008E50900088
:106C600000202300017178003E0090008000E800C1
:106C7000F00F20000080600030079800009881002D
:106C80008000E800F00F200000806000009889007C
:106C90000300370070C0B3008EDF02000000000068
:106CA0007E0890000000E000D8FB320000988100D0
:106CB000500F980010988100400F98000000EB00E2
:106CC000700F98000000EB00600F98000000EB00D0
:106CD00020988900E17F8100002020000080600072
:106CE0000000E00008003200005E0200000000002A
:106CF00051002000B0652000700402000100000077
:106D000010002000600F98000040EB001047980032
:106D10000040EB00004F78003305370011988100E8
:106D20000020230061407800005798000E5090002A
:106D30000080FB006101B9003217980043179800EA
:106D4000E0072000010020003E119000CE119000CD
:106D5000800F5100818F5900F7043E003E109000D3
:106D6000CE10900000600100F5043700F2043700F7
:106D7000F1043700F0043700EF043700EE04370069
:106D8000ED043700EC043700EB043700EA04370069
:106D9000EB043700E8043700E7043700E804370065
:106DA000E5043700E4043700E3043700E204370069
:106DB000E1043700E0043700DF043700DE04370069
:106DC000DD043700DC043700DB043700DA04370069
:106DD000D9043700D8043700D7043700D604370069
:106DE000D5043700D4043700D5043700B204370087
:106DF000EB02370045013700490137000A0237002E
:106E0000F8013700CC043700C5023700CA04370048
:106E1000C9043700CA043700C90437005E043700CC
:106E200077043700420437005F0337005E03370002
:106E30005D0337005C0337005B0337005A033700FC
:106E400059033700580337005703370056033700FC
:106E5000B9043700B804370013023700E3003700E5
:106E6000B5043700470037005B0137004D0137009C
:106E7000B10437006C003700D7013700AE0437008B
:106E8000AD043700AC043700AB043700AA04370068
:106E9000A90437007800370081003700A6043700C6
:106EA000A5043700A4043700A7003700A204370068
:106EB000A1043700F10137009F0437009E0437001A
:106EC0009D0437005A0137009B0437009A043700AD
:106ED00099043700100337002204370020033700DD
:106EE0005604370039043700930437002001370077
:106EF0002F00370042003700A9013700B9003700E2
:106F0000310037003300370016003700200037000B
:106F1000890437004E0037006D003700220037002B
:106F200085043700240037007500370082043700DD
:106F300097033700CD0137007F0437007E04370008
:106F40001F003700780137007B0437007A043700D0
:106F500079043700F9023700BF0037000903370012
:106F6000DD003700540707000000E00074043A0019
:106F700010988100400F980000988100500F9800F1
:106F80006F04370086040200010000006C04370023
:106F90008E090700B07F81000000E0006804320025
:106FA000C409070066043700B70607006404370009
:106FB000380B070062043700120B0700600437002B
:106FC0007E0A07005E0437000A810200000000000C
:106FD0005B043700B07F81000000E00005003A004C
:106FE000D1012000B0682000700402000100000000
:106FF00053043700747F0200000000005004370083
:10700000E15D2300114078000000A1000010A10004
:1070100080487800610120000066200070040200B2
:107020000100000046043700E15D230011407800B4
:107030000000A0000010A10080487800510120004D
:107040006067200070040200010000003C0437006B
:10705000E15D2300114078000000A1000010A000B5
:107060008048780071012000B045210070040200C2
:107070000100000032043700E15D23001140780078
:107080000000A0000010A0008048780071012000DE
:10709000204721007004020001000000280437008E
:1070A000E15D2300114078000030A00080487800A6
:1070B000C1012000408D2000E60302000100000015
:1070C00050902A00C4DB0200000000001C043700BE
:1070D000E15D2300114078000030A1008048780075
:1070E000B1012000908B2000E603020001000000A7
:1070F00050902A00C4DB020000000000100437009A
:10710000B07F81000000E00005003A00D1012000BE
:10711000B06820007004020001000000080437007D
:10712000E282A900E082A90051012000806A2000CB
:10713000E60302000100000050902A00C4DB0200B8
:1071400000000000FE033700B07F81000000E00077
:1071500005003A00D1012000B06820007004020050
:1071600001000000F6033700E05D230010407800C6
:10717000704060000004E00004003A00210220009A
:10718000D0FB20007004020001000000E082A80093
:10719000E282A90041012000D06B2000E60302003A
:1071A0000100000050902A00C4DB02000000000033
:1071B00021E3A80050C0B3003E000200010000001F
:1071C00080007800F0042000808F500003003E0013
:1071D000B0902A00C4DB02000000000021E3A900F7
:1071E000D7033700030B0700D50337001098810041
:1071F0008000E800F00F20000080600010988900F7
:107200001206070002040700700798007E00900035
:1072100092DE020000000000E0922A0098DB0200EB
:10722000000000007E00900030DE02000000000040
:10723000E0922A0098DB0200000000007E0090002F
:10724000F8DB02000000000050902A00C4DB0200BE
:1072500000000000BA033700109881008000E800A9
:10726000F00F20000080600010988900F7050700EB
:10727000E7030700700798007E0090000080FB0085
:10728000D001020001000000700798007E0090000D
:1072900092DE020000000000E0922A0098DB02006B
:1072A000000000007E00900030DE020000000000C0
:1072B000E0922A0098DB0200000000007E009000AF
:1072C000F8DB02000000000050902A00C4DB02003E
:1072D000000000009A033700B07F81000000E0004A
:1072E00005003A0011C0B30010C0B30058F6020008
:1072F0000000000092033700A1012000106D200063
:1073000070040200010000008D03370020932A0062
:1073100098DB020000000000AC080700880337007B
:1073200016050200010000000000E00084033200A6
:10733000A1002000006F2000700402000100000086
:10734000400620006E01020001000000B0FF0200B4
:1073500000000000BCDF0200000000000004E000AC
:10736000FCFF320081BF2A00014001007403370096
:107370002C0507000000E800100F980002003700FD
:1073800062890200000000001E0890000000E90071
:10739000100F98001E0890000000E000F8FF3A006F
:1073A000670337001F0507000000E800100F980072
:1073B0000200370012890200000000001E08900041
:1073C0000000E900100F98001E0890000000E00087
:1073D000F8FF3A005A033700120507000000E800E2
:1073E000100F98000B00370061012000A06F2000F3
:1073F000E603020001000000B28902000000000064
:1074000082DB02000000000050902A00C4DB020072
:10741000000000001E0890000000E900100F980016
:107420001E0890000000E000EFFF3A004403370020
:10743000B07F81000000E00005003A00D10120008B
:10744000B068200070040200010000003C03370017
:10745000C922A900CB22A80021E3A8002000200017
:107460006E010200010000000040EB003E0002003F
:107470000100000080007800001B2000808F500079
:107480001B00360020C0B3003E00020001000000D7
:1074900080007800702B2000808F50001400360090
:1074A0001101200000712000E6030200010000002D
:1074B00050902A00C4DB020000000000B17F810070
:1074C000000320000088B9000102200080804000F5
:1074D000C0C62200008040001000780000000100BB
:1074E000A0932A00C4DB0200000000000C0037005B
:1074F000C922A900CB22A900C0942A00C4DB020043
:10750000000000002101200010722000E6030200AC
:107510000100000050902A00C4DB020000000000BF
:1075200021E3A90006033700B07F81000000E000DE
:1075300005003A00D1012000B0682000700402006C
:1075400001000000FE023700B17F8100000320002F
:107550000088B9002102200080804000C0C62200BF
:10756000008040001000780000000100C0962A0052
:10757000C4DB020000000000C922A900CB22A90040
:107580002101200010722000E6030200010000002B
:1075900050902A00C4DB020000000000E80237001F
:1075A000F1002000C0362000E603020001000000C8
:1075B000580002000100000011002000B037200038
:1075C000E60302000100000050902A00C4DB020024
:1075D00000000000DA0237006A000200010000002B
:1075E000D70237008F040700100F980061002000B9
:1075F000F0732000E6030200010000001E08900066
:10760000D2DD0200000000002100200050742000A4
:1076100070040200010000001E0890009A010200A0
:1076200001000000C60237007E040700100F98001A
:1076300061002000F0732000E6030200010000005A
:107640001E089000D2DD0200000000002100200092
:107650001000210070040200010000001E089000CC
:107660006E01020001000000B5023700E07F8100DA
:107670000090A000E07F8900B1023700B07F810058
:107680000000E00005003A00D1012000B0682000B1
:107690007004020001000000A9023700248A0200E1
:1076A00000000000A602370010002000209889008A
:1076B00010002000700798000F003700119881001B
:1076C0007E00900080804000F00F200080806000ED
:1076D00000202300E1407800E0C3B30080CF5000D9
:1076E00002003A000000EB00209889007E00900024
:1076F0000000E80070079800119881007E0090005B
:1077000080804000F00F2000808060000020230077
:10771000614078000004E000E8FF3A00FE009000BD
:1077200020022000808F5000020034001000200052
:1077300020988900209881000000E00080023A0033
:10774000109881008000E800F00F200000806000A9
:1077500010988900AE020700700798001198810008
:10776000F00F20008080600000202300E1407800BE
:10777000D0C3B30080CF50003C003A007E009000A0
:107780000000E000360034007E009000E50F50005D
:1077900033003C00109881008000E800F00F2000CA
:1077A00000806000109889007E0090000000E900D1
:1077B000700798000000EB00100F98000A003700D7
:1077C0007E0090009E0890004500DD000101400011
:1077D000613023000040EB0000F178001E089000AB
:1077E0000000E800100F98001E089000FF0F5000E6
:1077F000F3FF34000000EB00100F98001100370079
:107800007E0190009E0990001198810000202300C5
:10781000614278004510DD008300400060302300A5
:10782000847078001E0890000000E800100F980097
:10783000109881008000E800F00F200000806000B8
:10784000109889001198810000202300E140780001
:10785000E0C3B30080CF5000E9FF3A0038023700A0
:107860001000200020988900350237007E0090002B
:107870000000E0001B003A000000EB00100F980031
:10788000140037001E0890000040E80030DE0200BF
:107890000000000010982A0098DB020000000000A1
:1078A0001E0890004500DD00800078006030230055
:1078B0000080400098DB020000000000A08E2A003B
:1078C000C4DB0200000000001E0890000000E80079
:1078D000100F98001E089000E40F5000E9FF3400DC
:1078E000170237007E0090000000E000090034001D
:1078F0007E009000E50F500006003C0050902A00EA
:10790000C4DB020000000000FE009000319D8900F1
:107910000B02370010002000209889000802370071
:10792000109881008000E800F00F200000806000C7
:107930001098890036020700300F980043040700B2
:1079400011988100F00F200080806000002023004B
:10795000E140780090C2B30080CF50000D003A00A3
:10796000B17F8100000320000088B900FC004000C6
:10797000C0C6220000804000900078003E089000C1
:107980000100010050902A00C4DB0200000000004A
:10799000EB0137001000200020988900E801370033
:1079A0001000200020988900100020007007980027
:1079B0000F003700119881007E0090008080400009
:1079C000F00F20008080600000202300E14078005C
:1079D00020C2B30080CF500002003A000000EB004C
:1079E000209889007E0090000000E8007007980051
:1079F000119881007E00900080804000F00F2000F0
:107A00008080600000202300614078000004E000D6
:107A1000E8FF3A00209881000000E000C8013A0029
:107A20007100200070742000E603020001000000D5
:107A300020C2B3008EDF02000000000020003700EB
:107A400011988100F00F20000080600010988900DC
:107A50001198810000202300614078008EDF020031
:107A60000000000011988100002023006140780090
:107A70000000FB00300F9800E05D2300104078000C
:107A8000684060000004E000040032003E089000FE
:107A9000D001020001000000300F9800B17F81008A
:107AA000000320000088B900E8004000C0C62200A2
:107AB00000804000900078003E0890000100010026
:107AC000109881000000E80010988900119881004A
:107AD000F00F20008080600000202300E14078004B
:107AE00020C2B30080CF5000D5FF3A00109881002B
:107AF000F10F2000010060001098890020C2B3003F
:107B00008EDF02000000000050902A00C4DB02005B
:107B1000000000008A013700B17F810000032000CF
:107B20000088B90080007800C0C6220000804000B4
:107B3000100078000000010081013700B17F810052
:107B4000000320000088B9008080E800C0C6220041
:107B5000008040001000780000000100780137002C
:107B6000B17F8100000320000088B900E4004000DC
:107B7000C0C6220000804000100078000000010014
:107B80006F013700B17F8100000320000088B90039
:107B9000E6004000C0C622000080400010007800CF
:107BA00000000100660137007100200070742000A1
:107BB000E60302000100000095010700300F980065
:107BC000109881000000E900109889001198810048
:107BD000F00F20000080600010988900110307005A
:107BE0000000E800100F98003003070040079800DD
:107BF0004E0090000000E0005B0032004E0090005C
:107C000080407800D05C2300014878004E0090004E
:107C1000E80F500005003400E15D230011407800BA
:107C20000050A000804878004F003700E15D23003D
:107C3000114078000050A100804878004A003700C9
:107C40003E089000C800020001000000E05D230033
:107C5000104078000042B2000004E00004003A0046
:107C6000D05C230010407800E84F500009003A0033
:107C7000E05D2300104078000042B2000004E00004
:107C80000B003200D05C230010407800F04F500011
:107C900007003200B0C3B3008EDF02000000000016
:107CA000D05C23001040780030DE020000000000AD
:107CB000E05D230010407800684060000004E000B0
:107CC000040032003E089000D001020001000000D4
:107CD000300F9800B17F8100000320000088B900B8
:107CE000E8004000C0C622000080400090007800FC
:107CF0003E08900001000100200F980000C2B30070
:107D00008EDF020000000000E05D230010407800DC
:107D10000044B2000004E0001300320061002000C3
:107D2000E0742000E603020001000000E05D230093
:107D300010407800684060000004E0000400320059
:107D40002E089000D001020001000000200F9800D2
:107D50002E089000C80002000100000000C2B3001D
:107D60008EDF0200000000001E0890000000E90005
:107D7000100F98001E0890000000E000B0FF3A00CD
:107D800050902A00C4DB020000000000EC00370025
:107D900061002000E0742000E60302000100000002
:107DA000E0020700004F78009E0207000000E80094
:107DB000100F9800BD020700400798004E00900089
:107DC0000000E000100032004E009000804078007B
:107DD000D05C2300014878004E009000E80F50006E
:107DE00005003400E15D2300114078000050A00040
:107DF0008048780004003700E15D230011407800DE
:107E00000050A100804878001E04E00037003200D6
:107E1000A07F8100104798001E80FB000000E90051
:107E2000A07F890031003700B17F8100000320006E
:107E30000088B900EA004000C0C62200008040006F
:107E40001000780000000100200F9800E05D230082
:107E500010407800684060000004E0000400320038
:107E60002E089000D001020001000000200F9800B1
:107E70002E089000C800020001000000E05D230011
:107E8000104078000042B2000004E00004003A0014
:107E9000D05C230010407800E84F500009003A0001
:107EA000E05D2300104078000042B2000004E000D2
:107EB0000B003200D05C230010407800F04F5000DF
:107EC00007003200B0C3B3008EDF020000000000E4
:107ED000D05C23001040780030DE0200000000007B
:107EE00000C2B3008EDF0200000000001E089000F8
:107EF0000000E900100F98001E0890000000E0004C
:107F0000C9FF3A001E04E000050032001E40900048
:107F10000080FB00A07F89000040EB00004F78004C
:107F200050902A00C4DB02000000000084003700EB
:107F30008100200040752000700402000100000054
:107F4000B17F8100000320000088B900EC004000F0
:107F5000C0C6220000804000100078000000010030
:107F60007700370081002000C075200070040200F7
:107F700001000000B17F8100000320000088B900EB
:107F8000EE004000C0C622000080400010007800D3
:107F9000000001006A003700E10020004076200068
:107FA0007004020001000000B17F81000003200086
:107FB0000088B900F0004000C0C6220000804000E8
:107FC00010007800000001005D003700E100200093
:107FD000207720007004020001000000B17F8100C2
:107FE000000320000088B900F2004000C0C6220053
:107FF00000804000100078000000010050003700B1
:10800000C100200030732000E603020001000000E0
:10801000B17F8100000320000088B900F400400017
:10802000C0C622000080400010007800000001005F
:1080300082DB02000000000041003700F901070068
:10804000100F9800D100200000792000E603020004
:10805000010000001E089000C8000200010000009E
:108060001E0890000000E800100F9800080037007C
:10807000B17F8100000320000088B900F6004000B5
:10808000C0C62200008040001000780000000100FF
:108090001E0890000000E900100F98001E089000D4
:1080A0000000E000F2FF3A0050902A00C4DB02001A
:1080B0000000000022003700DA0107000000E8009D
:1080C000100F9800A1002000D0792000E6030200E4
:1080D000010000000D003700B17F81000003200087
:1080E0000088B900F8004000C0C6220000804000AF
:1080F000100078000000010082DB02000000000098
:1081000000C2B3008EDF0200000000001E089000D5
:108110000000E900100F98001E0890000000E00029
:10812000EDFF3A00010120000078200070040200F9
:108130000100000002003700100020002098890094
:10814000109881008000E800F00F2000008060009F
:1081500010988900209881000000E0001C00320087
:1081600051012000707A2000E603020001000000A7
:10817000CE08900010988100808F500007003100D9
:1081800010988100804078004E08900000C0500098
:1081900030DE020000000000060037001098810069
:1081A000804078004E08900000C0500030DE020091
:1081B000000000000000EB00209889001000200063
:1081C000600F980050902A00C4DB020000000000FD
:1081D0001198810000988100808F500002003A00C1
:1081E00010002000600F98006E0890000000E00072
:1081F000CAFA32005E089000109889005E0890006C
:10820000009889000000EB00700F980069F63700B5
:108210000600FA000000EB00100798000000EB00D9
:10822000000F7800119881001E00900080804000AF
:10823000F00F20008080600000202300E1407800E3
:1082400000C3B30080CF50003E003400119881007D
:108250001E00900080804000F00F200080806000B1
:1082600000202300E140780090C3B30080CF50008D
:1082700034003C00119881001E0090008080400076
:10828000F00F200080806000002023006140780013
:108290008000FB0000FD2F00008F40001E009000BA
:1082A0000000E80010079800110037001E00780059
:1082B0006A00B900000F7800119881001E0090003C
:1082C00080804000F00F20008080600000202300AC
:1082D000614078000000FB009E00400000FD2F0080
:1082E000008F40001E0090000000E800100798007A
:1082F000119881001E00900080804000F00F200047
:108300008080600000202300E1407800F0C2B300CC
:1083100080CF500036013400119881001E0090007B
:1083200080804000F00F200080806000002023004B
:10833000E140780090C3B30080CF5000DBFF3400F1
:108340002B013700119881001E00900080804000B2
:10835000F00F20008080600000202300E1407800C2
:1083600000C3B30080CF50001C013A001E009000F3
:108370000000E80010079800119881001E0090008E
:1083800080804000F00F20008080600000202300EB
:10839000E140780020C6B30080CF50000A003200D0
:1083A000119881001E00900080804000F00F200096
:1083B0008080600000202300E140780020C4B300EA
:1083C00080CF50002A003A001E0090000000E80014
:1083D00010079800110037001E00780000004000D0
:1083E000000F7800119881001E00900080804000EE
:1083F000F00F2000808060000020230061407800A2
:108400000000FB009E00400000FD2F00008F400098
:108410001E0090000000E8001007980011988100ED
:108420001E00900080804000F00F200080806000DF
:1084300000202300E140780010C3B30080CF50003B
:10844000E5FF3200119881001E00900080804000FE
:10845000F00F20008080600000202300E1407800C1
:1084600000C3B30080CF5000DBFF3200E0003700D4
:10847000119881001E00900080804000F00F2000C5
:108480008080600000202300E140780080C7B300B6
:1084900080CF50000A003200119881001E00900029
:1084A00080804000F00F20008080600000202300CA
:1084B000E140780080C5B30080CF500082003A00D0
:1084C0001E0090000000E8001007980041003700EF
:1084D0001E0078004400DD00000F78001198810034
:1084E0001E00900080804000F00F2000808060001F
:1084F00000202300E1407800F0C2B30080CF50009C
:1085000016003400119881001E0090008080400009
:10851000F00F20008080600000202300E140780000
:1085200090C3B30080CF50000C003C001198810034
:108530001E00900080804000F00F200080806000CE
:1085400000202300614078000000FB009E004000F6
:1085500000FD2F00008F40001B00370011988100A4
:108560001E00900080804000F00F2000008160001D
:10857000119881001E00900080804000F00F2000C4
:108580008080600000202300E140780000C2B3003A
:1085900080C07000002023000171780011988100D4
:1085A0001E00900080804000F00F2000808060005E
:1085B00000202300614078000000FB009E00400086
:1085C00090FA2F00008F40001E0090000000E8008D
:1085D00010079800119881001E00900080804000D4
:1085E000F00F20008080600000202300E140780030
:1085F000F0C2B30080CF50000A003400119881000F
:108600001E00900080804000F00F200080806000FD
:1086100000202300E140780090C3B30080CF5000D9
:10862000ABFF3400119881001E0090008080400054
:10863000F00F20008080600000202300E1407800DF
:1086400000C4B30080CF50000A00340011988100AC
:108650001E00900080804000F00F200080806000AD
:1086600000202300E140780060C4B30080CF5000B8
:1086700097FF3400119881001E0090008080400018
:10868000F00F20008080600000202300E14078008F
:1086900000C6B30080CF500055003400119881000F
:1086A0001E00900080804000F00F2000808060005D
:1086B00000202300E140780060C6B30080CF500066
:1086C00083FF34004A003700119881001E0090009B
:1086D00080804000F00F2000808060000020230098
:1086E000E1407800F0C2B30080CF50004000340079
:1086F000119881001E00900080804000F00F200043
:108700008080600000202300E140780090C3B30027
:1087100080CF500036003C00119881001E00900070
:1087200080804000F00F2000808060000020230047
:10873000614078008000FB0000FD2F00008F4000AA
:10874000110037001E0078006A00B900000F7800A1
:10875000119881001E00900080804000F00F2000E2
:108760008080600000202300614078000000FB0052
:108770009E00400000FD2F00008F40001E00900072
:108780000000E80010079800119881001E0090007A
:1087900080804000F00F20008080600000202300D7
:1087A000E1407800F0C2B30080CF500010003400E8
:1087B000119881001E00900080804000F00F200082
:1087C0008080600000202300E140780090C3B30067
:1087D00080CF5000DBFF3400050037001000200080
:1087E000209889000000EB00200798000A0037005D
:1087F000119881001E0090000080400010988900B0
:1088000011988100F00F200000806000109889000E
:108810001E007800200798002E0090000080FA00CB
:10882000000006000400FA00109881008000E800B3
:10883000F00F20008080600000202300E1407800DD
:10884000A0C3B30080CF500013003A0010988100FD
:108850000080E8001098890011988100F00F200036
:10886000008060001098890069FE0700000F780002
:10887000109881000000E90010988900119881008B
:10888000F00F200000806000109889001E00780022
:108890001007980002003700100020001007980011
:1088A0001E0090000080FA00000006000400FA009C
:1088B000109881008000E800F00F200080806000A8
:1088C00000202300E1407800B0C3B30080CF500007
:1088D0000F003A00109881008080E800F00F20001F
:1088E000008060001098890049FE0700000F7800A2
:1088F000109881008000E900F00F200000806000E7
:10890000109889001E0078001007980002003700B8
:108910000000EB00100798001E0090000080FA0095
:10892000000006000200FA00109881008000E800B4
:10893000F00F20008080600000202300E1407800DC
:1089400080C7B30080CF500008003A001098810023
:108950008000E800F00F200000806000109889007F
:1089600010002000000F78003500370010988100BB
:108970008000E800F00F20008080600000202300CD
:10898000E140780040C6B30080CF500008003A00B4
:10899000109881008000E800F00F20000080600047
:1089A0001098890020002000000F78002400370074
:1089B000109881008000E800F00F200080806000A7
:1089C00000202300E140780020C6B30080CF500093
:1089D00008003A00109881008000E800F00F2000A5
:1089E000008060001098890030002000000F78009F
:1089F00013003700109881008000E800F00F20007D
:108A00008080600000202300E140780070C7B30040
:108A100080CF500008003A00109881008000E800E4
:108A2000F00F2000008060001098890040002000B6
:108A3000000F7800020037000000EB00000F780004
:108A40001E0078000080FA00000006000000FA0016
:108A500005003700109881008000E800F00F20002A
:108A60000080600010988900119881000020230088
:108A7000E140780000C2B30080CF5000F5FF320023
:108A80000080FA00000006000400FA000000EB007D
:108A9000000F7800109881008000E800F00F20009F
:108AA0000080600010988900E8FF0700D8FD0700EB
:108AB000000F78001E00E00053003A000000EB00B9
:108AC00010079800130037001E0090000040E800D7
:108AD00030DE02000000000050982A0098DB0200FF
:108AE000000000009E009000000320000088B900F4
:108AF0008102200080804000C0C62200008040002B
:108B0000C4DB0200000000001E0090000000E8002E
:108B1000100798001E009000EA0F5000EAFF340092
:108B200071012000C07B20007004020001000000E1
:108B30000000EB002098890013002000B200200004
:108B40001100200010002000FA000700000FE900CB
:108B5000E0FF2F009E0F1000030032000080EB00AA
:108B60009E0F100005003A00E1002000307D20003B
:108B7000700402000100000048003700B17F81004E
:108B8000000320000088B9002102200080804000FE
:108B9000C0C62200008040001000780000000100E4
:108BA000B0FF0200000000001E007800B07F8900C6
:108BB000B17F8100000320000088B900FE00400062
:108BC000C0C62200008040001000780000000100B4
:108BD000C0962A00C4DB0200000000001E00E00076
:108BE00004003200CB02A80080982A00C4DB0200F7
:108BF0000000000051002000B06520007004020059
:108C000001000000250037001E0FE900A000200031
:108C10009E0F10001D003C00B17F8100000320006A
:108C20000088B9002102200080804000C0C62200D8
:108C3000008040001000780000000100B0FF02003A
:108C4000000000001E007800B07F8900B17F810025
:108C5000000320000088B900FE004000C0C62200CA
:108C60000080400010007800000001001E00E000BD
:108C700001003200CB02A80051002000B0652000A6
:108C800070040200010000000400370051012000C0
:108C90002081200070040200010000000098810083
:108CA0008000E900F00F200000806000109889002B
:108CB0000080FA00000006002600FA0010002000E4
:108CC00020079800109881000000E90080007800DB
:108CD000F00F200000806000100798003D00370072
:108CE0001E0090000120230060C078000004E00016
:108CF00033003A001E0090008000E800F00F2000D2
:108D00008080600000202300614078000004E000C3
:108D10002B0032002E00900030DE02000000000028
:108D200050982A0098DB020000000000100020008C
:108D3000000F7800090037001E0090009E004000E0
:108D4000F00F200080806000002023006140780048
:108D50008EDF0200000000001E0FE8001E009000E1
:108D60009E004000F00F2000808060000020230063
:108D7000614078000004E000EFFF3A00AE0190008F
:108D80001E0090008000E800F00F200000816000CD
:108D9000E60047000380410002B078002E009000FA
:108DA0000000E800200798002E009000EF0F500010
:108DB0000C00320050902A00C4DB020000000000CA
:108DC0001E0090008000E900F00F2000008060008D
:108DD000100798009E00900010988100808F50002E
:108DE000BFFF3A00809C2A00C4DB020000000000A4
:108DF0007100200070822000700402000100000059
:108E0000130020002E019000110020000000EB0054
:108E100048000700100798001E009000E10F400076
:108E2000030032001E0090000000E00006003A003F
:108E300050902A00C4DB0200000000001000200057
:108E400020179800380037000000EB00200798003A
:108E500014003700019881002E00900080804000AF
:108E6000F00F2000008160001E009000E600470027
:108E700000004000E08078002E00900080804000DC
:108E8000F00F20008080600000202300E140780087
:108E900000202300017178002E0090000000E800FF
:108EA000200798001E009000E600470000004000E8
:108EB000E08078002E00900080804000F00F2000BD
:108EC0008080600000202300614078000004E00002
:108ED000E0FF3A00009881008000E900F00F2000D8
:108EE0000080600010988900119881002E00900089
:108EF000008040008080E800F00F200000806000CB
:108F000000988900009881008000E900F00F20009F
:108F100000816000012023000040EB0000F1780098
:108F20000000EB00201798002E1090000080FA003F
:108F3000000006001E00FA00100F9800210F980094
:108F4000320F9800430F98000000EB004007980094
:108F50000000EB00200798000000EB0010079800CD
:108F60000000EB00000F7800A09C2A0098DB0200B4
:108F7000000000001E0890000000E00004003D001A
:108F8000E09C2A0098DB020000000000030037008C
:108F90001E08900030DE020000000000009D2A0044
:108FA00098DB02000000000067003700ECDF0200E1
:108FB00000000000204F98002E4890000000FB00A9
:108FC000600F98006E089000ED0F500029003200ED
:108FD000EE089000ED8F500007003C006E099000F5
:108FE000E80F51000D0032006E089000EA0F5000AB
:108FF0002000320035003700D0022000EE0890003B
:10900000808F50001E003200800720006E09900003
:10901000800F5100270032002C0037004E009000D6
:109020000000E000070032004E0090000000E90060
:1090300040079800C08E2A0098DB02000000000064
:10904000410037001E00E000060032000000EB0087
:10905000000F7800C08E2A0098DB0200000000009C
:109060003900370070C0B3008EDF0200000000003E
:10907000350037001000200020079800320037002C
:109080004E0090000000E00006003A00D0C2B3009D
:109090008EDF02000000000010002000000F7800AA
:1090A0002900370070C0B3008EDF0200000000000E
:1090B000250037004E0890000000E0000300320059
:1090C0000080EB00500F98005D003700AE48900024
:1090D000F0C2B30080CF500018003400AE489000BA
:1090E00090C3B30080CF500014003C004E009000AD
:1090F000E30F50000600340070C0B3008EDF0200A2
:109100000000000040002000400798000E003700DB
:109110002E4890008EDF020000000000CE0090007C
:109120006B0047002E499000827078004E0090003E
:109130000000E800400798000300370070C0B3004B
:109140008EDF0200000000002E0090000000E00012
:1091500096FF320050902A00C4DB0200000000009D
:109160004E0090000000E00003003A001E0890004E
:10917000500F9800320037000000EB0010079800F5
:109180004E0090000000E90040079800CE009000DB
:1091900031079800110037001E0090006A00B900E6
:1091A00010079800BE0090004E0090008080500094
:1091B0006B004700614078008000FB001E009000BB
:1091C0008080400000FD2F000080400010079800C4
:1091D0004E0090000000E900400798004E0090000B
:1091E0000000E000ECFF3D009E0090002E08900083
:1091F000808F50000D0035009E0090003E089000CA
:10920000808F500009003C001E00E0000400320086
:109210001E0090000000EA00500F98000800370080
:109220001E019000520F980005003700B101200088
:1092300060FE2000700402000100000042FF3700C1
:109240005E0890000080FA00000006002C00FA0082
:10925000500F9800610F9800720F98000417980043
:1092600015179800231798000000EB00500798008E
:109270000000EB00300798006000B800008FBE00CF
:109280000000EB0020079800A09C2A0098DB020059
:10929000000000005E089000EE089000E00F500013
:1092A000E08F580004003D00E09C2A0098DB02009B
:1092B00000000000040037005E089000EE089000F7
:1092C00032DC020000000000009D2A0098DB020052
:1092D000000000006A003700ECDF02000000000020
:1092E000404F98004E4890000000FB005017980037
:1092F0005E109000ED0F50002A003200DE1090004A
:10930000ED8F500007003C005E119000E80F510007
:109310000D0032005E109000EA0F50002100320074
:1093200038003700D0022000DE109000808F5000FF
:109330001F003200800720005E119000800F510056
:10934000280032002F0037005E0090000000E0008F
:10935000070032005E0090000000E900500798000E
:10936000C08E2A0098DB0200000000004400370095
:109370002E0090000000E000060032000000EB002C
:1093800020079800C08E2A0098DB02000000000031
:109390003B00370070C0B3008EDF02000000000009
:1093A00037003700100020003007980034003700E5
:1093B0005E0090000000E00006003A00D0C2B3005A
:1093C0008EDF02000000000010002000200798003F
:1093D0002B00370070C0B3008EDF020000000000D9
:1093E000270037002E1090000000E000050032003A
:1093F0000080EB008080EB00301798004117980048
:109400006E003700CE489000F0C2B30080CF50000D
:1094100018003400CE48900090C3B30080CF5000B5
:1094200014003C005E009000E90F5000060034007C
:1094300070C0B3008EDF020000000000A00020001A
:10944000500798000E0037004E4890008EDF020053
:1094500000000000DE0090006D0047004E499000C3
:10946000827078005E0090000000E80050079800CD
:109470000300370070C0B3008EDF02000000000060
:109480003E0090000000E00093FF320050902A0060
:10949000C4DB0200000000005E0090000000E0005D
:1094A00005003A005E089000EE0890003017980022
:1094B00041179800410037006000B800008FBE00DF
:1094C0005E0090000000E90050079800DE00900068
:1094D000410798001A0037009E007800A000200085
:1094E000000AB8001E0078006000B900050178008D
:1094F000000141001E0090006A00B9000001410017
:1095000082027800048FBE00CE0090005E009000C2
:10951000808050006D004700614078008000FB00B3
:1095200000FD2F0000804000CF80DE001E0F4000B5
:109530005E9748005E0090000000E9005007980028
:109540005E0090000000E000E3FF3D007E08900018
:10955000CF80DE00BE0F5000AE8F580012003C00DE
:109560000E1090009E109000BE0F1000AE8F1800DD
:109570000D003C002E0090000000E00006003200CC
:109580001E00BE0060001000E08018003017980038
:1095900041179800090037001E00BE0030179800E0
:1095A0004117980005003700B101200060FE20003F
:1095B00070040200010000002BFF37003E109000F5
:1095C000CE1090000080FA00000006000400FA00AF
:1095D000309D2A00C4DB020000000000109E2A001B
:1095E00098DB02000000000050902A00C4DB02005B
:1095F000000000006100200090842000E6030200CB
:1096000001000000C07F8100E2DE020000000000D7
:1096100071002000F0FD2000E603020001000000C0
:10962000D07F8100E2DE020000000000C09F2A001F
:1096300098DB020000000000D07F81001007980036
:109640001E009000E10F5000040032001E00900048
:10965000E30F50000500320008003700C0A02A00C8
:1096600098DB02000000000007003700F0A02A008D
:1096700098DB0200000000000300370020A12A0050
:1096800098DB02000000000060A12A00C4DB020099
:1096900000000000E1012000F084200070040200BE
:1096A000010000000000EB00000F78000080FA00CD
:1096B000000006000200FA0080A12A0098DB0200E8
:1096C00000000000A17F25001000200068DF0200DC
:1096D00000000000E2DE02000000000000C2B30053
:1096E0008EDF02000000000051002000C0A3200017
:1096F000E603020001000000C17F250010002000E9
:1097000068DF020000000000E2DE0200000000004E
:109710006100200010A42000E60302000100000008
:10972000E17F25001000200068DF0200000000003B
:10973000E2DE02000000000050902A00C4DB0200BC
:1097400000000000C1002000D0862000700402004C
:109750000100000099000700CBC2BF00624060001A
:109760000004E0000500320011012000007120001B
:10977000E603020001000000040037002101200080
:1097800010722000E603020001000000C0C2B30016
:109790008EDF02000000000000C2B3008EDF020076
:1097A00000000000E2C2BF00704060000004E00062
:1097B0000500320041012000D06B2000E6030200CA
:1097C000010000000400370051012000806A2000E1
:1097D000E603020001000000C0C2B3008EDF0200F9
:1097E0000000000000C2B3008EDF02000000000095
:1097F000E8C2BF000042B2000004E00003003A00EB
:10980000F0A12A0098DB020000000000E8C2BF00BF
:10981000704060000004E00003003A0080A22A00CB
:1098200098DB020000000000E05D2300104078009B
:10983000704060000004E0000500320021022000BA
:10984000908720007004020001000000040037002F
:10985000E1012000B0892000700402000100000036
:10986000E05D230010407800684060000004E000E4
:1098700005003A00B1012000908B2000E6030200B1
:109880000100000004003700C1012000408D2000CD
:10989000E603020001000000C0C2B3008EDF020038
:1098A0000000000000C2B3008EDF020000000000D4
:1098B000B101200000352100E60302000100000094
:1098C000D05C23001040780030DE02000000000071
:1098D00050902A00C4DB020000000000E05D23007D
:1098E0009040780063C060000080FB00000F7800AB
:1098F0001E007800E10F5000130032009E00780037
:10990000E18F500004003C001E0078000000E000E1
:10991000080032001A0037009E007800E28F5000E5
:109920000E0032001E007800E30F500010003200DD
:10993000130037005101200060672000700402000E
:10994000010000000E0037006101200000662000C9
:1099500070040200010000000900370071012000BE
:10996000B04521007004020001000000040037002F
:109970007101200020472100700402000100000056
:10998000B17F8100000320000088B900610220003F
:1099900080804000C0C62200008040001000780097
:1099A00000000100C1002000D086200070040200E9
:1099B000010000000080FA00000006000000FA002C
:1099C000A100200020192100700402000100000005
:1099D00061052000703A21007004020001000000BF
:1099E00041022000D03F2100E603020001000000F8
:1099F000B17F8100000320000088B90041022000EF
:109A000080804000C0C62200008040001000780026
:109A100000000100A1002000601B2100E6030200FD
:109A20000100000010002000580007000010200076
:109A3000560007000002200054000700000120002B
:109A40005200070080002000500007004000200066
:109A50004E000700200020004C00070050902A0014
:109A6000C4DB0200000000004100200000232100B0
:109A7000E60302000100000021E3A80020C0B300BB
:109A80003E0002000100000024DF02000000000090
:109A900011002000B0372000E603020001000000A2
:109AA00090C0B3008EDF0200000000000040EB0019
:109AB0003E0002000100000024DF02000000000060
:109AC00011002000B0372000E60302000100000072
:109AD00090C0B3008EDF02000000000050C0B30051
:109AE0003E0002000100000024DF02000000000030
:109AF00011002000B0372000E60302000100000042
:109B000090C0B3008EDF02000000000010C0B30060
:109B10003E0002000100000024DF020000000000FF
:109B200011002000B0372000E60302000100000011
:109B300090C0B3008EDF02000000000021E3A90006
:109B40001000200020000700001020001E00070069
:109B5000000220001C000700000120001A0007007E
:109B600080002000180007004000200016000700B9
:109B7000200020001400070050902A00C4DB0200DF
:109B8000000000000080FA00000006000200FA0059
:109B9000000F7800C01680001E0060000000E0008A
:109BA0000400320020A32A0098DB0200000000001D
:109BB0000300370050A32A0098DB020000000000D9
:109BC0000080FA00000006000200FA00000F780092
:109BD000D01680001E0060000000E000040032008B
:109BE00080A32A0098DB0200000000000300370079
:109BF000B0A32A0098DB0200000000000080FA00F9
:109C0000000006000200FA00109881008000E800C1
:109C1000F00F200000806000109889008BFB070087
:109C20007BF90700000F78001E00E00006003400FA
:109C3000400020009E0F100003003C001E00E900C1
:109C4000A07F89000D0037000000EB0020988900FC
:109C500021022000D08F20007004020001000000CB
:109C60008001EB00420020001100200010002000C5
:109C7000B0FC07000000E900A07F8900210120005E
:109C8000F091200070040200010000000080FA0042
:109C9000000006000200FA000040EB00004F7800D0
:109CA000109881008000E800F00F20000080600024
:109CB0001098890065FB070055F9070010479800C8
:109CC0001E4090000004E000090032001E40900099
:109CD000EA4F500006003E001E4090000040E900A0
:109CE0008040780020FF2200014878000F003700F4
:109CF0000000EB0020988900E10B2000C0952000B7
:109D000070040200010000008001EB00A2002000AE
:109D1000110020009000200086FC07000040E900B0
:109D20008040780020FF22000148780020FF2200B8
:109D300010407800E94F500010003A0043FB070044
:109D400033F90700004F78001E04E0000B003A00D2
:109D50000000EB0020988900E0A32A00C4DB020089
:109D6000000000008001EB00F2FF27008000EB0004
:109D7000200220006FFC0700004F78004101200006
:109D8000A0A12000700402000100000011012000C9
:109D9000F03321007004020001000000BCDF02006B
:109DA000000000000004E000FCFF320020FF220061
:109DB00010407800E94F500003003A001E40780040
:109DC00022E00200000000001CE002000000000091
:109DD000ECDF0200000000008040780000C2B30009
:109DE00080CF500001003200F9FF37000080FA00F8
:109DF000000006000400FA00B07F81000000E000CF
:109E000007003A00D1012000B06820007004020071
:109E10000100000010002000209889007500370024
:109E2000E05D230010407800704060000004E00016
:109E300007003A0021022000D0FB2000700402003D
:109E40000100000010002000209889006900370000
:109E5000E8A2A800E882A800200020006E0102000D
:109E60000100000021E3A80050C0B3003E00020042
:109E7000010000008000780000102000808F50005A
:109E80000300360060A52A00C4DB020000000000C9
:109E900021E3A900109881008000E800F00F200065
:109EA0000080600010988900E8FA0700D8F80700E1
:109EB000000F7800209881000000E0000C003200C4
:109EC0000000EB002098890071052000504A210015
:109ED00070040200010000008001EB00320020004D
:109EE000110020001000200012FC0700000F780075
:109EF0001E007800100798001E009000E20F50002E
:109F0000120032001E009000E30F50001F003200CC
:109F10001E009000E10F5000010032002B003700BE
:109F2000E8A2A800E882A80091012000C04F21000B
:109F3000E60302000100000081002000C051210062
:109F400070040200010000002A003700E8A2A80007
:109F5000EA82A900E882A9004100200000C6200092
:109F6000E60302000100000091012000C04F210023
:109F7000E6030200010000007100200050512100A2
:109F800070040200010000001A003700E882A800F7
:109F9000EAA2A900E8A2A90021002000B0C5200083
:109FA000E60302000100000091012000C04F2100E3
:109FB000E603020001000000710020005051210062
:109FC00070040200010000000A003700E8A2A800A7
:109FD000E882A80091012000C04F2100E6030200A2
:109FE0000100000081002000C05121007004020027
:109FF000010000000080FA00000006000000FA00E6
:10A0000021438100C0862200E140780030C8B300BF
:10A0100080CF50000D003A00204381000000E8008E
:10A020002043890003003700204381000000E8003E
:10A030002043890021438100C0862200E14078004E
:10A0400000CEB30080CF5000F7FF36000080FA004A
:10A05000000006000A00FA00300798000000EB003C
:10A0600020079800AE009000C0862200E1407800F2
:10A0700000CEB30080CF500003003E000080EB0014
:10A080004007980020003700AE009000C0862200F4
:10A09000614078008080FB0000F22F0000804000CB
:10A0A000100798002E0090008000E800C086220073
:10A0B000614078000080FB004801DD002E00900028
:10A0C0008080E800C0862200614078000080FB00AC
:10A0D000000F41009E0078003E009000808F5000ED
:10A0E00003003A002E009000400798000600370059
:10A0F0009E0090002E009000008040006300400011
:10A1000020079800D7FF37004E0090000080FA002B
:10A11000000006000600FA00881F78000000EB002F
:10A12000000F780021438100C0862200E1407800C2
:10A1300080C2B30080CF50000F003A00204381005E
:10A140000000E8002043890013010700000F780099
:10A1500021438100C0862200E140780090C2B30014
:10A1600080CF5000B4003A00204381000000E80096
:10A1700020438900B000370021438100C0862200BF
:10A18000E140780000C4B30080CF500014003600D6
:10A1900021438100C0862200E1407800A0C5B300C1
:10A1A00080CF50000E003E0022438100C086220076
:10A1B000624078008080FB00F0FB2F0000804000B0
:10A1C00080004000408022000080400010007800A5
:10A1D000200798000200E80020438900980037001B
:10A1E00021438100C0862200E140780000C8B3000E
:10A1F00080CF50008400360021438100C0862200B9
:10A20000614078000080FB00100798000100E80022
:10A2100020438900700920009E009000808F50002C
:10A220004A003200700920009E009000808F50008C
:10A230000D003C00400920009E009000808F5000DF
:10A240001F003200600920009E009000808F5000A7
:10A2500034003200300920009E009000808F5000B2
:10A260002100320058003700A00920009E00900015
:10A27000808F50003F003200A00920009E00900017
:10A28000808F500005003C00800920009E00900057
:10A29000808F5000450032004B003700B00920008D
:10A2A0009E009000808F500039003200D0092000BD
:10A2B0009E009000808F5000160032004200370050
:10A2C000B17F8100000320000088B900EA0040004F
:10A2D000C0C622000080400010007800000001008D
:10A2E000000F780054003700B17F81000003200088
:10A2F0000088B900E8004000C0C62200008040008D
:10A3000010047800A400070008000100000F780086
:10A3100049003700B289020000000000000F7800F9
:10A3200045003700B17F8100000320000088B9009C
:10A33000F4004000C0C622000080400010007800F9
:10A3400000000100000F78003B003700B17F810062
:10A35000000320000088B900F8004000C0C62200B9
:10A36000008040001000780000000100000F78001D
:10A3700031003700CBC2BF000080FB000000D100DD
:10A38000614060000080FB00000F78002A00370069
:10A39000E2C2BF000080FB004400DE0061406000BC
:10A3A0000080FB00008FEA002300370021E3A800B3
:10A3B00010C0B3003E00020001000000000F780052
:10A3C00021E3A9001C0037000000EB00000F78001B
:10A3D000190037001E0078006A00B900000F7800ED
:10A3E00021438100C0862200614078000080FB008C
:10A3F0009E00400000FD2F00008F400020438100A0
:10A400000000E8002043890021438100C08622002B
:10A41000E1407800F0C2B30080CF50000600360063
:10A4200021438100C0862200E140780090C3B30040
:10A4300080CF5000E7FF36001E007800200798000C
:10A440002E0090004F0478000080FA000000060003
:10A450000600FA002FFF0700000F78000000370009
:10A4600021438100C0862200E1407800A0C2B300F1
:10A4700080CF50001500320021438100C0862200A9
:10A48000E1407800F0C2B30080CF50000F003200EE
:10A4900021438100C0862200E140780060C2B30001
:10A4A00080CF50000900320021438100C086220085
:10A4B000E1407800C0C7B30080CF500003003200F5
:10A4C0001E007800200798003000370021438100EB
:10A4D000C0862200614078000080FB0010079800D1
:10A4E0000100E80020438900A00220009E009000A7
:10A4F000808F500012003200A00220009E009000C9
:10A50000808F500005003C00600220009E009000FB
:10A51000808F500017003200D1FF3700F00220007A
:10A520009E009000808F50000B003200C00720007A
:10A530009E009000808F500011003200C8FF37004D
:10A54000F4FE0700800078001E0078000180B9004A
:10A55000000F7800C2FF3700EEFE07000001780010
:10A560001E007800110009000200D800000F7800DA
:10A57000BBFF3700E7FE07001E0F6000B8FF370083
:10A58000E4FE07001E0F7000B5FF37002E0090009C
:10A590000080FA00000006001200FA00ACFF07007D
:10A5A000000F78000000370021438100C0862200A0
:10A5B000E1407800D0C2B30080CF50001B003200D1
:10A5C00021438100C0862200E1407800B0C2B30080
:10A5D00080CF50001500320021438100C086220048
:10A5E000E1407800C0C3B30080CF50000F003200BC
:10A5F00021438100C0862200E1407800E0C3B3001F
:10A6000080CF50000900320021438100C086220023
:10A61000E1407800D0C3B30080CF50000300320087
:10A620001E00780020079800810037002143810038
:10A63000C0862200614078000080FB00100798006F
:10A640000100E80020438900C00320009E00900024
:10A65000808F50003A003200C00320009E0090001E
:10A66000808F500009003C00B00220009E00900046
:10A67000808F500011003200D00220009E00900018
:10A68000808F50000A003200C7FF3700D00320003F
:10A690009E009000808F50005B003200E00320009D
:10A6A0009E009000808F500007003200BEFF3700F0
:10A6B00067FF07001E0F1000BBFF370064FF070095
:10A6C0001E0F4000B8FF3700204381008000E800E3
:10A6D000C0862200E1407800D0C3B30080CF500094
:10A6E0000D003A005AFF07008000EB003107980088
:10A6F0009E0F500002003E0010002000300798001E
:10A70000BE009000010F7800204381000000E800A7
:10A7100020438900A4FF37004DFF07008000EB00B5
:10A72000410798009E0F50000200310010002000E9
:10A7300040079800CE009000010F78009AFF370084
:10A74000204381008000E800C0862200E1407800BC
:10A75000E0C3B30080CF50000D003A003CFF07007B
:10A760008000EB00510798009E0F5000020032005D
:10A770001000200050079800DE009000010F7800C4
:10A78000204381000000E8002043890086FF370055
:10A79000204381008000E800C0862200E14078006C
:10A7A000D0C3B30080CF50000D003A0028FF07004F
:10A7B0008000EB00610798009E0F500002003900F6
:10A7C0001000200060079800EE009000010F780054
:10A7D000204381000000E8002043890072FF370019
:10A7E0001BFF07008000EB00710798009E0F5000D0
:10A7F000020036001000200070079800FE00900054
:10A80000010F780068FF370011FF07008000EB00A0
:10A81000010F98009E0F500002003A001000200027
:10A82000000F98008E089000010F78005EFF37003F
:10A830002E0090000080FA00000006001C00FA00C4
:10A84000881F78000000EB00204389000000EB0027
:10A85000300798000000EB00200798000000EB0094
:10A86000100798000000EB00304389000000EB0067
:10A87000404389000000EB00504389000000EB00DA
:10A8800050079800E07F81000080A000E07F8900F1
:10A890000000EB0040079800090037004E009000D0
:10A8A0008000400040802200808040000000EB00DB
:10A8B000800878004E0090000000E80040079800F3
:10A8C0004E009000F90F5000F4FF34000B043700E5
:10A8D0001E0090000000E0001D003A0021438100AE
:10A8E000C0862200E1407800F0CDB30080CF500058
:10A8F00003003E00200020003007980002043700CB
:10A9000021438100C0862200614078008080FB00E6
:10A9100000F22F0000804000600798002043810073
:10A920008000E800C0862200614078000080FB00C3
:10A930004801DD00204381008080E800C0862200BD
:10A94000614078000080FB00000071005007980013
:10A950000000EB001007980020438100E300400056
:10A96000C0862200614078000080FB006101B900D0
:10A9700000F82F00F1FF2F00020140008381480002
:10A98000420F9800530F9800100220000100200091
:10A990004E099000DE099000800F5100818F590010
:10A9A000CA033E004E089000DE08900000600100DF
:10A9B0002100370034003700C4033700C3033700D9
:10A9C0006C0037007C0037009E003700B200370073
:10A9D000B90037002B01370073013700BB03370084
:10A9E000D50137001B023700770237008D02370090
:10A9F0007D023700A902370099023700B6023700FE
:10AA0000B20337005403370038033700AF03370071
:10AA1000AE033700DE023700CE0237007B0337007B
:10AA200089033700BC023700EE0237000E033700FF
:10AA300091033700A2033700100020002007980080
:10AA400020438100660040002043890020438100AC
:10AA50008080E900C0862200614078008080FB0091
:10AA6000F0FB2F0000844000CBFE070000017800BF
:10AA700088004400408022000080400002087800E6
:10AA80005EFD0700930337001000200020079800A8
:10AA9000204381006400400020438900BEFE07007F
:10AAA0000000E0001B00320021438100310F9800BC
:10AAB000C08622003E099000E24078008041EB0011
:10AAC0004357980020C8B30080CF500002003A00DE
:10AAD00010C0B30040579800BE0890000100E80085
:10AAE000204389004E5190000204E00079033200B7
:10AAF00010002000100798002043810063005000E0
:10AB00002043890073033700204381000000E800E0
:10AB10002043890021438100C0862200E140780063
:10AB200030C8B30080CF50000600320021438100BE
:10AB3000C0862200E140780000CEB30080CF5000F4
:10AB4000F1FF360021438100C0862200E1407800F9
:10AB500030C8B30080CF50005E033A0010002000E0
:10AB600010079800204381000080E90020438900FD
:10AB70005803370010002000200798002043810070
:10AB8000640040002043890083FE070031FD070078
:10AB9000000F78008081EB009E8F110003003200CF
:10ABA0001E007800204389004A033700600020001F
:10ABB0003007980047033700100020002007980056
:10ABC000204381006400400020438900404381000D
:10ABD000E90F500018003C004243810021438100EE
:10ABE0006E009000008040008001E900820041007A
:10ABF00080832200008040000308780040438100E9
:10AC00000000E8004043890063FE070011FD0700D3
:10AC1000000F78008080EB009E8F10000300320050
:10AC20001E017800224389002A03370060002000BB
:10AC30003007980027033700700020003007980085
:10AC400024033700C0A92A0098DB0200000000009E
:10AC50001000200020079800404381000000E00021
:10AC60000A003200404381000000E90040438900AF
:10AC7000404381008000400080832200008040002B
:10AC80001000780020438900120337008000200064
:10AC9000300798000F0337001000200020079800AD
:10ACA000214381006E00900000804000630040005E
:10ACB0002043890007033700100020002007980078
:10ACC0002043810064004000204389004F0037008A
:10ACD00021438100C0862200E140780020C2B300F9
:10ACE00080CF50001D003A00204381000000E800A2
:10ACF000204389000F003700E07F81000080A10021
:10AD0000E07F890021438100C086220061407800F5
:10AD1000004178000100E8002043890002407800EB
:10AD20008EDF020000000000E07F81000080A000B4
:10AD3000E07F890021438100C0862200E140780045
:10AD400020C2B30080CF5000EBFF3A0020438100C7
:10AD50000000E800204389002C00370021438100D7
:10AD6000C0862200E140780000C4B30080CF5000CC
:10AD70000600360021438100C0862200E1407800B1
:10AD8000A0C5B30080CF50000B00360021438100E6
:10AD9000C0862200614078000004E00012003D00FF
:10ADA00021438100C0862200E1407800F0CDB3004D
:10ADB00080CF50000C003E00F7FD0700000F780028
:10ADC000E07F81000080A100E07F89001E00780004
:10ADD000D2DD020000000000E07F81000080A000C2
:10ADE000E07F89000900370021438100C0862200EE
:10ADF000E1407800B0C3B30080CF500003003A00B8
:10AE0000204381000000E8002043890021438100A5
:10AE1000C0862200E1407800F0CDB30080CF500022
:10AE200006003E0021438100C0862200E1407800F8
:10AE300030C8B30080CF5000A5FF3A002043810006
:10AE40008000E900C0862200E1407800B0C3B30072
:10AE500080CF500009003200E07F81000080A10017
:10AE6000E07F890020B32A00C4DB0200000000005C
:10AE7000E07F81000080A000E07F89005FFC070088
:10AE8000940237001000200020079800E07F810026
:10AE90000080A100E07F8900204381006400400021
:10AEA0002043890021438100C0862200E1407800D0
:10AEB00020C2B30080CF500016003A00204381002A
:10AEC0000000E80020438900090037002143810089
:10AED000C086220061407800004178000100E8004F
:10AEE00020438900024078008EDF0200000000004D
:10AEF00021438100C0862200E140780020C2B300D7
:10AF000080CF5000F1FF3A00204381000000E800AC
:10AF10002043890021438100C0862200E14078005F
:10AF2000C0C2B30080CF500004003A00204381002B
:10AF30000000E800204389000200370030002000B4
:10AF40003007980021438100C086220061407800CC
:10AF50008080FB00F0FB2F00008440008001EB00AC
:10AF6000F2FF27008000EB000000EB009A47020090
:10AF700000000000000178008800440040802200AA
:10AF80000080400002087800204381000000E800B3
:10AF90002043890019FC0700E07F81000080A000A9
:10AFA000E07F89004B023700100020002007980046
:10AFB0002043810064004000204389003043810029
:10AFC000E30F500004003C00304381000000E80023
:10AFD000304389000200370040002000300798000D
:10AFE0003243810023438100C08622006340780001
:10AFF0008080FB0000FC2F00008240006610B9003A
:10B000008080E800C08422000080400004087800AE
:10B010000300E8002043890021438100C08622000C
:10B02000E1407800D0C3B30080CF500011003A0057
:10B03000204381000000E800204389003043810064
:10B040006600B9008080E800C084220000804000D3
:10B05000100078000004E9004FFD070000017800AF
:10B0600088004400408022000080400002087800F0
:10B070000200370030002000300798002343810091
:10B08000130F9800C08622001E099000E24078004D
:10B090008041EB0003579800B0C8B30080CF500048
:10B0A00002003A0010C0B300005798009E089000BC
:10B0B0000100E800204389000E5190000204E000E6
:10B0C000090032003843810033FD07000001780099
:10B0D0006640B900E4004000C084220000804000C7
:10B0E0000208780002003700300020003007980086
:10B0F00021438100C0862200E1407800F0CDB300FA
:10B1000080CF500008003600304381002243810088
:10B110006600B90080007800C084220000804000F2
:10B120000208780002003700300020003007980045
:10B13000B2FB0700E701370010002000200798004D
:10B1400020438100640040002043890022438100A5
:10B15000C0862200624078008080FB0000FC2F0047
:10B16000008F40000200E8002043890050002000CA
:10B17000300798000000EB00400798002F003700D0
:10B180004E0090006600B9008080E800C084220074
:10B1900000804000100078009E0F500024003A000C
:10B1A0001E00E90080004000408022000080400036
:10B1B000100178004E0090006600B900E4004000E5
:10B1C000C08422000080400010007800800F5100F1
:10B1D00012003D009E00E9000181400040802200F5
:10B1E00000004100100078000001E800818040006C
:10B1F0004080220000804000020878004E0090004D
:10B200006600B90080007800C08422000080400001
:10B21000100078002043890003003700304381008C
:10B220000000E900304389000000EB00300798007F
:10B230004E0090000000E800400798003143810074
:10B240004E009000810F5000CDFF34006BFB0700D3
:10B25000A001370010002000200798002043810043
:10B260006400400020438900504381000000E0005A
:10B2700023003A000000EB00400798000900370067
:10B28000CE009000C0862200614078008080FB00E4
:10B290004E0090008080400030F22F00008040007F
:10B2A000400798004E009000E3004000C086220056
:10B2B000E1407800E0C8B30080CF500005003200C4
:10B2C0004E009000C186220060C078000004E000BB
:10B2D000EBFF3A004E009000C186220060C078006B
:10B2E0000004E000040032004E00900064004000C2
:10B2F000504389000200370090002000300798007A
:10B3000023438100030F78005043810020438900CC
:10B310009E007800C0862200614078008080FB009B
:10B32000F0FB2F00008440007AFB0700000178004A
:10B33000880044004080220000804000020878001D
:10B3400020438100504389001E00E800204389000B
:10B3500051438100C0862200E1407800C0C2B300A2
:10B3600080CF500003003A00504381000000E80005
:10B370005043890051438100C0862200E14078009B
:10B3800000CEB30080CF50000D0036005043810046
:10B39000E3004000C0862200E1407800E0C8B3002E
:10B3A00080CF5000030032000000EB0050438900C2
:10B3B000030037005043810064004000504389007F
:10B3C0000EFB070043013700100020002007980003
:10B3D000214381006E009000008040006300400027
:10B3E000204389003B01370010002000200798000F
:10B3F000204381006400400020438900B17F810028
:10B40000000320000088B90080007800C0C6220038
:10B41000008040001000780000000100F7FA0700EB
:10B420002C013700100020002007980020438100E5
:10B430006400400020438900B17F810000032000A8
:10B440000088B9008080E800C0C62200008040006B
:10B450001000780000000100E8FA07001D01370025
:10B460001000200020079800204381006400400065
:10B4700020438900B17F8100000320000088B900CB
:10B48000E4004000C0C622000080400010007800A8
:10B4900000000100D9FA07000E013700100020005B
:10B4A0002007980020438100640040002043890069
:10B4B000B17F8100000320000088B900E600400051
:10B4C000C0C622000080400010007800000001008B
:10B4D000CAFA0700FF00370010002000200798007C
:10B4E000204381006400400020438900B17F810037
:10B4F000000320000088B900E8004000C0C6220018
:10B50000008040001004780023FC070008000100C0
:10B51000BAFA0700EF00370010002000200798005B
:10B520002043810064004000204389001AFC07008A
:10B530000000E00003003200128902000000000059
:10B54000020037006289020000000000ABFA070029
:10B55000E000370010002000200798002043810001
:10B5600064004000204389000BFC07000000E0005D
:10B5700003003200C922A900CB22A8000200370034
:10B58000C922A900CB22A9009CFA0700D1003700EC
:10B590001000200020079800204381006400400034
:10B5A00020438900FCFB07000000E0000600320099
:10B5B000E15D2300114078000000A0000010A10010
:10B5C0008048780005003700E15D230011407800D5
:10B5D0000000A0000010A1008048780087FA070052
:10B5E000BC00370010002000200798002043810095
:10B5F0006400400020438900E7FB070040AE89005B
:10B6000040AE81000000E00002003D000000EB00C1
:10B6100040AE890041AE810000FA2000808F5000CA
:10B620000200340000FA200040AE890050AE8100D4
:10B63000E10F500002003C002000200050AE8900C5
:10B6400051AE810030062000808F5000020034008F
:10B650003006200050AE8900D27E020000000000BB
:10B6600066FA07009B0037001000200020079800B2
:10B67000204381006400400020438900C6FB07008E
:10B6800050AE890040AE81000000E00002003D00A5
:10B690000000EB0040AE890041AE810000FA2000BE
:10B6A000808F50000200340000FA200040AE890074
:10B6B00050AE8100E10F500002003C00200020004D
:10B6C00050AE890051AE810030062000808F5000BE
:10B6D000020034003006200050AE8900D27E020005
:10B6E0000000000045FA07007A0037001000200033
:10B6F0002007980020438100640040002043890017
:10B70000A5FB07000000E00009003200B17F8100C6
:10B71000000320000088B900F0004000C0C62200ED
:10B720000080400010007800000001000800370091
:10B73000B17F8100000320000088B900F2004000C2
:10B74000C0C6220000804000100078000000010008
:10B750002AFA07005F003700100020002007980039
:10B760002043810064004000204389008AFB0700D9
:10B77000700798007E009000E10F5000100032002A
:10B78000FE009000E28F5000160032007E01900013
:10B790000200E000010032001A003700B17F810092
:10B7A000000320000088B900EE004000C0C622005F
:10B7B00000804000100078000000010011003700F8
:10B7C000B17F8100000320000088B900EC00400038
:10B7D000C0C6220000804000100078000000010078
:10B7E00008003700B17F8100000320000088B90005
:10B7F000F6004000C0C62200008040001000780023
:10B8000000000100FDF907003200370010002000A1
:10B8100020079800204381006400400020438900F5
:10B820005DFB07000000E00003003200E082A8009A
:10B83000E282A90002003700E282A900E082A900AA
:10B84000EEF90700230037001000200020079800C1
:10B850002043810064004000204389004EFB070024
:10B86000000F78001E0078006E0102000100000049
:10B87000E2F90700170037001000200020079800A9
:10B8800020438100640040002043890042FB070000
:10B89000000F7800B17F8100000320000088B9000C
:10B8A000FC004000C0C622000080400090007800EC
:10B8B0001E00780001000100D0F9070005003700E4
:10B8C00010002000300798000200370030002000F0
:10B8D000300798002E0090000000E00005003A00BC
:10B8E000214381006E009000008040006300400012
:10B8F000204389000000EB00200798003E009000E4
:10B900000000E000F2FB3200E07F81000080A10037
:10B91000E07F89003E009000E10F500018003200E7
:10B9200061002000C0372000E60302000100000093
:10B930003E009000D2DD02000000000081002000E7
:10B9400020382000E6030200010000005E009000A5
:10B95000D2DD020000000000B1002000A03820006D
:10B96000E60302000100000020438100D2DD020056
:10B970000000000020B32A00C4DB02000000000029
:10B980004F0478000080FA00000006000200FA0070
:10B99000000F780000C2B3008EDF0200000000003C
:10B9A0001E00780098DB02000000000000C2B30017
:10B9B0008EDF0200000000000080FA000000060098
:10B9C0000400FA000000EB00204389003C0037002F
:10B9D00020438100C186220060C178002247980080
:10B9E0002E4090000004E000040035002E4090003E
:10B9F0008EDF0200000000002E003700AE409000F5
:10BA000000CEB30080CF50001A00360020B32A00C9
:10BA1000C4DB020000000000204381008000E80039
:10BA2000C0862200614078000080FB004801DD00F4
:10BA3000204381008080E800C086220061407800B9
:10BA40000080FB0000004100000F780020438100CF
:10BA50000080E800204389001E007800D2DD02004B
:10BA60000000000000C2B3008EDF020000000000F2
:10BA70001000370000C2B3008EDF0200000000009B
:10BA80002E4090008080FB0000F82F0000804000D6
:10BA900080004000805023000080400010007800AB
:10BAA00098DB02000000000000C2B3008EDF02003D
:10BAB00000000000204381000000E80020438900CE
:10BAC00020438100C186220060C078000004E000AD
:10BAD000BFFF3A0020B32A00C4DB020000000000D0
:10BAE000204381000000E900D2DD020000000000D8
:10BAF0007100200050392000700402000100000095
:10BB00000080FA00000006000600FA001007980006
:10BB100010988100000F7800140037001E0090007C
:10BB200010417800119881000020230061407800C6
:10BB3000804F5100050032001E00780010988900E7
:10BB40000000EB00200798000E00370010988100DD
:10BB50008000E800F00F200000806000109889004D
:10BB60001E0090000000E800100798001E009000E2
:10BB7000104078000004E000E8FF3A0010002000C8
:10BB8000200798002E0090000080FA0000000600B8
:10BB90000400FA000000EB00000F780010003700EE
:10BBA0001E0078008000400080502300008040008C
:10BBB00010007800D4FF07000000E000070032000A
:10BBC0001E0078008040780000C8B30000C040002C
:10BBD0000080FB0010079800060037001E0FE800E9
:10BBE000100220009E0F1000EDFF34000000EB005B
:10BBF000100798001E0090000080FA000000060068
:10BC00003600FA0010988100000F98001B003700E2
:10BC10008E08900000202300E140780000C6B300A9
:10BC200080CF50000E0034008E08900000202300CA
:10BC3000E1407800A0C7B30080CF500008003C006E
:10BC40000E0990008E08900000202300E14078004B
:10BC5000F0CDB30080C060000020230001717800A7
:10BC60000E0890000000E800000F98008E08900079
:10BC7000F00F200000806000000F98008E089000F8
:10BC800000988100808F5000E1FF3A000000EB0037
:10BC9000000F98001198810000202300E1407800F7
:10BCA000F0C2B30080CF50001E0134001198810013
:10BCB00000202300E140780090C3B30080CF500003
:10BCC00018013C000000EB00000F9800080037004E
:10BCD0008E08900072004700808040000040EB001A
:10BCE000804878000E0890000000E800000F9800DF
:10BCF0008E08900020022000808F5000F4FF340056
:10BD00000841020000000000600798006E009000EB
:10BD10004880DE00804078007200470011409800A3
:10BD20006E0090008040780000C0EB0080C0600092
:10BD300072004700214098006E009000C5F807008F
:10BD4000500798005E009000E10F4000270032008D
:10BD5000DE009000C0862200614078008080FB00F9
:10BD600030F22F0000804000300798005E00900005
:10BD7000000F98000B0037000E0990008E0890000D
:10BD80003E00900080804000C0862200E1407800A4
:10BD9000C0862200017178000E0890000000E800C3
:10BDA000000F9800014020003E009000808050006D
:10BDB0000E089000808F5000EFFF3C000700370016
:10BDC0000E099000C18622000040EB0000F17800CF
:10BDD0000E0890000000E800000F98008E08900008
:10BDE000F03F2000808F5000F5FF3400300020002D
:10BDF000000F98000000EB00200798002645020085
:10BE000000000000400037002E0090000000E0001D
:10BE100002003A0026450200000000002E009000BB
:10BE20000000E00004003A0059FF07000080FB001A
:10BE300060079800020037000000EB0060079800E0
:10BE40006E0090000000E0000D0032000E0990002E
:10BE50006E009000804078007200470000004100B2
:10BE600001487800EE00900070082000808F50009C
:10BE700019003A0010002000200798001600370033
:10BE80001198810000202300E140780020C2B30017
:10BE900080CF500003003A002E0090000000A20066
:10BEA000200798000E0990001198810000202300BF
:10BEB0006140780080407800720047000000410037
:10BEC00001487800109881008000E800F00F200001
:10BED00000806000109889000E0890000000E800C3
:10BEE000000F98008E08900030022000808F5000D4
:10BEF0000500340091002000C039200070040200C9
:10BF000001000000CB0037001198810000988100EB
:10BF1000808F5000BCFF3A000E089000E30F5000E5
:10BF2000C40032000E089000E40F5000C10032003F
:10BF30000E08900080407800C0CDB30000C04000E3
:10BF40008040780072004700014878000000EB0054
:10BF5000000F98000000EB00400798000000EB0085
:10BF600050079800400037008E089000C0862200DD
:10BF7000E140780000CEB30080CF50002B003600A7
:10BF80008E089000C0862200614078008080FB000F
:10BF900000F22F0000804000300798000E0890004B
:10BFA0008000E800C0862200614078000080FB002D
:10BFB0004801DD000E0890008080E800C086220065
:10BFC000614078000080FB000000410010079800ED
:10BFD00072004700104090000080FB00C800DD00A8
:10BFE00072004700204090000080FB00008040006D
:10BFF000000F78001E0090009E0F500005003100D9
:10C000008E0890003E0090000080400063004000D9
:10C0100050079800BE0090000E089000008040007D
:10C0200063004000000F9800020037000E089000E7
:10C03000400798000E0890008000E800C0862200AB
:10C04000614078000080FB004801DD000E08900090
:10C050008080E800C0862200614078000080FB00FC
:10C0600000004100600798004E0090000000E000D2
:10C07000BDFF320072004700104078008080FB0056
:10C0800030F22F0000804000600798004E009000C2
:10C09000000F98000B0037008E0890006E00900093
:10C0A000008140008E089000C0862200E1407800A8
:10C0B000C0862200017178000E0890000000E9009F
:10C0C000000F98008E0890005E009000808F500056
:10C0D000F1FF3D000000EB00000F98000C0037005E
:10C0E000DE0090000E089000008140008E08900055
:10C0F000720047000080400090407800C086220017
:10C10000017178000E0890000000E800000F980010
:10C110008E0890006E009000808F5000F0FF350078
:10C120004400370030B32A0077FE07000000E0002B
:10C1300005003200C1F9070020B32A00C4DB020069
:10C14000000000003B00370070B32A006EFE0700BD
:10C150000000E0000200320019FE07003500370041
:10C16000C0B32A0068FE07000000E00004003200AF
:10C17000E07F81000090A100E07F89002D00370062
:10C1800010B42A0060FE07000000E0001F0032002B
:10C190000000EB00000F9800170037000000EB00D4
:10C1A000700798000E0037008E0890007E00900007
:10C1B00080804000C0862200614078000080FB0043
:10C1C00092DE02000000000000C2B3008EDF020019
:10C1D000000000007E0090000000E800700798005A
:10C1E0007E009000EF0F5000EFFF34000E0890002B
:10C1F00070004000000F98008E089000F03F200073
:10C20000808F5000E5FF34000A00370070B42A0028
:10C210003DFE07000000E0000200320007000700BA
:10C2200004003700C1002000503A200070040200D2
:10C23000010000000080FA00000006000200FA0081
:10C240000000EB00000F7800050037001E017800A9
:10C25000C18622000040EB0000F178001E0FE800CC
:10C26000F03F20009E0F1000F8FF3400C18622002E
:10C2700010CEB30080487800D186220000C0EB00C9
:10C2800080487800E186220000C0EB0080487800FA
:10C29000F186220010CAB300804878000080FA00BE
:10C2A00000000600575249005445200042495400FE
:10C2B0003A2020002A6E650078742000636C6F00BD
:10C2C000636B2000285E2900207769006C6C2000D9
:10C2D00075736500207468006973200076616C00D6
:10C2E00075654E006F2064006576690063652C00FB
:10C2F0002074720079202800414C4100524D2900E1
:10C30000205345004152430048206D006163720094
:10C310006F20660069727300744144004452450006
:10C32000535320004D414300524F200020302E0037
:10C330004D616300726F20006D656E00754D610088
:10C3400063726F00202020002020310057495200E6
:10C350004520610064647200657373000D0A20005B
:10C3600020202A003157490052452000524F4D00ED
:10C3700020434F004D4D41004E4420004D414300AD
:10C38000524F73003A0D0A00203531002E524500FD
:10C3900041442000524F4D002028300078333300B4
:10C3A00029202A00666F7200207369006E676C0096
:10C3B000652064006576690063652000627573001E
:10C3C0000D0A200038352E004D415400434820000E
:10C3D000524F4D00202830007835350029202A00A2
:10C3E000666F6C006C6F77006564200062792000D6
:10C3F0003634620069742000616464007265730001
:10C40000730D0A0020323000342E53004B49500087
:10C4100020524F004D20280030784300432920004F
:10C420002A666F006C6C6F0077656400206279008B
:10C4300020636F006D6D61006E640D000A20320094
:10C4400033362E00414C4100524D200053454100EF
:10C45000524348002028300078454300290D0A0047
:10C4600020323400302E5300454152004348200012
:10C47000524F4D00202830007846300029414C00B2
:10C4800041524D00205345004152430048202800AE
:10C49000307845004329530045415200434820006D
:10C4A00028307800463029004465760069636500CD
:10C4B00020494400732061007265200061766100AC
:10C4C000696C6100626C650020627900204D41005A
:10C4D00043524F002C20730065652000283029004E
:10C4E0002E52450041442000524F4D00202830007C
:10C4F00078333300293A20004D415400434820004E
:10C50000524F4D00202830007835350029534B001C
:10C5100049502000524F4D002028300078434300FE
:10C5200029556E006B6E6F00776E20006D616300A1
:10C53000726F2C002074720079203F00206F72000F
:10C5400020283000292066006F72200068656C008A
:10C550007042550053205200455345005420570067
:10C5600061726E00696E67003A202A0053686F009E
:10C57000727420006F7220006E6F200070756C0066
:10C580006C2D750070202A004E6F200064657600C7
:10C590006963650020646500746563007465640008
:10C5A000204453003138530032302000486967007E
:10C5B00068205000726573002044690067205400B1
:10C5C000686572006D4453003138420032302000FB
:10C5D00050726F0067205200657320004469670045
:10C5E0002054680065726D004453310038323200C7
:10C5F000204563006F6E2000446967002054680086
:10C6000065726D00445332003430340020456300BD
:10C610006F6E7200616D200074696D0065204300CB
:10C6200068697000445332003433310020314B00CC
:10C630002045450050524F004D556E006B6E6F0007
:10C64000776E2000646576006963650050574D0081
:10C6500020646900736162006C656400314B4800BE
:10C660007A2D34002C303000304B48007A205000B6
:10C67000574D46007265710075656E006379200044
:10C68000696E20004B487A00205072006573630089
:10C69000616C65003A505200323A4400757479007A
:10C6A00020637900636C650020696E0020252000FE
:10C6B00050574D0020616300746976006545520053
:10C6C000524F52003A205000574D200061637400D1
:10C6D000697665002C20670020746F002064690073
:10C6E000736162006C654100555820004672650018
:10C6F000717565006E6379003A204100555820003D
:10C70000494E500055542F0048492D005A415500BC
:10C71000582048004947480041555800204C4F00D8
:10C7200057564F004C544D004554450052204D0083
:10C730004F444500564F4C0054414700452050009F
:10C74000524F4200453A200056457200726F720007
:10C7500028292000406C69006E653A002040700076
:10C76000676D730070616300653A20006279740040
:10C7700065732E00546F6F00206C6F006E67210090
:10C7800053796E007461780020657200726F7200D8
:10C790004E6F200045455000524F4D0045726100DC
:10C7A00073696E0067646F006E655300617669009F
:10C7B0006E672000746F2000736C6F007420490056
:10C7C0006E7661006C69640020736C006F744C00BD
:10C7D0006F616400696E6700206672006F6D2000F3
:10C7E000736C6F007420450052524F00523A200083
:10C7F000636F6D006D616E006420680061732000DE
:10C800006E6F2000656666006563740020686500D1
:10C8100072654100434B4E0041434B004932430097
:10C8200020535400415254002042490054493200E0
:10C8300043205300544F50002042490054493200D5
:10C8400043206D006F6465003A0D0A0020312E0010
:10C8500020536F0066747700617265000D0A200036
:10C86000322E2000486172006477610072655300C7
:10C87000657420007370650065643A000D0A20003D
:10C88000312E20007E354B00487A0D000A20320000
:10C890002E207E0035304B00487A0D000A203300F0
:10C8A0002E207E00313030004B487A000D0A2000E7
:10C8B000342E20007E343000304B48007A5741003F
:10C8C000524E49004E473A0020484100524457001A
:10C8D0004152450020493200432069007320620024
:10C8E000726F6B00656E20006F6E200074686900C7
:10C8F0007320500049432100202852004556200053
:10C90000413329005365740020737000656564002D
:10C910003A0D0A0020312E0020313000304B480003
:10C920007A0D0A0020322E0020343000304B4800AF
:10C930007A0D0A0020332E0020314D00487A49003C
:10C9400032432000286D6F0064207300706429005A
:10C950003D28200020302E004D616300726F2000C2
:10C960006D656E00750D0A0020312E00376269007A
:10C970007420610064647200657373002073650045
:10C9800061726300680D0A0020322E0049324300B4
:10C9900020736E006966660065720D000A20330020
:10C9A0002E436F006E6E650063742000746F20006C
:10C9B0006F6E2D00626F610072642000454550006B
:10C9C000524F4D000D0A2000342E45006E6162006A
:10C9D0006C6520005772690074696E0067207400EE
:10C9E000686520006F6E2D00626F61007264200028
:10C9F00045455000524F4D00536561007263680019
:10CA0000696E67002049320043206100646472004F
:10CA10006573730020737000616365002E2046000B
:10CA20006F756E006420640065766900636573004D
:10CA3000206174003A536E006966660065724300B7
:10CA40006F6D6D00616E64006D6F6400653F0D0079
:10CA50000A312E00203662002F313400620D0A00A8
:10CA6000322E200034622F003136620044656C00A3
:10CA700061793F0050494300286D6F0064206400D5
:10CA80006C7929003D2843004D44440054416E0018
:10CA90006F20720065616400756E6B006E6F7700C9
:10CAA0006E206D006F6465002831290020676500E5
:10CAB000742064006576490044446500764944006A
:10CAC000203D20002052650076203D00204E6F0062
:10CAD000742069006D706C00656D65006E74650092
:10CAE000642028007965740029506C00656173002A
:10CAF000652065007869740020504900432070006B
:10CB0000726F670072616D006D696E0067206D0065
:10CB10006F64650028424100534943002952650073
:10CB200061647900612F41002F402000636F6E0027
:10CB300074726F006C7320004155580020706900BA
:10CB40006E612F00412F400020636F006E747200F1
:10CB50006F6C730020435300207069006E436F00B8
:10CB60006D6D61006E6420006E6F7400207573003F
:10CB700065642000696E20007468690073206D0090
:10CB80006F64650050756C006C2D7500702072002C
:10CB90006573690073746F00727320004F4646001E
:10CBA00050756C006C2D7500702072006573690003
:10CBB00073746F00727320004F4E5300656C6600F3
:10CBC0002D74650073742000696E200048695A0056
:10CBD000206D6F00646520006F6E6C007952450017
:10CBE00053455400424F4F00544C4F0041444500C0
:10CBF00052415500582049004E505500542F4800CE
:10CC0000492D5A002C205200454144003A20500042
:10CC10004F57450052205300555050004C49450095
:10CC200053204F004E504F0057455200205355009F
:10CC300050504C0049455300204F460046444100A7
:10CC4000544120005354410054453A0020444500CB
:10CC50004C415900207573005752490054453A0021
:10CC60002052450041443A0020434C004F434B00C2
:10CC70002C203100434C4F00434B2C00203044000B
:10CC800041544100204F550054505500542C200071
:10CC900031444100544120004F5554005055540038
:10CCA0002C203000202A7000696E2000697320005B
:10CCB0006E6F7700204869005A434C004F434B0089
:10CCC00020544900434B53003A2052004541440050
:10CCD00020424900543A200053796E007461780074
:10CCE00020657200726F720020617400206368001A
:10CCF00061722000782E2000657869007428770022
:10CD0000697468006F75740020636800616E670065
:10CD100065296E006F206D006F64650020636800F8
:10CD2000616E670065233A00204E6F0020736F002C
:10CD30006674770061726500207265007365740027
:10CD4000206F6E00207634002C2075007365200063
:10CD50007468650020726500736574002062750058
:10CD600074746F006E2E4E006F6E650078697300EC
:10CD700074656E0074207000726F74006F636F00D2
:10CD80006C2178002E206500786974000D0A490036
:10CD90006E7661006C696400206368006F696300EF
:10CDA000652C2000747279002061670061696E0053
:10CDB0004445560049443A0068747400703A2F00A4
:10CDC0002F6461006E676500726F7500737072008A
:10CDD0006F746F007479700065732E00636F6D005F
:10CDE0002A2D2D002D2D2D002D2D2D002D2D2A002D
:10CDF0004F7065006E206400726169006E206F00E4
:10CE00007574700075747300202848003D486900EF
:10CE10002D5A2C00204C3D00474E4400294E6F00F7
:10CE2000726D61006C206F00757470007574730012
:10CE3000202848003D332E0033762C00204C3D0046
:10CE4000474E4400294D53004220730065743A0058
:10CE5000204D4F0053542000736967002062690021
:10CE60007420660069727300744C53004220730092
:10CE700065743A00204C450041535400207369000A
:10CE80006720620069742000666972007374200074
:10CE9000426F6F00746C6F006164650072207600F1
:10CEA00020312E0020484500580D0A0020322E0067
:10CEB00020444500430D0A0020332E002042490043
:10CEC0004E0D0A0020342E002052410057446900C4
:10CED00073706C0061792000666F72006D61740080
:10CEE0002073650074566F006C74610067652000E4
:10CEF0006D6F6E0069746F0072733A0020355600D2
:10CF00003A2020007C2033002E3356003A202000A7
:10CF10007C20560050554C004C5550003A20530090
:10CF2000657420007365720069616C0020706F0089
:10CF3000727420007370650065643A0020286200F6
:10CF4000707329000D0A2000312E2000333030008C
:10CF50000D0A2000322E200031323000300D0A0040
:10CF600020332E002032340030300D000A203400EF
:10CF70002E203400383030000D0A2000352E2000DD
:10CF800039363000300D0A0020362E0020313900AD
:10CF9000323030000D0A2000372E200033383400A4
:10CFA00030300D000A2038002E2035003736300092
:10CFB000300D0A0020392E0020313100353230008A
:10CFC000300D0A0031302E0020496E00707574005B
:10CFD0002043750073746F006D204200415544007A
:10CFE0000D0A3100312E2000417574006F2D420072
:10CFF00061756400204465007465630074696F00A6
:10D000006E202800416374006976690074792000FD
:10D0100052657100756972006564290041646A0097
:10D020007573740020796F0075722000746572004A
:10D030006D696E00616C410072652000796F75004A
:10D040002073750072653F002043460047313A0067
:10D050002043460047323A00285C2D002F5F5C00D9
:10D060002D2928005C5F2F002D295300656C650079
:10D07000637420006F7574007075740020747900FB
:10D0800070653A000D0A2000312E20004F706500B7
:10D090006E206400726169006E202800483D4800DF
:10D0A000692D5A002C204C003D474E0044290D00AC
:10D0B0000A2032002E204E006F726D00616C20003D
:10D0C00028483D00332E3300562C20004C3D4700AD
:10D0D0004E4429005232570020287300706420000B
:10D0E00068697A00293D2800202030002E4D61001B
:10D0F00063726F00206D65006E750D000A203100AF
:10D100002E4953004F37380031362D00332041006F
:10D1100054520D000A2032002E4953004F37380078
:10D1200031362D00332070006172730065206F006E
:10D130006E6C790049534F002037380031362D008E
:10D1400033204100545220002852450053455400DA
:10D15000206F6E0020435300290D0A0052455300F2
:10D160004554200048494700482C2000434C4F00BC
:10D17000434B2000544943004B2C200052455300A0
:10D18000455420004C4F570049534F00203738007A
:10D1900031362D003320720065706C007920280034
:10D1A000757365007320630075727200656E74009C
:10D1B000204C53004220730065747400696E670050
:10D1C000293A200050726F00746F63006F6C3A0050
:10D1D00020736500726961006C332000776972000A
:10D1E00065322000776972006552460055756E0001
:10D1F0006B6E6F00776E5200656164002074790079
:10D2000070653A0020746F0020656E0064766100DE
:10D2100072696100626C6500206C65006E67740065
:10D220006844610074612000756E690074733A008F
:10D23000206E6F0020696E0064696300617469008C
:10D240006F6E44006174610020756E006974200087
:10D250006C656E0067746800202862006974730052
:10D26000293A200043532000454E4100424C4500DE
:10D270004443530020444900534142004C4544007C
:10D2800052335700202873007064200063736C00D1
:10D29000206869007A293D00282029000D0A4400F1
:10D2A000697363006F6E6E006563740020616E00C9
:10D2B0007920640065766900636573000D0A430098
:10D2C0006F6E6E00656374002028410044432000A7
:10D2D000746F20002B332E003356290043747200E4
:10D2E0006C415500584D4F00444520004C454400CA
:10D2F00050554C004C55500020485000554C4C00A7
:10D30000555020004C5652004547410044432000F0
:10D31000616E64002073750070706C007935560082
:10D3200056505500332E3300564144004342750099
:10D3300073206800696768004275730020486900BF
:10D340002D5A20003042750073204800692D5A0084
:10D3500020314D004F4445002C20560052454700D7
:10D360002C2061006E64200055534200204C450083
:10D370004473200073686F00756C64002062650060
:10D38000206F6E0021466F00756E640020206500DE
:10D3900072726F0072732E004D4F530049434C0060
:10D3A0004B4D4900534F430053204F004B20460044
:10D3B00041494C005365740020737000656564003A
:10D3C0003A0D0A0020312E00203330004B487A00FD
:10D3D0000D0A2000322E2000313235004B487A00F1
:10D3E0000D0A2000332E2000323530004B487A00E1
:10D3F0000D0A2000342E2000314D48007A436C0085
:10D400006F636B0020706F006C617200697479004B
:10D410003A0D0A0020312E00204964006C6520007E
:10D420006C6F7700202A640065666100756C74007B
:10D430000D0A2000322E200049646C00652068002F
:10D44000696768004F7574007075740020636C0024
:10D450006F636B002065640067653A000D0A200069
:10D46000312E200049646C00652074006F2061003B
:10D470006374690076650D000A2032002E20410099
:10D480006374690076652000746F200069646C0025
:10D4900065202A006465660061756C0074496E0041
:10D4A00070757400207361006D706C0065207000F1
:10D4B00068617300653A0D000A2031002E204D008E
:10D4C000696464006C6520002A646500666175000B
:10D4D0006C740D000A2032002E2045006E6453004B
:10D4E0005049200028737000642063006B70200096
:10D4F000736B650020736D0070206300736C2000F7
:10D5000068697A00293D2800202030002E4D6100F6
:10D5100063726F00206D65006E750D000A2031008A
:10D520002E536E006966660020435300206C6F0026
:10D53000770D0A0020322E00536E690066662000C7
:10D54000616C6C00207472006166660069632D0076
:10D5500070202D0066202A00427974006573200037
:10D5600064726F0070706500642A460041494C0087
:10D5700045442C00204E4F002044410054414400BB
:10D58000617461002062690074732000616E640040
:10D590002070610072697400793A0D000A20310030
:10D5A0002E2038002C204E004F4E4500202A6400CB
:10D5B00065666100756C7400200D0A0020322E0033
:10D5C00020382C0020455600454E20000D0A200032
:10D5D000332E2000382C20004F444400200D0A0038
:10D5E00020342E0020392C00204E4F004E45530091
:10D5F000746F70002062690074733A000D0A200095
:10D60000312E200031202A006465660061756C00AF
:10D61000740D0A0020322E0020325200656365002E
:10D620006976650020706F006C6172006974790022
:10D630003A0D0A0020312E00204964006C6520005C
:10D6400031202A006465660061756C00740D0A0063
:10D6500020322E00204964006C65200030554100C6
:10D66000525420002873700064206200726720000A
:10D67000646270002073620020727800702068007D
:10D68000697A29003D28200020302E004D6163007A
:10D69000726F20006D656E00750D0A0020312E003E
:10D6A000547261006E737000617265006E742000C8
:10D6B00062726900646765000D0A2000322E4C001A
:10D6C00069766500206D6F006E6974006F720D00E1
:10D6D0000A2033002E4272006964670065207700DB
:10D6E0006974680020666C006F772000636F6E00BD
:10D6F00074726F006C0A0D0020342E0041757400A6
:10D700006F20420061756400204465007465630009
:10D7100074696F006E2028004163740069766900A7
:10D72000747920004E6565006465640029554100E8
:10D73000525420006272690064676500526573008C
:10D7400065742000746F2000657869007452610070
:10D75000772055004152540020696E0070757400A6
:10D760005541520054204C00495645002044490080
:10D7700053504C0041592C00207D2000544F200074
:10D7800053544F00504C4900564520004449530023
:10D79000504C410059205300544F50005045440014
:10D7A000574152004E494E00473A200070696E00C2
:10D7B00073206E006F7420006F7065006E2064002F
:10D7C000726169006E20280048695A0029205200C1
:10D7D00045564900443A0D000A496E0076616C00D6
:10D7E0006964200063686F00696365002C20740021
:10D7F0007279200061676100696E6D007352530099
:10D80000204C4F00572C2000434F4D004D414E00FF
:10D8100044204D004F4445005253200048494700E2
:10D82000482C20004441540041204D004F44450005
:10D83000416464007265730073206F0066205000BD
:10D8400043463800353734003F5468006973200080
:10D850006D6F640065207200657175006972650006
:10D86000732061006E206100646170007465720055
:10D870004C4344002074790070653A000D0A200082
:10D88000312E20004844340034373800302028003E
:10D89000757369006E6720005043460038353700C5
:10D8A000342049004F206500787061006E64650087
:10D8B00072294C00434420002874790070206100D4
:10D8C0006464720029203D002028200020302E00B2
:10D8D0004D616300726F20006D656E00750D0A006A
:10D8E00020312E004C4344002052650073657400C3
:10D8F0000D0A2000322E49006E697400204C43004E
:10D90000440D0A0020332E00436C65006172200034
:10D910004C4344000D0A2000342E430075727300FE
:10D920006F722000706F7300697469006F6E200061
:10D9300065783A002834290020300D000A2036008E
:10D940002E5772006974650020746500737420009E
:10D950006E756D006265720073206500783A28006C
:10D960003629200038300D000A2037002E5772006B
:10D970006974650020746500737420006368610039
:10D98000726163007465720073206500783A280044
:10D990003729200038304400697370006C617900C9
:10D9A000206C69006E6573003A0D0A0020312E006C
:10D9B000203120000D0A2000322E20004D756C0011
:10D9C000746970006C6549004E495400434C450031
:10D9D00041524300555253004F52200053455400CA
:10D9E0004E6F200041434B002C20630068656300AC
:10D9F0006B2061006461700074657200434C4B00E1
:10DA0000094D4F0053490900435309004D49530044
:10DA10004F5069006E73740061746500733A47007B
:10DA20004E440900332E3300560935002E3056007F
:10DA3000094144004309560050550900415558001A
:10DA400009500900500950000949090049092D00F1
:10DA5000094F570044092D00092D2D000954780065
:10DA600044092D0009527800445343004C095300E7
:10DA7000444109002D092D0050474300095047003B
:10DA800044092D00092D31002E2842005229090099
:10DA9000322E28005244290009332E00284F52000C
:10DAA000290934002E28590057290900352E28004D
:10DAB000474E290009362E0028424C00290937001C
:10DAC0002E28500055290900382E280047522900D9
:10DAD00009392E0028575400290930002E28420009
:10DAE0006C6B2900474E440009474E004409410031
:10DAF00044430900352E3000560933002E335600BA
:10DB000009565000550941005558090065786500CF
:10DB10006375740065203A0020205400494D45008B
:10DB20004F55540020302E00204D610063726F006D
:10DB3000206D65006E750D000A2031002E204C000E
:10DB40006976650020696E0070757400206D6F0045
:10DB50006E6974006F7249006E70750074206D00FC
:10DB60006F6E6900746F72002C2061006E79200066
:10DB70006B6579002065780069747300202A730052
:10DB800074617200746269007420650072726F00C3
:10DB900072202A0070617200697479002065720039
:10DBA000726F7200202A7300746F700062697400D3
:10DBB00020657200726F7200204E4F004E452000AB
:10DBC000554E4B004E4F57004E20450052524F00CD
:10DBD0005220610075746F0072616E0067652000ED
:10DBE0002B4D48007A292B006B487A0029496E009A
:10DBF000707574002061200063757300746F6D0090
:10DC0000204241005544200072617400653A57007B
:10DC100041524E00494E47003A2050006F73730046
:10DC200069626C00652062007566660065726F004F
:10DC300076657200666C6F0077416E0079206B002C
:10DC400065792000746F2000657869007453700056
:10DC50006163650020746F0020636F006E7469005B
:10DC60006E7565004E756D0062657200206F66000E
:10DC7000206269007473200072656100642F770070
:10DC800072697400653A200043533A000D0A20007F
:10DC9000312E200043530D000A2032002E202F0089
:10DCA000435320002A646500666175006C7450005F
:10DCB0006F73690074696F006E2069006E206400E4
:10DCC000656772006565730053657200766F2000AA
:10DCD00061637400697665002331320020202000E2
:10DCE00020092300313120002020200009233100A9
:10DCF000302020002020090023303900202020007F
:10DD0000092330003820200020092300303720006C
:10DD10002020090023303600202020000923300075
:10DD20003520200020092300303420002020090065
:10DD3000233033002020200009233000322020002F
:10DD40002009230030312000202047004E440900E4
:10DD5000352E3000560933002E3356000956500038
:10DD6000550941004443090041555800320941001A
:10DD700055583100094155005809430053094D00D9
:10DD800049534F0009434C004B094D004F53490084
:10DD90002D092D00092D09004F5744002D0952006F
:10DDA000784409002D09540078442D00092D0900FC
:10DDB00053434C0009534400412D09002D095000E4
:10DDC0004743090050474400612F41002F40200085
:10DDD000636F6E0074726F006C73200041555800C1
:10DDE00031207000696E61002F412F0040206300D8
:10DDF0006F6E7400726F6C007320410055583200D2
:10DE0000207069006E45450050524F004D5343004D
:10DE10004C5344004157500052454100442657009E
:10DE2000524954004556750073625300656C650095
:10DE3000637420005670750020285000756C6C00CB
:10DE40007570290020536F0075726300653A0D00EC
:10DE50000A2031002920450078746500726E610047
:10DE60006C2028006F7220004E6F6E0065290D0037
:10DE70000A20320029204F006E626F006172640038
:10DE800020332E0033760D000A20330029204F0066
:10DE90006E626F006172640020352E0030762000C3
:10DEA0006F6E2D00626F61007264200070756C00EF
:10DEB0006C75700020766F006C74610067652000DF
:10DEC000656E6100626C6500646469007361620084
:10DED0006C6564004E6F72006D616C0020746F00A1
:10DEE000206578006974570061697400696E670085
:10DEF0002061630074697600697479002E2E2E000B
:10DF00002A2A2000456172006C792000457869005A
:10DF100074212A002A204200617564003E313600D7
:10DF20006D3A200054686500204250002063610073
:10DF30006E6E6F0074206D00656173007572650010
:10DF4000206162006F76650020313600303030008D
:10DF5000303030002C2044006F6E65002E0A0D001A
:10DF600043616C0063756C0061746500643A200065
:10DF7000090A0D0045737400696D610074656400E1
:10DF80003A2020000920620070734700656E65002A
:10DF900072616C000909090009095000726F740070
:10DFA0006F636F006C2069006E74650072616300BE
:10DFB00074696F006E2D2D002D2D2D002D2D2D003F
:10DFC0002D2D2D002D2D2D002D2D2D002D2D2D0035
:10DFD0002D2D2D002D2D2D002D2D2D002D2D2D0025
:10DFE0002D2D2D002D2D2D002D2D2D002D2D2D0015
:10DFF0002D2D2D002D2D2D002D2D2D002D2D2D0005
:10E000002D2D2D002D2D2D002D2D2D002D2D2D00F4
:10E010002D2D2D002D2D2D002D3F09005468690058
:10E0200073206800656C7000090909002830290018
:10E03000094C6900737420006375720072656E008C
:10E0400074206D00616372006F733D00582F7C0077
:10E05000580943006F6E7600657274007320580093
:10E060002F726500766572007365200058090900FB
:10E0700028782900094D610063726F0020787E00C6
:10E08000095365006C667400657374000909090022
:10E090005B09530074617200746F0900536574006A
:10E0A000206F7500747075007420740079706500BD
:10E0B000090909005D095300746F700024094A00C2
:10E0C000756D700020746F0020626F006F746C00BB
:10E0D0006F61640065720900097B09005374610077
:10E0E00072742000776974006820720065616400B2
:10E0F000262F2500094465006C617900203120003D
:10E1000075732F006D73090009097D0009537400B0
:10E110006F7061002F412F00400941005558500099
:10E12000494E2000286C6F00772F4800492F52007D
:10E130004541440029090900226162006322090067
:10E1400053656E0064207300747269006E6762002C
:10E150000953650074206200617564007261740087
:10E16000650909000931320033095300656E640006
:10E1700020696E00746567006572200076616C002E
:10E18000756563002F432F006B2F4B00094155002D
:10E190005820610073736900676E6D00656E7400CE
:10E1A00020284100302F4300532F4100312F4100E0
:10E1B00032290900307831003233090053656E008E
:10E1C000642068006578200076616C0075656400E5
:10E1D0002F4409004D656100737572006520410090
:10E1E00044432000286F6E0063652F00434F4E00AC
:10E1F000542E290009306200313130000953650086
:10E200006E64200062696E006172790020766100A0
:10E210006C75650066094D00656173007572650077
:10E220002066720065717500656E630079090900EA
:10E230007209520065616400672F53000947650049
:10E240006E65720061746500205057004D2F5300B9
:10E25000657276006F0909002F0943004C4B2000BE
:10E260006869680009436F006D6D61006E64680045
:10E27000697374006F727900090909005C09430031
:10E280004C4B20006C6F6900095665007273690081
:10E290006F6E69006E666F002F7374006174750095
:10E2A00073696E00666F0900095E0900434C4B00FC
:10E2B00020746900636B6C002F4C09004269740084
:10E2C0006F72640065722000286D7300622F4C002D
:10E2D0005342290009092D000944410054206800D7
:10E2E000696D0900436861006E676500206D6F000D
:10E2F0006465090009095F000944410054206C006D
:10E300006F65090053657400205075006C6C7500D2
:10E3100070204D00657468006F640900092E0900C3
:10E320004441540020726500616470002F50090060
:10E3300050756C006C757000207265007369730015
:10E34000746F7200732028006F6666002F4F4E00B6
:10E350002909210009426900742072006561640086
:10E36000730953006372690070742000656E670062
:10E37000696E6500090909003A0952006570650077
:10E3800061742000652E67002E2072003A31300043
:10E3900076095300686F770020766F006C74730005
:10E3A0002F73740061746500730909003B09420012
:10E3B0006974730020746F002072650061642F001F
:10E3C0007772690074652000652E67002E2030008A
:10E3D000783535003B3277002F57090050535500F0
:10E3E00020286F0066662F004F4E290009093C0067
:10E3F000783E2F003C783D00203E2F003C303E0010
:10E400000955730065726D00616372006F207800BA
:10E410002F617300736967006E2078002F6C6900AC
:10E4200073742000616C6C000200FA00000F780029
:10E430009E0078000040EB00804878009E00780045
:10E440000040EB00904098001E0178006000B8008A
:10E4500010019800210198009E0078000000EB0058
:10E46000B00098009E0078000040EB00B048980093
:10E470009E0078000040EB00804898009E007800E5
:10E4800010C0B300904898009E00780010C0B30000
:10E49000A04898001E0178006000B80000099800AC
:10E4A000110998009E0078000000EB00A008980079
:10E4B0001E0178006000B8006001980071019800AA
:10E4C0000000EB000080FA00000006000200FA00E5
:10E4D000000F78000080FA00000006000800FA0033
:10E4E000008FBE0072002000030020003E004100AB
:10E4F000AE80490020079800310798002E00900058
:10E50000BE009000E00F5000E08F580006003D0074
:10E510002E019000BE01900067014100E08149009A
:10E5200022079800330798002E019000BE0190004A
:10E530004D1ADD004310DE0000007200C398DE00BB
:10E540000080FA00000006000200FA00000F7800C8
:10E550009E00780010002000B806020001000000B4
:10E560008000EB000000EB00B80602000100000094
:10E57000110020000000EB00B806020001000000BE
:10E580000080FA00000006000C00FA002007980046
:10E59000614798000000EB00000F78006E4090008B
:10E5A0000004E00017003A0010002000E6FF07001A
:10E5B0000000EB00100798000B0037008000EB0014
:10E5C0000000EB00B806020001000000110020006E
:10E5D0000000EB00B8060200010000001E009000E1
:10E5E0000000E800100798001E009000E40F5000A3
:10E5F000F2FF3400AE0090000040EB00804878004D
:10E60000080137002E009000904078006E40900086
:10E6100080CF5000110032006E409000E74F500054
:10E6200004003A002E00900010407800E64F5000A1
:10E6300007003A006E409000EE4F500007003A008D
:10E640002E00900010407800ED4F50000300320083
:10E6500050002000000F7800F20037002E009000DC
:10E66000904078006E40900080CF5000E8003A0063
:10E670006E409000E64F500006003A001000200067
:10E68000B1FF0700AE00900070C0B3008048780072
:10E69000DF0037006E409000ED4F5000DC003A0084
:10E6A00010002000A8FF0700AE009000E0C0B300FB
:10E6B00080487800D60037002E0090001040780087
:10E6C0000080FB006101B9004207980053079800E1
:10E6D000F0002000010020004E019000DE019000BB
:10E6E000800F5100818F5900C4003E004E00900001
:10E6F000DE009000006001000F00370014003700BA
:10E700001900370027003700350037003A0037007E
:10E71000480037004D0037005B00370069003700C4
:10E720006E0037007C003700810037008F00370013
:10E7300094003700A20037000000EB0082FF0700C2
:10E74000AE00900010C0B30080487800B0003700E1
:10E75000100020007CFF0700AE00900020C0B30036
:10E7600080487800AA0037006E409000E84F5000C3
:10E77000060036001000200073FF0700AE00900076
:10E7800090C0B30080487800A10037000000EB0083
:10E790006DFF0700AE00900030C0B30080487800E5
:10E7A0009B0037006E409000E44F500006003A0096
:10E7B0000000EB0064FF0700AE00900040C0B30013
:10E7C0008048780092003700100020005EFF0700AC
:10E7D000AE00900050C0B300804878008C00370035
:10E7E0001000200058FF0700AE00900050C0B3009A
:10E7F00080487800860037006E409000E64F500059
:10E8000006003A000000EB004FFF0700AE0090004A
:10E8100060C0B300804878007D0037001000200001
:10E8200049FF0700AE00900080C0B3008048780028
:10E83000770037001000200043FF0700AE00900073
:10E8400070C0B30080487800710037006E409000BF
:10E85000E44F500006003A000000EB003AFF0700CA
:10E86000AE00900040C0B3008048780068003700D8
:10E870001000200034FF0700AE00900080C0B300FD
:10E8800080487800620037006E409000E14F5000F1
:10E8900006003A000000EB002BFF0700AE009000DE
:10E8A00010C0B300804878005900370010002000E5
:10E8B00025FF0700AE00900020C0B300804878001C
:10E8C000530037000000EB001FFF0700AE00900070
:10E8D000A0C0B300804878004D0037006E40900023
:10E8E000EB4F500006003A000000EB0016FF070057
:10E8F000AE009000B0C0B3008048780044003700FC
:10E900001000200010FF0700AE009000C0C0B30050
:10E91000804878003E003700100020000AFF070002
:10E92000AE009000C0C0B3008048780038003700C7
:10E930006E409000ED4F500006003A000000EB00E2
:10E9400001FF0700AE009000D0C0B30080487800FF
:10E950002F00370010002000FBFE0700AE009000E3
:10E96000F0C0B30080487800290037001000200074
:10E97000F5FE0700AE009000E0C0B30080487800CC
:10E98000230037006E409000EB4F500006003A0025
:10E990000000EB00ECFE0700AE009000B0C0B3003A
:10E9A000804878001A00370010002000E6FE0700BB
:10E9B000AE009000F0C0B30080487800140037002B
:10E9C0006E409000E14F500006003A000000EB005E
:10E9D000DDFE0700AE00900010C0B3008048780054
:10E9E0000B00370010002000D7FE0700AE0090009B
:10E9F00020C0B30080487800050037005000200098
:10EA0000000F78002E009000EE4090000148780042
:10EA10002E009000904078006E40900080CF500013
:10EA200025FF3A001E0078000080FA000000060072
:10EA30001400FA00500798006107980072079800C8
:10EA4000030F9800140F98000000EB0030079800A7
:10EA50000E0890000000E0000A0032007E009000E6
:10EA6000900078000E089000010878000E089000D1
:10EA70008080E8007E009000100078000080400058
:10EA8000300798007E0090008080E8007E009000B3
:10EA90001000780000804000400798004F003700C9
:10EAA0004E0090000000E900400798004E009000E2
:10EAB00090407800414798000040EB0030479800B4
:10EAC0000000EB00000F7800330037005E0090007C
:10EAD000EE00900061005000E08058005007980060
:10EAE000610798001E0890000000E0000900320055
:10EAF0005E009000EE009000E00F5000E08F5800A4
:10EB000004003A001100200010002000B8060200A6
:10EB1000010000004E4090000080FB00E10060001A
:10EB200020002000B8060200010000004E409000C6
:10EB30000080FB000000D100404798008000EB00FF
:10EB40000000EB00B8060200010000003E0090004B
:10EB50000000E0000B003200780702000100000016
:10EB6000204798002E4090008080FB001E00780017
:10EB70000008DD00804078003E40900000C070003A
:10EB800030479800110020000000EB00B80602009A
:10EB9000010000001E0FE8005E009000EE009000F3
:10EBA000E00F5000E08F580003003200700020009A
:10EBB0009E0F1000C5FF34003E0090000000E000F2
:10EBC000060032003E0090000000E9003007980087
:10EBD0003E009000BE409000014878005E0090002A
:10EBE000EE009000E00F5000E08F5800ACFF3A00BC
:10EBF0000080FA00000006001C00FA0040079800A0
:10EC0000214F98006207980073079800040F98003E
:10EC1000150F9800260F9800370F98000000EB00A2
:10EC2000300798000000EB00200798000040EB0040
:10EC3000204798000000EB00500F9800AE4890006D
:10EC40000EF8970080CF5000020032001400200020
:10EC5000540F98005E089000000F78006E0090003E
:10EC6000FE009000E00F5000E08F58000D003A00C9
:10EC70002EB89700BEB89700E00F5000E08F580004
:10EC80006600320011C0B3004E0090003EFE070047
:10EC90002EB89700BEB89700880702000100000058
:10ECA0005E003700AE4890004E00900036FE070030
:10ECB0001E0278009E0990000E0990006E009000E0
:10ECC000FE0090005AFF07002E0890000000E000B0
:10ECD0000C0032003E0990009E0890002E08900023
:10ECE0007E02020001000000800078000000EB00BE
:10ECF000200798000100E00002003A001000200008
:10ED0000200798001E00E000330032004E00900003
:10ED1000104078008040E8004E00900001487800E4
:10ED20002E0090000000E0001C0032002EB897007A
:10ED3000BEB89700E00F5000E08F58001700320077
:10ED4000AE4090002EF0970080CF500013003100AD
:10ED500061C0B3004E0090000BFE070041C0B3003D
:10ED60004E00900008FE07002EB89700BEB897002E
:10ED7000C289DE004E0ADD004201DE00020172009F
:10ED80002EB89700BEB8970000004100818049006E
:10ED900020BF9F0031BF9F00030037008EF897000F
:10EDA0004E009000F8FD07002EB89700BEB89700FF
:10EDB000E00F5000E08F58000700320011C0B30090
:10EDC0004E009000F0FD07002EB89700BEB89700E7
:10EDD00088070200010000002E0090000000E00003
:10EDE0000E0032000040EB00005F9800AE40900043
:10EDF0002EF0970080CF50000200310014C0B30005
:10EE0000045F98002E4090000040E80020479800E2
:10EE10000E5890000004E000A2FF3A002E0090007F
:10EE20000000E0000C0032002EF097000004E0002B
:10EE300007003200AE4090002EF0970080CF5000C7
:10EE40000300360030002000300798000200370031
:10EE500020002000300798003E0090000080FA005B
:10EE6000000006001000FA00000F7800120798005A
:10EE70002307980031079800440798005507980029
:10EE80006607980077079800BE0090004E0090003B
:10EE9000BC030200010000006E0090000000E000D2
:10EEA00004003200BE0090006E009000BC0302001F
:10EEB000010000008F87E8002EF09700E0FF9F0020
:10EEC0002EB89700BEB89700809FBE008F87E800DD
:10EED0008EF89700E1FF9F00FE0390006E03900004
:10EEE000DE0290004E0290001E019000AE019000E4
:10EEF00041C0B3001E0078003FFF0700E8875700BD
:10EF00000080FA00000006001200FA005007980086
:10EF10006107980072079800030F98007E01900027
:10EF2000DE0090005E0090004E0302000100000031
:10EF30000040EB00304798000040EB00204798006D
:10EF40006E009000100F78000E08900010007800FE
:10EF50000000E90040079800480037004E0090008C
:10EF60008E0890000080E80001004000904078008A
:10EF7000414798004E4090000004E0003C00320001
:10EF80004E009000DE0090000080E800010040008C
:10EF9000904078006147980010C0B3005047980037
:10EFA0002A0037004E4090000080FB0061006000A6
:10EFB0000004E0001E0032002E4090000004E0003B
:10EFC00009003A001E0FE9001E007800EE009000D4
:10EFD0000080E80001004000904078003147980030
:10EFE00010C0B300204798003E409000AE40900013
:10EFF000014060000004E000050032006E40900017
:10F00000DE40900001407000604798000500370026
:10F010005E40900080C0EA006E40900000C060003A
:10F02000604798002E409000004040002047980024
:10F030005E40900000404000504798004E409000D5
:10F040000080FB000000D100404798004E40900037
:10F050000004E000D3FF3A004E009000DE00900074
:10F060000080E80001004000EE4090000148780078
:10F070004E0090000000E900400798004E0090000C
:10F080000000E000B5FF3D000080FA00000006002F
:10F090000200FA00000F78009E0078004000200077
:10F0A000B00098001E007800300090000080FA0048
:10F0B000000006000200FA00000F78009E007800B1
:10F0C00010C0B300804878000000EB000080FA0018
:10F0D000000006000200FA00000F78001E00780011
:10F0E000A0089000820B20001E004100BC0302001B
:10F0F000010000000000EB000080FA0000000600A4
:10F100000800FA00889FBE008A1F78003007980028
:10F11000640047000E070200010000004E4090000E
:10F120000080FB0001002000ECFC070010079800A5
:10F130009E00900020032000808F500003003400C8
:10F1400060002000000F7800240037004E4090003F
:10F150000080FB0001002000E0FC07008000780038
:10F160003E00900076004000BC0302000100000059
:10F170003E00900060019000F00190003E00900081
:10F18000904890003E009000760240004E40900073
:10F190000084FB00090020003E009000680540004C
:10F1A0008F87E8000040EB00E0FF9F00829FBE00D9
:10F1B0008F87E800E1FF9F008003EB000003EB0076
:10F1C0008002EB000801BE00B1C0B3000A00780065
:10F1D00089FE0700E8875700000F78001E00E00056
:10F1E000030032003E0090009E007800310098003D
:10F1F0001E0078004F0578004F04BE000080FA0022
:10F20000000006000A00FA00881F780040079800F6
:10F210004E0090007600400021002000BC03020058
:10F22000010000004E00900076004000180202002D
:10F230000100000020079800310798002E00900080
:10F24000BE009000A5FC0700100798009E009000EB
:10F2500020032000808F5000030034006000200055
:10F26000000F7800210037002E009000BE009000B3
:10F270009AFC0700800078004E0090007600400065
:10F28000BC030200010000004E00900060019000ED
:10F29000F00190004E009000904890004E009000C9
:10F2A000760240004E009000680440008F87E8001E
:10F2B0000040EB00E0FF9F00829FBE008F87E800C8
:10F2C000E1FF9F008003EB000003EB008002EB00F6
:10F2D0002E019000BE019000B1C0B300080078007C
:10F2E00045FE0700E8875700000F78001E00E00089
:10F2F000030032004E0090009E007800310098001C
:10F300001E0078004F0478000080FA00000006001C
:10F310000400FA00889FBE008A9FBE001007980074
:10F320001E009000A00890001E0090007600400093
:10F33000BC030200010000001E009000B0489000D5
:10F340001E00900060019000F00190001E009000EF
:10F35000204A90001E009000870B2000808343000D
:10F360001E009000C5042000808242001E00900014
:10F370002A082000000545001E009000F605400008
:10F380001E009000000C9000900C90001E00900059
:10F39000680040008F87E800E1FF9F00829FBE0069
:10F3A0008F87E800E4FF9F00050378008A02780059
:10F3B0000B0278000801BE0041C0B3000EFE07003A
:10F3C000E8875700000F78001E00E00003003200BD
:10F3D0001E0090009E007800310098001E0078000A
:10F3E0004F05BE004F04BE000080FA00000006007A
:10F3F0000200FA00000F78009E007800768040003E
:10F4000041002000BC030200010000009E007800C3
:10F410007680400018020200010000001E01780002
:10F4200060019800710198000000EB000080FA0074
:10F43000000006000200FA00000F78009E0078002D
:10F440006B8040000E070200010000000000EB008E
:10F450000080FA00000006000400FA00100798007F
:10F460000000EB00000F78001E00900076004000C6
:10F4700041002000BC030200010000001E009000BB
:10F480007600400018020200010000001E019000FA
:10F4900000099800110998001E0090009008900043
:10F4A000000890000DFC0700800078001E0090000E
:10F4B000210898001E009000A00890002003200062
:10F4C000808F50000500340060002000000F78009D
:10F4D0001E0090009E007800310098001E00780009
:10F4E0000080FA00000006000400FA00889FBE00B9
:10F4F0008A9FBE008C1F7800100798001E009000A5
:10F50000B04890001E00900060019000F001900053
:10F510001E009000204A90001E009000870B2000E3
:10F52000808343001E009000C504200080824200BA
:10F530001E0090002A082000000545001E009000D3
:10F54000F60540001E009000200E90001E00900066
:10F55000000C9000900C90001E009000680040008D
:10F560008F87E800E1FF9F00829FBE008F87E80041
:10F57000E4FF9F00050378008A0278000B02780000
:10F580008C0078000801BE0036FE0700E8875700AF
:10F59000000F78001E00E000030032001E00900003
:10F5A0009E007800310098001E0078004F06780019
:10F5B0004F05BE004F04BE000080FA0000000600A8
:10F5C0000200FA00000F78001E007800A0089000EA
:10F5D000E20E20001E004100BC03020001000000FA
:10F5E0001E007800A0089000421220001E0041007A
:10F5F000BC030200010000000000EB000080FA00E4
:10F60000000006000A00FA00889FBE008A9FBE0024
:10F61000400798004E009000A00890004E00900017
:10F6200076004000BC030200010000004E00900084
:10F63000B04890004E00900060019000F0019000F2
:10F640004E009000204A90004E009000870B200052
:10F65000808343004E009000C50420008082420059
:10F660004E0090002A082000000545004E00900042
:10F67000F60540004E009000000C9000900C9000A9
:10F680004E009000680040008F87E800E1FF9F0077
:10F69000829FBE008F87E800E4FF9F00050378008B
:10F6A0008A0278000B0278000801BE0041C0B30056
:10F6B00051FD0700E8875700200798002E009000B2
:10F6C0000000E00066003A000000EB001007980020
:10F6D0000040EB00004F7800150037001E80FB0053
:10F6E000CE0090006012B000010040009040780011
:10F6F000114798000A0037001E4090000080FB0070
:10F70000E10060001E00900001004000100798001A
:10F710001E4090000080FB000000D10010479800C0
:10F720001E4090000004E000F3FF3A001E4FE80086
:10F730001E80FB00CE009000A1109100810F5000B0
:10F74000E6FF3500660047000E07020001000000DA
:10F750000040EB00004F78003B0037001E00900097
:10F76000CF80DE005DFB0700800078004E00900037
:10F77000A015B000BC030200010000004E00900084
:10F7800042122000000141004E009000E40E2000D3
:10F79000000242004E009000A11520008080400031
:10F7A0004E0090007600400082017800040178004D
:10F7B000D5FD07004E009000B04890004E0090002C
:10F7C00060019000F00190004E009000204A9000EF
:10F7D0004E009000870B2000808343004E00900075
:10F7E000C5042000808242004E0090002A082000BC
:10F7F000000545004E009000F60540004E009000C8
:10F80000000C9000900C90004E00900068004000AA
:10F810008F87E800E1FF9F00829FBE008F87E8008E
:10F82000E4FF9F00050378008A0278000B0278004D
:10F830000801BE0041C0B300EFFC0700E887570095
:10F84000200798001E4FE8002E0090000000E00006
:10F8500003003A006E4090009E4F1000BFFF390039
:10F860002E0090000000E000030032004E009000E7
:10F87000AE009000310098002E0090004F05BE00B1
:10F880004F04BE000080FA00000006000800FA00E5
:10F89000889FBE00200798002E0090001040900026
:10F8A000EE4F500004003A002E00900020489000D7
:10F8B000604798000200370040C0B30060479800DE
:10F8C000EE409000214798002E0090007602400004
:10F8D0002E009000200C90002E0090000009900057
:10F8E000900990002E009000E80440008F87E80007
:10F8F0000040EB00E0FF9F006000B800809FBE006A
:10F900008F87E8002E409000E0FF9F008003EB000F
:10F910000003EB008002EB0088007800090078000B
:10F9200050FD0700E8875700000F78001E00E00038
:10F93000030032002E0090009E00780031009800F5
:10F940001E0078004F04BE000080FA000000060090
:10F950000800FA00889FBE008A1F780020079800E0
:10F960002E00900010409000F14F500004003A002B
:10F970002E00900020489000604798000200370059
:10F9800040C0B30060479800EE40900021479800C7
:10F990002E009000C4042000000242002E009000BF
:10F9A00025082000808242002E009000760440004E
:10F9B0002E009000A00C90002E00900000099000F6
:10F9C000900990002E009000680540008F87E800A5
:10F9D0000040EB00E0FF9F006000B800809FBE0089
:10F9E0008F87E8002E409000E0FF9F008003EB002F
:10F9F0000403780008027800890078000A00780083
:10FA000018FD0700E8875700000F78001E00E0008F
:10FA1000030032002E0090009E0078003100980014
:10FA20001E0078004F0578004F04BE000080FA00E9
:10FA3000000006000600FA00200798000E80E8008B
:10FA40000E07020001000000AE4090002E00900062
:10FA500068004000CCFA0700000F78001E00E000AC
:10FA6000030032002E0090009E00780031009800C4
:10FA70001E0078000080FA00000006000600FA0070
:10FA8000200798000000EB00000F78000E80E800CF
:10FA90000E070200010000002E4090000004E0006C
:10FAA000060032002E409000E14F5000030032006B
:10FAB00050002000000F7800190037002E00900041
:10FAC00010409000F34F50000B003A002E40900081
:10FAD0000004E00004003A00AE00900010C0B30043
:10FAE000904898000E003700AE009000D0C0B300E0
:10FAF000904898000A0037002E4090000004E00073
:10FB000004003A00AE00900010C0B300A048980076
:10FB100003003700AE00900060C0B300A04898001A
:10FB20001E00E000030032002E0090009E007800CE
:10FB3000310098001E0078000080FA0000000600E6
:10FB40000400FA00100798000E0078000E0702006B
:10FB5000010000001E4078000004E000FAFF3A00B7
:10FB60009E0090000000EB00B00098001E00900086
:10FB7000300090000080FA00000006000800FA0043
:10FB8000300798003E0090007600400011002000F1
:10FB9000BC030200010000003E009000805890006D
:10FBA000514798003E009000760040001100200070
:10FBB000BC030200010000003E009000805890004D
:10FBC000414798003E009000760040004100200030
:10FBD000BC030200010000003E00900076004000DF
:10FBE0001802020001000000008FBE003E009000DD
:10FBF000804890005E40900080CF500004003200AA
:10FC00003E00900068004000DE4090005EFA070071
:10FC10001E00BE0088070200010000003E009000A8
:10FC2000804890004E40900080CF50000400320089
:10FC30003E00900068004000CE40900052FA07005D
:10FC40000000EB000080FA00000006000200FA004D
:10FC5000000F78001E007800F3F90700800078009C
:10FC60001E007800310098001E00780030009000DF
:10FC70000000E00007003A009E0078006880400025
:10FC80008040EB0040FA0700800078001E007800FA
:10FC9000310098001E007800300090000080FA00CB
:10FCA000000006000200FA00000F78001E00780035
:10FCB000300090000000E0001F003A001E007800B5
:10FCC000104078000004E0001B003A001E00E8002D
:10FCD0000E070200010000001E007800A000900046
:10FCE0001000900061004000E08048001E01780094
:10FCF00010019800210198001E007800104090002B
:10FD0000F74F50000A003E001E007800104090009F
:10FD10000080FB0080004000E05423000080400091
:10FD2000900078001E0078000100010002003700FA
:10FD30001E007800D6FC07001E00780030009000FE
:10FD40000080FA00000006000200FA00000F7800B0
:10FD50001E007800DDF907000080FA0000000600B0
:10FD60009001FA000E007800B8FF0700020037008B
:10FD70000E007800CBFF07003E0090000000E0007E
:10FD800003003A001E4078000004E000F8FF320053
:10FD90000E007800ECFF07003E0090000080FA00A3
:10FDA000000006000600FA000000EB008008880052
:10FDB0000000EB00F00888000000EB00C00D880098
:10FDC00040AE81000000E00008003A00416D2000D4
:10FDD0009140780000CCB30000C06000D4E6B700CA
:10FDE0000000EB0030AD89003D00370040AE8100DF
:10FDF000E30F500005003C00E0032000000F7800F6
:10FE000010A1A8001081A8001500370040AE8100A5
:10FE1000FE0F500005003C00A00F2000000F7800EE
:10FE200010A1A8001081A9000D00370041AE81008B
:10FE3000400F2000808F500005003C00007D200016
:10FE4000000F780010A1A9001081A800040037005D
:10FE500000E82300000F780010A1A9001081A9007C
:10FE600040AE8100000178001E00780011000900FA
:10FE70000280D8000000E900200798002E009000C2
:10FE80006008880050AE8100800078002E0090004D
:10FE90000088B90042062000110009000280D80045
:10FEA00010079800416D20009140780000CCB3000D
:10FEB00000C060006041B300D4E6B7001E009000AF
:10FEC000F00D88001E009000E00D8800600020000A
:10FED000C00D880011E1A8002000200030AD89008D
:10FEE0000080FA00000006001200FA000000EB009B
:10FEF000800888000000EB00F00888000000EB009C
:10FF0000C00D880030AD8100E20F500013003A00B0
:10FF1000416D20009140780000CCB30000C060002B
:10FF2000D4E6B700C1002000E02B200070040200DE
:10FF3000010000000000EB0030AD89001098810046
:10FF40008000E800F00F2000808060000020230087
:10FF5000614078000004E000AC0032000000EB00DB
:10FF600020079800109881008000E800F00F200022
:10FF70000080600010988900264502000000000003
:10FF800008410200000000004007980026450200DA
:10FF9000000000000841020000000000CF80DE00E9
:10FFA000B022020000000000008FBE004E00900052
:10FFB0000000E00007003200CE009000F0F92000C1
:10FFC000808F500003003E002E0090000000E800EB
:10FFD000200798006011B8001E00BE000623020032
:10FFE000000000000000E00001003C000B003700B2
:10FFF00002002000832C24001E00BE000A23020001
:020000040001F9
:10000000000000000000E0000100350003003700A0
:100010002E0090000000E800200798002E009000BD
:10002000E20F5000110032000000EB002098890020
:1000300011012000A02C200070040200010000002B
:1000400011012000B02D2000E60302000100000095
:100050008001EB0002FA20001100200020032000A4
:100060009A47020000000000400798004E009000F0
:10007000E30F500005003E00E00320003007980029
:1000800010A1A8001081A800150037004E009000B4
:10009000FE0F500005003E00A00F20003007980022
:1000A00010A1A8001081A9000D003700CE0090001B
:1000B000400F2000808F500005003E00007D200092
:1000C0003007980010A1A9001081A8000400370093
:1000D00000E823003007980010A1A9001081A900B2
:1000E0003E0090004E019000110009000280D800EF
:1000F0000000E900600798002E009000E20F500019
:100100000E00320001012000902F2000E6030200C3
:10011000010000008001EB00320620008000EB00AF
:10012000200320009A47020000000000CF80DE007C
:10013000B022020000000000008FBE00020020007C
:10014000832C24001E00BE000E23020000000000CD
:10015000008FBE006E009000CF80DE00B022020053
:100160000000000070079800010F98006E009000DA
:100170000000E00008003D00020020000378240099
:100180007E0090008E089000942302000000000082
:1001900070079800010F98001E01BE007E009000BD
:1001A0008E0890004E24020000000000B6240200D9
:1001B0000000000050079800416D20009140780039
:1001C00000CCB30000C060006041B300D4E6B700CB
:1001D0005E009000F00D88005E009000E00D880049
:1001E00060002000C00D88006E009000600888004C
:1001F00011E1A800A100200090302000700402004E
:10020000010000002000200030AD89000080FA00CD
:10021000000006002400FA0030AD8100E20F50001B
:1002200005003A00F1012000303120007004020086
:1002300001000000F3023700F1002000203320000D
:10024000E6030200010000000000EB00F008880057
:100250000000EB0080088800D8A2A8006168200098
:100260009140780000CCB30000C060004041B30072
:1002700086E6B700A003200080088800100307006E
:1002800040079800510798000000EB0060079800B5
:100290000000EB00700798004E029000DE02900014
:1002A0006E039000FE039000F0FF23000100200089
:1002B0006011B8000020E10001A8E10002B0E100F7
:1002C00003B8E100130036004E009000DE009000FD
:1002D0006E019000FE019000C819DD004812DE009A
:1002E000830172004811DD00480ADE00020172003D
:1002F000C808DD004802DE00810072004800DD0011
:10030000400798005107980062079800730798000B
:100310000D003700B1002000202E2100E60302006E
:1003200001000000A000200080088800E40207000F
:1003300040079800510798000000EB006007980004
:100340000000EB00700798004E029000DE02900063
:100350006E039000FE039000F0F9200001002000E1
:100360006011B8000020E10001A8E10002B0E10046
:1003700003B8E100080036004E009000DE00900057
:10038000BEDC02000000000020CC2A00C4DB02001A
:1003900000000000910237004E009000DE00900047
:1003A0006E019000FE019000E00F5000E08F5800B9
:1003B000E00F5900E08F590085023200B1002000A3
:1003C000202E2100E6030200010000004E009000F4
:1003D000EB020700008FBE000000EB002007980032
:1003E0000000EB00300798003E02BE002E03BE0066
:1003F00000A82100610020006011B8000020E10089
:1004000001A8E10002B0E10003B8E1009500360068
:100410003E00BE002E01BE00E00F5000E08F5800ED
:10042000E00F5900E08F5900070035003E00BE0084
:100430002E01BE00EC24020000000000001798000E
:10044000111798001F0037003E02BE002E03BE00A9
:1004500010002000010020006011B80004006000BE
:100460008580600006016100878161003E02BE0058
:100470002E03BE008703D1000683D3008582D300FC
:100480000482D300000072008180720002017300B8
:1004900083817300EC240200000000000017980024
:1004A000111798000E1190009E1190000E109000F0
:1004B0009E10900094230200000000000017980096
:1004C000111798000E1190009E119000703B2400AF
:1004D000A13B25000E23020000000000642502005D
:1004E000000000004007980051079800620798003C
:1004F000730798004E009000DE0090006E0190009F
:10050000FE019000046A2800150020006033B80046
:100510009A26020000000000BEDC0200000000007D
:10052000E0C2B3008EDF0200000000004E00900029
:10053000DE0090006E019000FE019000046A280029
:10054000150020006033B800A8260200000000005B
:1005500040079800510798006207980073079800B9
:100560004E029000DE0290006E039000FE039000A9
:10057000F0702200010020006011B8000020E100AE
:1005800001A8E10002B0E10003B8E10003003E0071
:1005900000C3B3008EDF0200000000004E02900096
:1005A000DE0290006E039000FE039000703E20007B
:1005B000010020006011B8000020E10001A8E10066
:1005C00002B0E10003B8E10003003E0000C3B30045
:1005D0008EDF0200000000004E029000DE0290005C
:1005E0006E039000FE039000300620000100200002
:1005F0006011B8000020E10001A8E10002B0E100B4
:1006000003B8E10003003E0000C3B3008EDF020028
:10061000000000004E029000DE0290006E03900089
:10062000FE03900090002000010020006011B8003F
:100630000020E10001A8E10002B0E10003B8E10000
:1006400003003E0000C3B3008EDF02000000000084
:100650004E009000DE00900032DC0200000000003E
:10066000D70137003E02BE002E03BE00B0E12E00CF
:10067000110020006011B8000020E10001A8E10095
:1006800002B0E10003B8E100850036003E00BE0084
:100690002E01BE00E00F5000E08F5800E00F59001F
:1006A000E08F5900070035003E00BE002E01BE005D
:1006B000EC24020000000000600F9800710F980009
:1006C0001F0037003E02BE002E03BE0010002000B7
:1006D000010020006011B800040060008580600007
:1006E00006016100878161003E02BE002E03BE004C
:1006F0008703D1000683D3008582D3000482D30010
:100700000000720081807200020173008381730017
:10071000EC24020000000000600F9800710F9800A8
:100720006E099000FE0990006E089000FE0890008F
:100730009423020000000000600F9800710F9800E1
:100740006E099000FE099000902F20005121250095
:100750000E230200000000006425020000000000DB
:1007600040079800510798006207980073079800A7
:100770004E009000DE0090006E019000FE0190009F
:1007800004712200050020006033B8009A260200A0
:1007900000000000BEDC020000000000E0C2B30068
:1007A0008EDF0200000000004E009000DE0090008E
:1007B0006E019000FE0190000471220005002000EF
:1007C0006033B800A826020000000000400798002F
:1007D0005107980062079800730798004E02900036
:1007E000DE0290006E039000FE039000703E200039
:1007F000010020006011B8000020E10001A8E10024
:1008000002B0E10003B8E10003003E0000C3B30002
:100810008EDF0200000000004E029000DE02900019
:100820006E039000FE0390003006200001002000BF
:100830006011B8000020E10001A8E10002B0E10071
:1008400003B8E10003003E0000C3B3008EDF0200E6
:10085000000000004E029000DE0290006E03900047
:10086000FE03900090002000010020006011B800FD
:100870000020E10001A8E10002B0E10003B8E100BE
:1008800003003E0000C3B3008EDF02000000000042
:100890004E009000D2DD0200000000004801370049
:1008A0003E02BE002E03BE0000C42900010020004D
:1008B0006011B8000020E10001A8E10002B0E100F1
:1008C00003B8E100760036003E00BE002E01BE00F7
:1008D000E00F5000E08F5800E00F5900E08F590002
:1008E000070035003E00BE002E01BE00EC240200D1
:1008F00000000000400F9800510F98001F003700C3
:100900003E02BE002E03BE001000200001002000A9
:100910006011B8000400600085806000060161007D
:10092000878161003E02BE002E03BE008703D10016
:100930000683D3008582D3000482D30000007200B6
:10094000818072000201730083817300EC24020035
:1009500000000000400F9800510F98004E099000D1
:10096000DE0990004E089000DE08900094230200FB
:1009700000000000400F9800510F98004E099000B1
:10098000DE09900080B22600E10625000E23020059
:1009900000000000642502000000000040079800ED
:1009A0005107980062079800730798004E00900066
:1009B000DE0090006E019000FE019000843E200059
:1009C000050020006033B8009A26020000000000F5
:1009D000BEDC020000000000E0C2B3008EDF0200B7
:1009E000000000004E009000DE0090006E019000BC
:1009F000FE019000843E2000050020006033B80016
:100A0000A826020000000000400798005107980047
:100A100062079800730798004E029000DE02900073
:100A20006E039000FE0390003006200001002000BD
:100A30006011B8000020E10001A8E10002B0E1006F
:100A400003B8E10003003E0000C3B3008EDF0200E4
:100A5000000000004E029000DE0290006E03900045
:100A6000FE03900090002000010020006011B800FB
:100A70000020E10001A8E10002B0E10003B8E100BC
:100A800003003E0000C3B3008EDF02000000000040
:100A90004E009000D2DD020000000000C8003700C8
:100AA0003E02BE002E03BE0090162300010020006F
:100AB0006011B8000020E10001A8E10002B0E100EF
:100AC00003B8E100670036003E00BE002E01BE0004
:100AD000E00F5000E08F5800E00F5900E08F590000
:100AE000070035003E00BE002E01BE00EC240200CF
:100AF00000000000200F9800310F98001F00370001
:100B00003E02BE002E03BE001000200001002000A7
:100B10006011B8000400600085806000060161007B
:100B2000878161003E02BE002E03BE008703D10014
:100B30000683D3008582D3000482D30000007200B4
:100B4000818072000201730083817300EC24020033
:100B500000000000200F9800310F98002E0990002F
:100B6000BE0990002E089000BE0890009423020059
:100B700000000000200F9800310F98002E0990000F
:100B8000BE09900000C22B00E1EB24000E230200FE
:100B900000000000642502000000000040079800EB
:100BA0005107980062079800730798004E00900064
:100BB000DE0090006E019000FE01900044062000CF
:100BC000050020006033B8009A26020000000000F3
:100BD000BEDC020000000000E0C2B3008EDF0200B5
:100BE000000000004E009000DE0090006E019000BA
:100BF000FE01900044062000050020006033B8008C
:100C0000A826020000000000400798005107980045
:100C100062079800730798004E029000DE02900071
:100C20006E039000FE039000900020000100200061
:100C30006011B8000020E10001A8E10002B0E1006D
:100C400003B8E10003003E0000C3B3008EDF0200E2
:100C5000000000004E00900030DE020000000000A6
:100C6000570037003E00BE002E01BE00E00F5000CE
:100C7000E08F5800E00F5900E08F59000700350061
:100C80003E00BE002E01BE00EC2402000000000069
:100C9000000F9800110F98001F0037003E02BE00A1
:100CA0002E03BE0010002000010020006011B800DB
:100CB000040060008580600006016100878161009A
:100CC0003E02BE002E03BE008703D1000683D30080
:100CD0008582D3000482D3000000720081807200FC
:100CE0000201730083817300EC2402000000000005
:100CF000000F9800110F98000E0990009E099000B7
:100D00000E0890009E08900094230200000000004E
:100D1000000F9800110F98000E0990009E09900096
:100D20000068290081D124000E2302000000000089
:100D30006425020000000000400798005107980059
:100D400062079800730798004E009000DE00900044
:100D50006E019000FE019000A4002000050020001C
:100D60006033B8009A26020000000000BEDC0200DA
:100D700000000000E0C2B3008EDF020000000000AF
:100D80004E009000DE0090006E019000FE01900089
:100D9000A4002000050020006033B800A82602004F
:100DA0000000000040079800510798006207980073
:100DB000730798004E00900030DE02000000000033
:100DC00020CC2A00C4DB0200000000000300370032
:100DD00060CC2A00C4DB0200000000006168200033
:100DE0009140780000CCB30000C06000F041B30037
:100DF00086E6B7000000EB00F00888000000EB007A
:100E0000800888000080FA00000006000400FA0054
:100E10000000EB00F00888000000EB00800888006C
:100E2000D8A2A800616820009140780000CCB300EF
:100E300000C060004041B30086E6B700A003200078
:100E4000800888001E000700008FBE00F00F200001
:100E500001002000BE0F1000AE8F18000700360002
:100E60001E00BE00C808DD000080FD008040780044
:100E70000040EB00008FBE0004003700A0002000FF
:100E8000800888000E000700008FBE006168200007
:100E90009140780000CCB30000C06000F041B30086
:100EA00086E6B7000000EB00F00888000000EB00C9
:100EB000800888001E00BE000080FA0000000600C6
:100EC0000000FA000080EB00700888000080EB0052
:100ED000600888000000EB00400888000000EB007C
:100EE000300888000000EB00B00888000000EB002C
:100EF000A008880080002000F0088800400F200033
:100F0000E008880000402200D00888008780A900FF
:100F10001FE1A80011E1A80087C0BF007040600079
:100F20000004E000FCFF320011E1A9001FE1A9006C
:100F30003008800060AD890040088000010020007A
:100F400040AD890051AD890040AD810051AD8100B7
:100F5000C001DD000200200060AD81000100200022
:100F6000020040008380480040AD890051AD8900F7
:100F700040AD810051AD81000080FA000000060004
:100F80000200FA00000F780084A0A9008420A900C4
:100F9000F16820009140780000CCB30000C06000F0
:100FA0004041B3008FE6B700E1682000914078002F
:100FB00000CCB30000C060004041B3008EE6B70033
:100FC0000000EB00B00888000000EB00A0088800DB
:100FD00080002000F00888001FE1A80030C0200039
:100FE000400A880030802000000A8800400120006C
:100FF000500A880040012000100A880004003700D1
:10100000200A80000100200010AE890021AE890076
:1010100040C1BF00684060000004E000F8FF3A00F3
:1010200004003700600A800001002000F0AD890054
:1010300001AE890048C1BF00684060000004E000C4
:10104000F8FF3A0040C1BF00684060000004E000C3
:10105000FCFF3200200A800001002000F0AD890072
:1010600001AE8900600A800001002000B0AD890057
:10107000C1AD89006000B80070AD890081AD890004
:101080000000EB0030AE89003100370040C1BF00E6
:10109000684060000004E000FCFF3200200A80008D
:1010A0000100200010AE890021AE8900600A800096
:1010B00001002000D0AD8900E1AD8900D2AD8100F2
:1010C000E3AD8100B0AD8100C1AD810000005100F1
:1010D00081805900C002DD000400200012AE8100B2
:1010E00023AE8100F0AD810001AE8100000051000F
:1010F00081805900040040008580480090AD89003F
:10110000A1AD890072AD810083AD810090AD8100F9
:10111000A1AD8100020040008380480070AD8900CD
:1011200081AD8900D0AD8100E1AD8100B0AD890015
:10113000C1AD890010AE810021AE8100F0AD890003
:1011400001AE890030AE81000000E80030AE8900B9
:1011500030AE81009E0F5000CCFF39000000EB0044
:10116000000A88000000EB00100A88001FE1A900B7
:1011700074AD810085AD81001E0078006101B8006A
:101180000400BE00BC270200000000000080FA003E
:10119000000006000200FA00E05D230090407800A5
:1011A00063C060000080FB00000F78001E00780024
:1011B000E10F5000100032009E007800E18F5000D7
:1011C00004003C001E0078000000E000080032002F
:1011D0000E0037009E007800E28F500008003200B9
:1011E0001E007800E30F50000700320007003700B0
:1011F000D8A2A80005003700D882A8000300370055
:10120000D902A80001003700D802A800E1002000A0
:1012100010342000E6030200010000000080FA0004
:10122000000006000200FA00E05D23009040780014
:1012300063C060000080FB00000F78001E00780093
:10124000E10F5000110032009E007800E18F500045
:1012500004003C001E0078000000E000080032009E
:10126000120037009E007800E28F50000A00320022
:101270001E007800E30F50000A0032000B00370018
:10128000D8A2A900DAA2A80008003700D882A900D5
:10129000DA82A80005003700D902A900DB02A80005
:1012A00002003700D802A900DA02A800810020005D
:1012B000F034200070040200010000000080FA00F9
:1012C000000006000200FA00E05D23009040780074
:1012D00063C060000080FB00000F78001E007800F3
:1012E000E10F5000110032009E007800E18F5000A5
:1012F00004003C001E0078000000E00008003200FE
:10130000120037009E007800E28F50000A00320081
:101310001E007800E30F50000A0032000B00370077
:10132000D8A2A900DAA2A90008003700D882A90033
:10133000DA82A90005003700D902A900DB02A90062
:1013400002003700D802A900DA02A90071002000CB
:101350007035200070040200010000000080FA00D7
:10136000000006000400FA00E05D230090407800D1
:1013700063C060000080FB00100798001E00900012
:10138000E10F5000170032009E009000E18F5000E6
:1013900004003C001E0090000000E0000800320045
:1013A000260037009E009000E28F500016003200A9
:1013B0001E009000E30F50001A0032001F0037009B
:1013C000D8A2A8000000000000000000DAC2BF00A0
:1013D0000080FB004500DE0061406000004F7800A7
:1013E00016003700D882A8000000000000000000AE
:1013F000DAC2BF000080FB004400DE0061406000F4
:10140000004F78000D003700D902A800000000004E
:1014100000000000DBC2BF0061406000004F7800A8
:1014200006003700D802A8000000000000000000FD
:10143000DAC2BF0061406000004F78001E80FB00F0
:101440000080FA00000006000E00FA000040EB00E9
:10145000404798000000EB00800888000000EB0087
:10146000F00888000000EB00C00D880030AD81005E
:10147000E20F500014003A00109881008000E8004C
:10148000F00F200080806000002023006140780081
:101490000004E0000C003A00416D2000914078000B
:1014A00000CCB30000C06000D4E6B700C10020004B
:1014B000E02B200070040200010000000000EB009F
:1014C00030AD89007D003700109881008000E80071
:1014D000F00F20000080600010988900264502006F
:1014E000000000000841020000000000CF80DE0084
:1014F000B022020000000000008FBE002098810092
:101500000000E00008003A000200200043332400FD
:101510001E00BE0006230200000000000000E000E4
:1015200001003C00120037000000EB002098890009
:101530003101200080382100700402000100000009
:101540008001EB00420B20008000EB00A005200092
:101550009A47020000000000CF80DE00B0220200A7
:1015600000000000008FBE0010C0B300404798008C
:1015700010A1A8001081A800204E2000400798006C
:1015800002002C00A35524001E00BE000E23020002
:1015900000000000008FBE004E009000CF80DE00F3
:1015A000B022020000000000500798006107980078
:1015B0004E0090000000E00008003D000200200006
:1015C000037824005E009000EE0090009423020057
:1015D0000000000050079800610798001E01BE003F
:1015E0005E009000EE0090004E240200000000001B
:1015F0000200200083272400942302000000000042
:10160000B62402000000000030079800416D200061
:101610009140780000CCB30000C060006041B3008E
:10162000D4E6B7003E009000F00D88003E00900028
:10163000E00D880060002000C00D88004E00900082
:101640006008880011E1A800C1002000B039210025
:1016500070040200010000002000200030AD89006D
:101660004E409000E14F500014003A00130020005B
:10167000420B20008000EB000080EB009A47020044
:1016800000000000CF80DE00B02202000000000059
:10169000008FBE006011B8001E00BE000A230200C9
:1016A000000000000000E00001003500B0FF37003E
:1016B000B0CE2A00C4DB0200000000000080FA0067
:1016C000000006000400FA00A0080200010000006B
:1016D0000004E0002200320032C2BF006840600017
:1016E0000004E000040032003100200000E020008F
:1016F000E60302000100000032C2BF006440600047
:101700000004E000040032003100200030E020003E
:10171000E603020001000000900802000100000042
:10172000000F780032C2BF00624060000004E00099
:1017300008003200F100200060E02000E603020013
:101740000100000090118000D1FF2F000100600017
:10175000901188001E0078001007980006003700DE
:10176000F100200050E12000E6030200010000002B
:101770000000EB00100798001E0090000080FA00A7
:10178000000006000200FA00000F78001E0078003A
:101790007C080200010000000000EB000080FA005D
:1017A000000006000000FA0001022000B0EC20005A
:1017B000E603020001000000C05C23001040780036
:1017C00030DE02000000000000C2B3008EDF020025
:1017D00000000000C05C230010407800E94F50007A
:1017E00007003A00C0118000D2DD020000000000B6
:1017F00000C2B3008EDF0200000000000C003700C2
:10180000C05C2300104078000080FB008000400096
:10181000E05723000080400010007800D2DD020075
:101820000000000000C2B3008EDF020000000000D4
:10183000806423009040780063C0600030DE0200C6
:101840000000000000C2B3008EDF020000000000B4
:10185000806423001080FB004200DE0061406000D5
:1018600030DE02000000000000C2B3008EDF020084
:1018700000000000806423001080FB004300DE00B5
:101880006140600030DE02000000000000C2B300D2
:101890008EDF020000000000E05D23001080FB00EE
:1018A0004400DE006140600030DE02000000000005
:1018B00000C2B3008EDF02000000000031002000F3
:1018C00090BF2000E6030200010000000080FA0043
:1018D000000006001000FA000000EB00200798004E
:1018E0006000B800008FBE0081642300F0CDB3001B
:1018F00091486000264502000000000008410200F7
:1019000000000000700798007E009000EA0F500071
:1019100005003A00264502000000000008410200D0
:10192000000000002007980026450200000000008B
:1019300008410200000000006007980026450200F0
:10194000000000000841020000000000500798005D
:1019500026450200000000000841020000000000CF
:1019600040079800264502000000000008410200E0
:1019700000000000300798007E0090000000E000AA
:10198000090034007E009000EA0F500006003C0081
:101990007E0090000040E90080407800C05C230099
:1019A00001487800020037000000EB007007980043
:1019B0006E0090000000E0000C0034006E0090000B
:1019C000E40F500009003C006E0090000040E90068
:1019D000E34060008064230063C16000C1CFB300B6
:1019E00010C8600010487100020037000000EB00D2
:1019F000700798005E0090000000E0000D003400C9
:101A00005E009000E20F50000A003C005E00900073
:101A10000040E900E140600080642300E1C0600014
:101A20004209DD00B1CFB30010C86000104871005A
:101A3000020037000000EB00700798004E00900095
:101A40000000E0000D0034004E009000E20F500056
:101A50000A003C004E0090000040E900E1406000B8
:101A600080642300E1C060004309DD0071CFB30052
:101A700010C8600010487100020037000000EB0041
:101A8000700798003E0090000000E0000F00340056
:101A90003E009000E20F50000C003C003E00900021
:101AA0000040EA00E1406000E35D2300134078005D
:101AB000E1C060004409DD00F1CEB30001406000E8
:101AC0000240700080497800020037000000EB00FF
:101AD000700798007E0090000000E0008A003A0045
:101AE0000000EB0020988900E10B2000C095200049
:101AF00070040200010000008001EB00B200200031
:101B000011002000100020009A4702000000000091
:101B10000040E90080407800C05C23000148780064
:101B2000C05C230010407800EA4F50000C003A00DF
:101B3000C15C230080C0B300804878001000200002
:101B400001002000008FBE008164230000C2B300AA
:101B50009148700000C02A00C4DB020000000000B1
:101B6000C05C230010407800E94F50001C003A0090
:101B700091012000702F210070040200010000007C
:101B80008001EB00F4232400F50020001200200067
:101B900000202C0011002000264902000000000057
:101BA000008FBE001E01BE0000902000D103200067
:101BB000BC270200000000000081EB008081EB00E8
:101BC000021F4000039748009E01780023079800F9
:101BD0006000B800008FBE002E009000C011880089
:101BE0004105200040E22000E60302000100000061
:101BF0008001EB00420020001100200010002000B6
:101C00009A470200000000000040E900E340600045
:101C10008064230063C16000C1CFB30010C86000BE
:101C2000104871001102200080E72000E603020046
:101C3000010000008001EB002200200011002000C4
:101C4000100020009A470200000000000040E90058
:101C5000E140600080642300E1C060004209DD00D3
:101C6000B1CFB30010C860001048710021032000FC
:101C700090E92000E6030200010000008001EB0073
:101C80002200200011002000100020009A470200CE
:101C9000000000000040E900E14060008064230093
:101CA000E1C060004309DD0071CFB30010C86000DF
:101CB00010487100F104200050A5200070040200BB
:101CC000010000008001EB00220020001100200034
:101CD000100020009A470200000000000040EA00C7
:101CE000E1406000E35D230013407800E1C0600044
:101CF0004409DD00F1CEB3000140600002407000F5
:101D00008049780017003700C05C2300104078003D
:101D1000E94F500012003A002E009000CF80DE0004
:101D2000008FBE001E01BE0000902000D1032000E5
:101D3000BC270200000000000081EB008081EB0066
:101D4000021F4000039748009E0178002307980077
:101D50006000B800008FBE002E009000C011880007
:101D600090FE07000080FA00000006000600FA005E
:101D7000C05C230010407800E94F500019003A0081
:101D8000806423001080FB004200DE0061406000A0
:101D900080417800806423009040780063C0600038
:101DA00080427800806423001080FB004300DE0046
:101DB0006140600000417800E05D23001080FB007E
:101DC0004400DE006140600080407800C011800067
:101DD0000342780085417800B2070200010000004C
:101DE0001F003700806423001080FB004200DE00EB
:101DF00061406000004178008064230090407800DA
:101E000063C0600080417800806423001080FB0084
:101E10004300DE006140600080427800E05D230006
:101E20001080FB004400DE00614060000043780049
:101E3000C05C2300104078000080FB008000400060
:101E4000E057230000804000100078000242780034
:101E50000541780086407800B207020001000000CA
:101E6000806423001040780063406000E34F50001E
:101E700003003A00D15C230090C0B3008048780092
:101E80004A08020001000000C111800040118000DA
:101E9000808F500004003100010220000031210039
:101EA00070040200010000008064230010407800EC
:101EB0000042B2000004E0005C003200580802005A
:101EC00001000000A0C12A00C4DB020000000000E5
:101ED0000000EB00BA0107006B0107001007980033
:101EE00021079800A0C12A00C4DB02000000000006
:101EF0001E009000AE009000E00F5000E08F5800F0
:101F000019003A00806423001080FB004200DE00CC
:101F10006140600080417800806423009040780038
:101F200063C0600080427800806423001080FB0062
:101F30004300DE006140600000417800E05D230066
:101F40001080FB004400DE006140600080407800AB
:101F500070AC81000342780085417800B20702002E
:101F60000100000027003700C15C230090C0B300CF
:101F7000804878001E019000AE0190000090200083
:101F8000D1032000BC2702000000000061005000C7
:101F9000E080580010079800210798001E0090006C
:101FA000000F7800806423001080FB004200DE00F8
:101FB0006140600080417800806423009040780098
:101FC00063C0600080427800806423001080FB00C2
:101FD0004300DE006140600000417800E05D2300C6
:101FE0001080FB004400DE0061406000804078000B
:101FF0001E0078000342780085417800B207020095
:10200000010000004A08020001000000C111800028
:1020100040118000808F5000040031000102200038
:102020000031210070040200010000000080FA006D
:10203000000006000000FA0058080200010000003D
:102040000080FA00000006000400FA00000F78008B
:102050001E007800100798001E009000E20F50004C
:10206000480032001E009000E20F500007003E00C2
:102070001E0090000000E0000B0032001E009000E7
:10208000E10F50000D0032006E0037001E0090007E
:10209000E30F5000090032001E009000E40F5000D2
:1020A0005900320067003700C1072000B0EE200061
:1020B000E60302000100000066003700B1002000C6
:1020C00070F620007004020001000000E100200012
:1020D00040522100700402000100000016050200B9
:1020E000010000000000E0005A0032009011800062
:1020F000D1FF2F0001006000901188000000370020
:10210000D3C2BF000044B2000004E000510032001E
:1021100032C2BF00614060000004E00003003200F2
:10212000B01180008EDF020000000000C4DF02005A
:1021300000000000E14F500008003A0033C2BF0029
:10214000624060000004E00004003A00ECDF02009E
:10215000000000000080FB00A011880032C2BF0018
:10216000624060000004E000E5FF32009011800052
:10217000D1FF2F000100600090118800CB02A90060
:10218000DFFF3700E1002000F0F7200070040200BC
:1021900001000000F1002000003321007004020063
:1021A0000100000090118000D1FF2F0001006000AD
:1021B00090118800D3C2BF000044B2000004E000C8
:1021C00024003200A0080200010000000004E0002A
:1021D0000400320090080200010000008EDF0200BF
:1021E00000000000C4DF020000000000E14F5000CA
:1021F000F0FF3A00ECDF0200000000000080FB006E
:10220000000F78001300370058080200010000009A
:102210000000EB00EA0007004A080200010000008D
:10222000C111800040118000808F500009003100F2
:1022300001022000003121007004020001000000B2
:102240000400370041022000E01D2000700402005D
:10225000010000000080FA00000006000000FA0003
:1022600091118000D0FF2F00008060009011880045
:10227000806423001044A000E15D23001140780039
:102280000020A00080487800C1012000D0F8200084
:1022900070040200010000000080FA000000060047
:1022A0000000FA0081642300F0CEB3009148600082
:1022B000E15D2300114078000020A10080487800F3
:1022C0004101200090FA200070040200010000008B
:1022D0000080FA00000006000200FA000000EB0097
:1022E000000F78003400370080642300104078002D
:1022F000704060000004E0002B003200C0C12A00E2
:10230000C4DB02000000000061002000E074200037
:10231000E60302000100000032C2BF006840600016
:102320000004E000040032003100200000E0200042
:10233000E60302000100000032C2BF0064406000FA
:102340000004E000040032003100200030E02000F2
:10235000E6030200010000009008020001000000F6
:10236000C80002000100000032C2BF0062406000ED
:102370000004E00008003200F100200060E02000CE
:10238000E60302000100000090118000D1FF2F0041
:102390000100600090118800C0C12A00C4DB020067
:1023A0000000000002003700900802000100000059
:1023B00010002000000F7800A008020001000000BB
:1023C0000004E000C8FF3A001E0078000080FA0018
:1023D000000006000000FA00B1002000A043210028
:1023E00070040200010000000080FA0000000600F6
:1023F0000000FA000000EB00F00888000000EB008D
:102400008008880080002000800888000000EB0021
:10241000400888000000EB00300888000000EB0056
:10242000B00888000000EB00A008880080002000B1
:10243000F00888000080FA00000006000000FA00A2
:1024400011E1A9001FE1A900616820009140780016
:1024500000CCB30000C06000F041B30086E6B700D6
:102460000000EB00F00888000000EB008008880006
:102470000000EB00300888000000EB0040088800F6
:102480000080FA00000006001600FA0070079800AD
:10249000010F98006000B80050079800610798008D
:1024A0006000B80030079800410798006000B8004D
:1024B000100798002107980010002000000F7800F6
:1024C000380037001E007800C200DD00E0C12A009D
:1024D000008040001001BE007E0090008E08900039
:1024E000800F5100818F59002D0036001E00E90039
:1024F000C200DD00E0C12A00008040001001BE00E3
:1025000032079800430798001E007800C200DD00E3
:10251000E0C12A00008040001001BE005207980070
:10252000630798005E019000EE0190003E0090006D
:10253000CE00900000005100818059008101D1003F
:102540000081D3003E009000CE00900002014000C8
:10255000838148007E0090008E089000800F51001B
:10256000818F5900050031005E009000EE00900060
:10257000100F9800210F9800040037003E019000D2
:10258000CE019000120F9800230F98001E089000B3
:10259000AE0890001007980021079800040037004B
:1025A0001E0FE800E10020009E8F1000C5FF3400E0
:1025B0001E009000AE0090000080FA0000000600AF
:1025C0001000FA00500798000000EB004007980048
:1025D0006000B80020079800310798006000B8003C
:1025E000008FBE00DA62A900D862A8005E009000E9
:1025F0000000E00006003A003101200020532100D5
:10260000700402000100000001003700000000001B
:10261000DAC2BF00684060000004E000040032003D
:1026200022C2BF00614060000004E000F7FF3200FA
:1026300022C2BF00614060000004E0000B003200D5
:1026400030118000400798007CFF0700E100200067
:102650005054210070040200010000006000B80026
:102660006007980071079800760037000000EB00C3
:1026700040079800420037005DFF0700DAC2BF0044
:10268000684060000004E000FCFF32001FE1A80089
:1026900011E1A800DAC2BF00684060000004E00059
:1026A000FCFF3A0011E1A9001FE1A90061682000C8
:1026B0009140780000CCB30000C06000F041B3004E
:1026C00086E6B7000000EB00F00888000000EB0091
:1026D0008008880040088000010020002007980042
:1026E000310798002E009000BE009000C000DD0071
:1026F0000000200020079800310798003008800073
:102700006101B8002E009000BE0090000000410062
:102710008180490020079800310798004E00900002
:102720000000E000100032001E00BE00E00F50006C
:10273000E08F580004003A002E009000BE00900088
:10274000008FBE00080037002E009000BE009000F1
:10275000BE0F1000AE8F1800030036002E00900050
:10276000BE009000008FBE006000B80020079800F7
:10277000310798004E0090000000E80040079800E4
:102780004E009000F80F5000BBFF36002BFF0700F3
:102790001E01BE0000402200410F2000BC270200A5
:1027A00000000000008FBE005E0090000000E0000E
:1027B00021003A00009F240021002000BE0F1000DD
:1027C000AE8F18000500360081032000305521002F
:1027D000700402000100000017003700F100200023
:1027E000B0582100E6030200010000001E00BE00F8
:1027F00032DC02000000000041002000905A21005D
:102800007004020001000000F1002000A059210026
:10281000E6030200010000001E00BE001AFF0700D0
:1028200032DC02000000000041002000905A21002C
:1028300070040200010000001E00BE006007980046
:10284000710798006E009000FE0090000080FA0072
:10285000000006000000FA00E0C52A0098DB020034
:10286000000000000080FA00000006000400FA00EA
:1028700081642300C0CFB3009148600081642300CD
:10288000B0CFB300914860008164230070CFB300E3
:1028900091486000E15D2300114078000040A000F5
:1028A0008048780090AC810010B2890081642300D8
:1028B000F0CEB30091486000806423001080FB00DC
:1028C0004200DE00614060008041780080642300A7
:1028D0009040780063C060008042780080642300EC
:1028E0001080FB004300DE00614060000041780082
:1028F000E05D23001080FB004400DE0061406000CA
:102900008040780010B28100034278008541780051
:10291000B2070200010000004A08020001000000A6
:10292000CCFF070000003700A008020001000000F3
:102930000004E0000C0032008064230010407800A6
:10294000704060000004E0000500320090080200C2
:10295000010000008EDF02000000000002003700CE
:10296000900802000100000032C2BF006240600017
:102970000004E0000400320090118000D1FF2F001D
:102980000100600090118800C4DF02000000000018
:10299000E14F5000E4FF3A00ECDF020000000000CD
:1029A0008040780060642300014878006064230060
:1029B000104078000080FB004400DE00804078007A
:1029C00050642300014878005064230010407800D0
:1029D0000080FB00100798001E009000E50F5000DB
:1029E000C90032009E009000E58F50000A003C00B4
:1029F0001E009000E10F5000950032009E009000F4
:102A0000E48F5000B80032001E0090000000E0008B
:102A100009003200640137009E009000E68F5000EC
:102A2000C00032009E00900068805000E10F50000E
:102A30005D013E00F0003700606423001040780024
:102A40000080FB00000F78001E007800E20F5000AD
:102A5000190032009E007800E28F500007003C0011
:102A60001E0078000000E0000E0032009E0078009A
:102A7000E18F50000E003200710037001E00780018
:102A8000E70F5000210032009E007800EF8F5000C9
:102A90004F0032001E007800E30F50001400320097
:102AA00067003700580802000100000042013700AB
:102AB00068FF07009CFF370010C0B3008EDF0200E4
:102AC0000000000032C2BF00624060000004E0006D
:102AD0000400320090118000D1FF2F00010060003F
:102AE00090118800806423001044A0008EFF3700FE
:102AF00081642300F0CEB3009148600010C0B300A1
:102B00008EDF02000000000087FF370010C0B30016
:102B10008EDF0200000000005808020001000000E3
:102B2000ECDF0200000000000080FB004800DD0038
:102B300010B2890010C0B3008EDF02000000000058
:102B4000ECDF0200000000008080FB0010B281007A
:102B50000080700010B28900806423001080FB00A8
:102B60004200DE0061406000804178008064230004
:102B70009040780063C06000804278008064230049
:102B80001080FB004300DE006140600000417800DF
:102B9000E05D23001080FB004400DE006140600027
:102BA0008040780010B281000342780085417800AF
:102BB000B2070200010000004A0802000100000004
:102BC00010C0B3008EDF02000000000056FF370087
:102BD00010C0B3008EDF02000000000090118000E2
:102BE000D1FF2F0001006000901188000000370025
:102BF00032C2BF00614060000004E0000300320008
:102C0000B01180008EDF020000000000C4DF02006F
:102C100000000000E14F5000F5FF3A0033C2BF0052
:102C2000624060000004E000F1FF3A00ECDF0200C7
:102C3000000000000080FB00A0118800ECFF3700BE
:102C40000040EB008EDF02000000000036FF37007E
:102C50006064230090407800F0C0B30080C0600042
:102C6000606423000148780060642300104078000D
:102C70008040E800606423000148780010C0B30081
:102C80008EDF020000000000416423000040EB00E2
:102C9000804878000D003700ECDF020000000000E3
:102CA0000080FB007C0802000100000010C0B3009F
:102CB0008EDF020000000000406423001040780016
:102CC0008040E8004064230001487800406423000D
:102CD00090407800606423001040780080CF50005E
:102CE000EDFF390010FF37006064230010407800CA
:102CF000940A02000100000010C0B3008EDF020041
:102D00000000000008FF37006064230010407800D6
:102D1000120B0200010000008EDF02000000000024
:102D200001FF37006064230090407800F0C0B300DA
:102D300080C0600060642300014878006064230064
:102D400010407800EA4F5000030036006164230011
:102D5000A0C0B30080487800606423001040780071
:102D60000080FB00800040002059230000804000CC
:102D70001000780010B2890058080200010000001D
:102D8000806423001080FB004200DE006140600090
:102D900080417800806423009040780063C0600028
:102DA00080427800806423001080FB004300DE0036
:102DB0006140600000417800E05D23001080FB006E
:102DC0004400DE00614060008040780010B2810065
:102DD0000342780085417800B2070200010000003C
:102DE0004A0802000100000010C0B3008EDF02009C
:102DF00000000000CCFE370081642300C0CFB30088
:102E00009148600081642300B0CFB3009148600016
:102E10008164230070CFB30091486000E15D23001E
:102E2000114078000040A1008048780060642300D1
:102E3000104078000080FB004300DE00610060006D
:102E40000004E0000A003200806423009040780013
:102E500063C060000014A000E340600080642300B1
:102E600063C16000C1CFB30010C86000104871009A
:102E700060642300104078000080FB004200DE0008
:102E8000610060000004E0000A003200806423005A
:102E90009040780063C060000004A000E340600040
:102EA0008064230063C16000C1CFB30010C860001C
:102EB0001048710060642300104078000080FB001F
:102EC0000000D100610060000004E0000200320058
:102ED000806423001024A000606423001040780068
:102EE0000080FB00610060000004E000020032008E
:102EF000806423001034A000606423001040780038
:102F00000080FB004400DE000000A20061006000C1
:102F10000004E00004003200E15D2300114078006D
:102F20000040A0008048780058080200010000001E
:102F3000806423001080FB004200DE0061406000DE
:102F400080417800806423009040780063C0600076
:102F500080427800806423001080FB004300DE0084
:102F60006140600000417800E05D23001080FB00BC
:102F70004400DE00614060008040780010B28100B3
:102F80000342780085417800B2070200010000008A
:102F90004A0802000100000010C0B3008EDF0200EA
:102FA0000000000060FE37000040EB008EDF0200F2
:102FB000000000005CFE37000080FA000000060000
:102FC0000000FA00E15D2300114078000060A000DD
:102FD00080487800606523001040780068406000F9
:102FE0000004E00002003200DA82A900010037008C
:102FF000DA82A80060652300104078006840600015
:103000000004E00003003200F0C2B3008EDF0200D3
:1030100000000000A100200000BD2000700402009C
:10302000010000000080FA00000006000000FA0025
:10303000E15D2300114078000060A1008048780025
:103040006065230010407800684060000004E000E4
:1030500002003200DA82A90001003700DA82A800FB
:103060006065230010407800684060000004E000C4
:1030700003003200F0C2B3008EDF02000000000047
:10308000A100200000BD200070040200010000002B
:103090000080FA00000006000000FA0060652300CE
:1030A00010407800684060000004E0000200320038
:1030B000DA82A80001003700DA82A90060652300E7
:1030C00010407800684060000004E0000300320017
:1030D000F0C2B3008EDF020000000000B10020004B
:1030E000A0BD200070040200010000000080FA0072
:1030F000000006000000FA0000C0EB0055020700C7
:103100000080FB000080FA00000006000600FA00C4
:10311000100798001E0090004E020700004F780034
:10312000E05D2300104078000044B2000004E0009D
:10313000030032001E80FB002007980002003700C9
:103140000000EB00200798002E0090000080FA009D
:10315000000006000000FA0001022000C0DA200092
:10316000E603020001000000C05C2300104078006C
:103170000040E80030DE02000000000000C2B300A2
:103180008EDF0200000000006065230090407800A0
:1031900061C0600030DE02000000000000C2B30029
:1031A0008EDF020000000000606523001080FB003D
:1031B0000000D1006140600030DE0200000000002D
:1031C00000C2B3008EDF0200000000006065230033
:1031D0001080FB004200DE006140600030DE020033
:1031E0000000000000C2B3008EDF020000000000FB
:1031F000606523001080FB004300DE00614060003A
:1032000030DE02000000000000C2B3008EDF0200CA
:1032100000000000E05D23001080FB004400DE00A1
:103220006140600030DE02000000000000C2B30018
:103230008EDF0200000000003100200090BF20005F
:10324000E6030200010000000080FA000000060012
:103250000C00FA00264502000000000008410200B0
:103260000000000050079800264502000000000002
:1032700008410200000000004007980026450200B7
:103280000000000008410200000000003007980024
:103290002645020000000000084102000000000076
:1032A00020079800264502000000000008410200A7
:1032B00000000000000F780026450200000000001A
:1032C0000841020000000000100798005E00900016
:1032D0000000E000090034005E009000E40F5000A0
:1032E00006003C005E0090000040E900804078004D
:1032F000C05C230001487800020037000000EB00AA
:10330000500798004E0090000000E0000C003400D0
:103310004E009000E20F500009003C004E0090006B
:103320000040E900E14060006065230061C1600089
:10333000E1CFB30010C860001048710002003700F0
:103340000000EB00500798003E0090000000E000F5
:103350000D0034003E009000E20F50000A003C00D7
:103360003E0090000040E90061406000616523007C
:103370006140600000414000D0CFB3009148600040
:1033800091487100020037000000EB0050079800E0
:103390002E0090000000E0000D0034002E00900090
:1033A000E20F50000A003C002E0090000040E900AF
:1033B000E140600060652300E1C060004209DD007B
:1033C000B1CFB30010C86000104871000200370090
:1033D0000000EB00500798001E00E0000D003400D4
:1033E000200020009E0F10000A003C001E00780004
:1033F0000040E900E140600060652300E1C060003A
:103400004309DD0071CFB30010C86000104871009F
:10341000020037000000EB00500798001E009000EB
:103420000000E0000F0034001E009000E20F50008A
:103430000C003C001E0090000040EA00E1406000EB
:10344000E35D230013407800E1C060004409DD0023
:10345000F1CEB30001406000024070008049780066
:10346000020037000000EB00500798005E0090005B
:103470000000E0006C003A000000EB00209889009A
:1034800071032000C0CC2000700402000100000085
:103490008001EB00420020001100200010002000FD
:1034A0009A470200000000000040E90080407800D8
:1034B000C05C2300014878005103200030D0200078
:1034C00070040200010000008001EB0022002000D7
:1034D00011002000100020009A47020000000000A8
:1034E0000040E900E14060006065230061C16000C8
:1034F000E1CFB30010C86000104871003104200013
:1035000080D3200070040200010000008001EB0065
:103510002200200011002000200020009A47020015
:10352000000000000040E900614060006165230088
:103530006140600000414000D0CFB300914860007E
:103540009148710011032000B0D7200070040200E0
:10355000010000008001EB0022002000110020008B
:10356000100020009A470200000000000040E9001F
:10357000E140600060652300E1C060004209DD00B9
:10358000B1CFB30010C8600010487100D101200015
:10359000B036210070040200010000008001EB0041
:1035A0002200200011002000200020009A47020085
:1035B000000000000040E900E14060006065230079
:1035C000E1C060004309DD0071CFB30010C86000A6
:1035D00010487100F104200050A520007004020082
:1035E000010000008001EB002200200011002000FB
:1035F000100020009A470200000000000040EA008E
:10360000E1406000E35D230013407800E1C060000A
:103610004409DD00F1CEB3000140600002407000BB
:103620008049780001003700CAFE0700E15D2300F1
:10363000114078000060A100804878000080FA0006
:10364000000006000000FA00C05C23001040780073
:103650008080FB0000612300614078009400070037
:10366000606523001080FB004300DE0061406000C5
:10367000614060004401DD00A12D200091407800F0
:10368000F0CEB30000C0600002407000DAE2B70084
:103690000080FA00000006000000FA00D6000700D3
:1036A0000080FA00000006000600FA00000F780013
:1036B0001E0078006101B8001207980023079800E7
:1036C000F0002000010020001E019000AE019000DB
:1036D000800F5100818F590068003E001E0090004D
:1036E000AE009000006001000F00370013003700AB
:1036F0001E00370065003700600037005F003700AC
:103700005E0037005D0037005C0037005B0037006B
:103710002200370025003700270037002A00370035
:103720002C0037002F00370041032000C0DC2000B0
:1037300070040200010000005400370071002000F6
:10374000D05A20007004020001000000F1002000A7
:1037500000332100700402000100000011C0B3001A
:103760000040EB00C900070048003700710020004E
:10377000D05A20007004020001000000F100200077
:1037800000332100700402000100000011C0B300EA
:1037900010C0B300BD0007003C0037006165230086
:1037A000E0CFB3009148600010003700606523004F
:1037B0001004A0000D00370061652300D0CFB300D6
:1037C0009148600009003700606523001014A000D4
:1037D0000600370061652300B0CFB3009148600058
:1037E00002003700606523001024A00060652300FC
:1037F0009040780061C06000614060004601DD00DB
:103800002124200091407800F0CBB30000C060007C
:103810000240700042E2B700606523001080FB00A8
:103820000000D1006140600061416000312420004F
:1038300091407800E0CFB30000C06000024070000B
:1038400043E2B700606523001080FB004200DE0009
:103850006140600061406000004140003124200070
:1038600091407800D0CFB30000C0600002407000EB
:1038700043E2B70037FE0700040037004102200092
:10388000E01D200070040200010000000080FA002A
:10389000000006000000FA00010120001042210093
:1038A00070040200010000000080FA000000060021
:1038B0000200FA00004F780041E2A900E05D230019
:1038C00010407800704060000004E0000400320006
:1038D000DE62A800DE42A800DE82A80003003700F6
:1038E000DE62A900DE42A900DE82A900816A200012
:1038F0009140780000CCB30000C060006041B3008C
:10390000A8E6B700816D20009140780000CCB3009C
:1039100000C060007040B300D8E6B700716D2000B1
:103920009140780000CCB30000C060000034A000DB
:10393000D7E6B700DA82A800D882A900D842A90049
:10394000D862A800D822A9001E80FB0010128800AF
:1039500042A2A800606523009040780061C060002A
:10396000614060004601DD00212420009140780084
:10397000F0CBB30000C060000240700042E2B7002C
:10398000606523001080FB000000D10061406000F2
:10399000614160003124200091407800E0CFB30005
:1039A00000C060000240700043E2B7006065230081
:1039B0001080FB004200DE0061406000614060005A
:1039C000004140003124200091407800D0CFB30066
:1039D00000C060000240700043E2B7000000EB004E
:1039E000201288000000EB000012880041E2A800CD
:1039F0000080FA00000006000000FA0041E2A90081
:103A0000816A20009140780000CCB30000C06000C3
:103A1000F041B300A8E6B700816D20009140780026
:103A200000CCB30000C06000D8E6B700716D200084
:103A30009140780000CCB30000C06000D7E6B7002A
:103A4000DE62A900DE42A900DE82A9000080FA0041
:103A5000000006000200FA00004F78001E80FB0004
:103A60004012880085C0BF00644060000004E00090
:103A7000FCFF320040128000004F78008540A90012
:103A80001E80FB000080FA00000006000400FA001F
:103A9000204798003147980010C0B300004F7800CD
:103AA0000AE0020000000000D3FF070081000700C9
:103AB0002E4090000004E00002003A0042E2A8001C
:103AC00062E2A8002E409000E14F500002003E004C
:103AD00041E2A80061E2A8001E04E00009003A00EB
:103AE000DAC2BF00704060000004E0000500320050
:103AF000D0C5B300A6DF02000000000010C0B30074
:103B0000004F780040C2BF000042B2000004E00055
:103B10002F003A0060C2BF000042B2000004E00083
:103B20002B003A00401280001047980010C0B300EC
:103B30009E4F100005003A00B0C5B300A6DF02009A
:103B4000000000000040EB00004F78003E40900075
:103B50000004E000050032001E4090000080FB00E1
:103B6000B8DE02000000000006003700C0C5B30048
:103B7000A6DF0200000000001E409000A6DF020049
:103B80000000000040138000104798003E40900065
:103B90000004E0000B00320080C2B300A6DF020088
:103BA000000000001E4090000080FB00B8DE020014
:103BB0000000000090C2B300A6DF02000000000079
:103BC000030037001E409000A6DF02000000000046
:103BD00040C2BF000044B2000004E00009003A0007
:103BE00060C2BF000044B2000004E00005003A00DB
:103BF000E07F810001402000010060000000E00043
:103C000014003200E07F81000140200001006000CC
:103C10000000E00002003A00F8DF020000000000AF
:103C20000000EB00001288000000EB000013880089
:103C30003E4090000004E00004003200A0D02A00C2
:103C4000C4DB02000000000093FF3700CB02A90094
:103C50000F00370010E0020000000000C4DF020087
:103C600000000000E14F50009BFF3A00ECDF020033
:103C700000000000104798003E4090000004E00063
:103C800003003200B0D12A00C4DB020000000000B3
:103C900083000700C05C2300104078008080FB0098
:103CA000006123006140780001FF07000080FA00F6
:103CB000000006000000FA00D882A800D842A80040
:103CC000D862A800D822A800A16A200091407800FC
:103CD00000CCB30000C060009041B300AAE6B7007A
:103CE000E16A20009140780000CCB30000C0600081
:103CF0009041B300AEE6B700816A200091407800A1
:103D000000CCB30000C060008041B300A8E6B7005B
:103D1000916A20009140780000CCB30000C06000A0
:103D20007041B300A9E6B700C16A20009140780055
:103D300000CCB30000C060006041B300ACE6B70047
:103D4000D16A20009140780000CCB30000C0600030
:103D50007041B300ADE6B700C05C230010407800AE
:103D60008080FB0000612300614078000080FB0040
:103D700010128800606523009040780061C06000E8
:103D8000614060004601DD00212420009140780060
:103D9000F0CBB30000C060000240700042E2B70008
:103DA000606523001080FB000000D10061406000CE
:103DB000614160003124200091407800E0CFB300E1
:103DC00000C060000240700043E2B7000000EB005A
:103DD000201288000000EB0000128800C05C230065
:103DE000104078008080FB00006123006140780073
:103DF0000080FB001013880060652300904078006D
:103E000061C06000614060004601DD0021262000A5
:103E100091407800F0CBB30000C060000240700019
:103E200062E2B700606523001080FB000000D10053
:103E300061406000614160003126200091407800BF
:103E4000E0CFB30000C060000240700063E2B70042
:103E50000000EB00201388000000EB000013880036
:103E60000000EB00401288000000EB0040138800C7
:103E70004322A9006322A9004362A80042A2A9002C
:103E80006362A80062A2A90040C2A90060C2A900A2
:103E90004402A8006402A8000080FA0000000600A6
:103EA0000000FA0041E2A9004362A90061E2A90012
:103EB0006362A900A16A20009140780000CCB300A1
:103EC00000C06000F041B300AAE6B700E16A20003C
:103ED0009140780000CCB30000C06000F041B30016
:103EE000AEE6B700816A20009140780000CCB300B4
:103EF00000C06000F041B300A8E6B700916A20005E
:103F00009140780000CCB30000C06000F041B300E5
:103F1000A9E6B700C16A20009140780000CCB30048
:103F200000C06000F041B300ACE6B700D16A2000E9
:103F30009140780000CCB30000C06000F041B300B5
:103F4000ADE6B7000080FA00000006000000FA00AD
:103F5000C0D12A0098DB0200000000000080FA00B7
:103F6000000006001400FA00881F7800C15C2300DE
:103F700010C0B3008048780061652300E0CFB30033
:103F800091486000606523001014A0006165230063
:103F9000B0CFB30091486000E15D2300114078008C
:103FA0000040A00080487800C05C230010407800EA
:103FB0008080FB0040612300614078003CFE0700E8
:103FC000E2FF070000003700ECDF02000000000005
:103FD0008040780040652300014878004065230058
:103FE000104078000080FB004400DE008040780034
:103FF00030652300014878003065230010407800C8
:104000000080FB00100F98001E089000E40F500085
:10401000A20132009E089000E48F500007003C008F
:104020001E0890000000E0000E0032009E08900084
:10403000E18F500076013200F80137001E08900031
:10404000E60F5000A40132009E089000E68F500059
:104050009A0135001E089000E80F5000B2013200AE
:10406000EE01370040652300104078000080FB001F
:10407000000F98008E089000E58F500014003C005F
:104080000E089000E40F50003C003D008E089000A8
:10409000E18F50001A0032000E089000E10F50002E
:1040A00004003C008E0890000100E0001200320085
:1040B000530137000E089000E20F5000120032004A
:1040C0008E089000E38F5000170032004C0137003B
:1040D0000E089000ED0F50001A0032008E0890007C
:1040E000EE8F50001E0032000E089000E60F5000C8
:1040F00098003200420137003FFE0700CB01370035
:1041000092FF0700B0FF3700E0168000F1FE2F009D
:1041100001006000E016880010C0B3008EDF0200CE
:1041200000000000A8FF3700E01680000040A0005B
:10413000E016880010C0B3008EDF0200000000000F
:10414000A1FF370010C0B3008EDF020000000000A6
:104150008040EB0010C0B3004CFE07009AFF370010
:1041600010C0B3008EDF0200000000008040EB00B2
:104170000040EB0045FE070093FF3700ECDF020034
:10418000000000000080FB00500798005E009000D7
:104190004800DD0050079800ECDF0200000000003E
:1041A0008080FB005E0090000100700050079800C6
:1041B000ECDF0200000000000080FB0040079800D8
:1041C0004E0090004800DD0040079800ECDF020040
:1041D000000000008080FB004E0090000100700095
:1041E00040079800DE00900000002100808F500002
:1041F00004003E00CE00900000002100808F50009F
:10420000040036000040EB008EDF020000000000DA
:104210006DFF37000000EB006007980009003700D1
:10422000817F81006E00900000844000ECDF02007E
:1042300000000000004C78006E0090000000E800D4
:1042400060079800EE0090005E009000808F5000A4
:10425000F3FF39004065230010407800E44F500020
:1042600001003A00DA82A9000000EB006007980024
:1042700008003700817F81006E00900000804000C0
:1042800010407800F3FD07006E0090000000E80089
:1042900060079800EE0090005E009000808F500054
:1042A000F4FF3900100020009A0102000100000014
:1042B0000000EB006007980009003700817F810053
:1042C0006E0090000084400000C0EB00E1FD07009C
:1042D000004C78006E0090000000E8006007980035
:1042E000EE0090004E009000808F5000F3FF3900E8
:1042F0004065230010407800E44F500001003A0070
:10430000DA82A80010C0B3008EDF020000000000B7
:104310000000EB006007980009003700817F8100F2
:104320006E00900000804000104078008EDF020098
:10433000000000006E0090000000E8006007980098
:10434000EE0090004E009000808F5000F3FF390087
:104350001DFF370010C0B3008EDF02000000000018
:10436000ECDF020000000000804078004065230080
:104370000148780040652300104078000080FB0071
:1043800070079800FE009000E18F50000B00320093
:104390007E009000E20F500012003200FE009000FC
:1043A0000100E000010032009100370010C0B300AE
:1043B0008EDF02000000000003FF370010C0B300D2
:1043C0008EDF0200000000000040EB008EDF0200E4
:1043D0000000000010C0B3008EDF020000000000EB
:1043E000F9FE37006000B8002007980031079800F8
:1043F0000000EB006007980016003700ECDF0200B9
:1044000000000000804078004065230001487800EB
:104410002E009000BE0090004809DD00C801DE00BB
:10442000830171004801DD004065230010407800E1
:104430000080FB00010020000000710081807100FD
:1044400020079800310798006E0090000000E800F7
:10445000600798006E009000E30F5000E7FF360001
:104460006000B800008FBE000000EB0060079800FD
:1044700013003700ECDF02000000000080407800ED
:1044800040652300014878001E00BE004809DD0099
:10449000C801DE00830171004801DD004065230092
:1044A000104078000080FB0001002000001F710018
:1044B000019771006E0090000000E800600798000E
:1044C0006E009000E30F5000EAFF36002E019000CE
:1044D000BE019000F0FF2F0001002000800F51006E
:1044E000818F59000E003E00F0FF2F0001002000D8
:1044F000BE0F1000AE8F180009003E002E00900085
:10450000BE0090003E014000AE814800F0FF2F0049
:1045100001002000800F5100818F590004003600F7
:104520000040EB008EDF020000000000A6FE370016
:1045300010C0B3008EDF0200000000002E009000CB
:10454000600798002500370000C2B30041FD070056
:104550006E0090004800DE003EFD07006E009000F7
:104560003CFD07000040EB003AFD07008EDF020033
:10457000000000000080EB008080EB001E0F400078
:104580005E9748001E00BE00E00F5000E08F58000C
:104590008DFE320080C2B3002EFD07006E00900039
:1045A0004800DE002BFD07006E00900029FD07008B
:1045B0000040EB0027FD07008EDF02000000000036
:1045C0000080EB008080EB001E0F40005E974800EB
:1045D0006E0090000000E800600798001E00BE001A
:1045E000E00F5000E08F5800D7FF3A0076FE37000A
:1045F0000040EB008EDF02000000000072FE37007A
:104600000040EB008EDF0200000000006EFE37006D
:104610004065230090407800F0C0B30080C0600087
:104620004065230001487800406523001040780071
:104630008040E800406523000148780010C0B300C6
:104640008EDF020000000000216523000040EB0027
:10465000804878000A003700ECDF0200000000000C
:10466000FCFC07008EDF0200000000002065230034
:10467000104078008040E800206523000148780061
:1046800020652300904078004065230010407800AA
:1046900080CF5000F0FF39004BFE3700406523000B
:1046A00010407800940A02000100000010C0B3001E
:1046B0008EDF02000000000043FE3700406523004B
:1046C00010407800120B0200010000008EDF020093
:1046D000000000003CFE3700406523009040780059
:1046E00070C0B30080C060004065230001487800BE
:1046F0004065230090407800C05C230001487800AA
:10470000C05C2300104078008080FB0040612300E3
:104710006140780066FC070010C0B3008EDF020025
:104720000000000028FE370061652300E0CFB300E1
:104730009148600061652300D0CFB30091486000CC
:1047400061652300B0CFB30091486000E15D2300B4
:10475000114078000040A1008048780040652300A7
:10476000104078000080FB004200DE006100600025
:104770000004E00002003200606523001004A00085
:1047800040652300104078000080FB000000D1004D
:10479000610060000004E000020032006065230058
:1047A0001014A00040652300104078000080FB003A
:1047B000610060000004E000020032006065230038
:1047C0001024A00040652300104078000080FB000A
:1047D0004300DE000000A200610060000004E00071
:1047E00004003200E15D2300114078000040A00089
:1047F00080487800C05C2300104078008080FB0077
:10480000406123006140780029FC070010C0B3001C
:104810008EDF020000000000EBFD37000040EB00DF
:104820008EDF020000000000E7FD37004F04780033
:104830000080FA00000006000000FA0020D62A00DE
:1048400098DB0200000000000080FA000000060073
:104850001000FA00881F7800E15D23001140780005
:104860000040A00080487800E15D230011407800FE
:104870000030A10080487800C15C230010C0B30064
:1048800080487800D15C230080C0B3008048780065
:10489000A160230020C0B3008048780080C0EB00F6
:1048A00020C0B30062EF020000000000D822A9007F
:1048B000D842A900D862A80010C0B300F2F10200EB
:1048C00000000000DCFF070000003700ECDF020002
:1048D0000000000080407800E0602300014878007C
:1048E000E0602300104078000080FB004400DE0000
:1048F00080407800D060230001487800D060230019
:10490000104078000080FB006101B9004207980068
:1049100053079800F0002000010020004E01900095
:10492000DE019000800F5100818F5900CF033E00BF
:104930004E009000DE009000006001000F00370084
:104940009B003700F0003700020137003D033700BD
:10495000440337004A033700C40337005F033700BE
:10496000C203370032013700C0033700BF033700EE
:10497000BE033700BD03370091033700E06023001A
:10498000104078000080FB006101B90062079800C8
:1049900073079800D0002000010020006E019000F5
:1049A000FE019000800F5100818F59007C003E0075
:1049B0006E009000FE00900000600100AF03370021
:1049C0000C0037000D0037001200370017003700C9
:1049D0001D0037002300370044003700480037002F
:1049E0004C00370052003700580037005E00370097
:1049F0006400370090FF0700B4FF3700F0EF0200BB
:104A00000000000010C0B3008EDF020000000000B4
:104A1000AEFF370030F002000000000010C0B3000D
:104A20008EDF020000000000A8FF37000040EB000E
:104A3000F2F102000000000010C0B3008EDF02009F
:104A400000000000A1FF370010C0B300F2F1020027
:104A50000000000010C0B3008EDF02000000000064
:104A60009AFF3700A060230010407800E24F50000A
:104A700006003A0016F102000000000080407800B5
:104A8000C06023000148780006003700F00F2000C6
:104A900050F002000000000080407800C060230059
:104AA00001487800E05D2300104078006840600015
:104AB0000004E00008003200C060230010407800CD
:104AC0000080FB00D001020001000000804078005F
:104AD000C060230001487800C060230010407800C7
:104AE0008EDF02000000000078FF370064F1020052
:104AF000000000008EDF02000000000073FF37009E
:104B000004F20200000000008EDF0200000000003E
:104B10006EFF370010C0B300A8F1020000000000D3
:104B200010C0B3008EDF02000000000067FF3700F6
:104B30000040EB00E0F102000000000010C0B300F4
:104B40008EDF02000000000060FF370010C0B300DD
:104B5000E0F102000000000010C0B3008EDF020090
:104B60000000000059FF37000040EB00CEF10200CA
:104B70000000000010C0B3008EDF02000000000043
:104B800052FF370010C0B300CEF102000000000059
:104B900010C0B3008EDF0200000000004BFF3700A2
:104BA0000040EB008EDF02000000000047FF3700EE
:104BB000E060230090407800F0C0B30080C0600047
:104BC000E060230001487800E06023001040780096
:104BD0008040E800E06023000148780010C0B30086
:104BE0008EDF020000000000C16023000040EB00E7
:104BF000804878003D003700ECDF02000000000034
:104C000080407800B060230001487800E05D230018
:104C100010407800684060000004E00008003200A6
:104C2000B0602300104078000080FB00D00102003B
:104C30000100000080407800B06023000148780047
:104C4000A060230010407800E24F500009003A00B5
:104C5000B0602300104078000080FB00C2F002002A
:104C60000000000010C0B3008EDF02000000000052
:104C700019003700B0602300104078000080FB006E
:104C800050F002000000000080407800B060230077
:104C900001487800E05D2300104078006840600023
:104CA0000004E00008003200B060230010407800EB
:104CB0000080FB00D001020001000000804078006D
:104CC000B060230001487800B060230010407800F5
:104CD0008EDF020000000000C0602300104078005A
:104CE0008040E800C060230001487800C0602300D5
:104CF00090407800E06023001040780080CF5000A2
:104D0000BDFF3900F1FE3700E060230090407800DD
:104D1000F0C0B30080C06000E0602300014878006C
:104D2000E0602300104078008040E800E06023004D
:104D300001487800E060230010407800A8F10200EC
:104D40000000000010C0B3008EDF02000000000071
:104D5000DEFE3700E060230090407800F0C0B30032
:104D600080C06000E060230001487800E06023001C
:104D7000104078008040E800E0602300014878009F
:104D800010C0B3008EDF020000000000ECDF020064
:104D90000000000080407800D060230001487800C7
:104DA000C16023000040EB00804878001600370007
:104DB000D0602300104078000004E00004003D00B3
:104DC00010C0B30086F102000000000003003700AD
:104DD0000040EB0086F1020000000000D0602300DC
:104DE000104078000040400080407800D0602300F0
:104DF00001487800C0602300104078008040E8003F
:104E0000C060230001487800C06023009040780013
:104E1000E06023001040780080CF5000E4FF3900AC
:104E200010C0B3008EDF020000000000A7FE3700B4
:104E3000E0602300104078000080FB0030079800FD
:104E4000400A2000BE009000808F50001B003200FE
:104E5000400A20003E019000800F510005003C00F8
:104E6000000A2000BE019000808F51000A0032002D
:104E7000F0013700500A2000BE009000808F5000E3
:104E8000B8003200700A20003E019000800F5100EF
:104E900020013200E7013700ECDF020000000000D3
:104EA00080407800606723000148780010C0B3009C
:104EB0008EDF02000000000084FE370060672300E0
:104EC000104078000080FB0020079800AE019000A1
:104ED000E18F5100040032002E009000E20F5000DC
:104EE000360032009B003700ECDF020000000000BB
:104EF0000080FB0040B0890040B081006300B90031
:104F000040B089000000EB0010B0890009003700B4
:104F1000817F810010B0810000844000ECDF02003E
:104F200000000000004C780010B081000000E80094
:104F300010B0890011B0810040B08100808F500016
:104F4000F3FF39000000EB0010B0890013003700B8
:104F5000817F810010B08100008040000080E80067
:104F600010417800817F810010B0810000804000F6
:104F70000000E80090417800817F810010B081003E
:104F80000080400010407800834078009E020700B7
:104F900010B081006300400010B0890011B08100A2
:104FA00040B08100808F5000E9FF390010C0B3008D
:104FB0008EDF02000000000044FE3700ECDF02003C
:104FC000000000000080FB0040B0890040B081007C
:104FD0004200DD0040B089000000EB0010B0890005
:104FE00009003700817F810010B0810000844000FB
:104FF000ECDF020000000000004C780010B08100DF
:105000000000E80010B0890011B0810040B08100BC
:10501000808F5000F3FF39000000EB0010B08900D2
:10502000440037000040EB0086F102000000000061
:105030000040EB0086F10200000000000040EB00A1
:1050400086F10200000000000040EB0086F1020043
:1050500000000000817F810010B0810000804000CE
:10506000104078000080FB00C2F002000000000049
:10507000817F810010B08100008040000000E800C6
:10508000104078000080FB00C2F002000000000029
:10509000817F810010B08100008040000080E80026
:1050A000104078000080FB00C2F002000000000009
:1050B000817F810010B081000080400063014000CA
:1050C000817F810010B081000080400063004000BB
:1050D000104078006F40600000497800C1602300F4
:1050E0000040EB008048780006003700800207008F
:1050F000C0602300104078008040E800C0602300BA
:1051000001487800817F810010B08100008040005C
:105110006300400090407800C06023001040780099
:1051200080CF5000F1FF3E0010B0810064004000CD
:1051300010B0890011B0810040B08100808F500014
:10514000B8FF390010C0B3008EDF0200000000007D
:10515000DEFD37000040EB008EDF020000000000A3
:10516000DAFD370060672300104078000080FB0004
:10517000100798009E009000E18F5000040032005C
:105180001E019000E20F510040003200CFFD3700B9
:10519000ECDF0200000000000080FB0040B089004E
:1051A000ECDF02000000000080407800D0602300A7
:1051B000014878000000EB0010B089002E00370095
:1051C000D060230090407800B06023000148780050
:1051D000C16023000040EB008048780019003700D0
:1051E000B0602300104078000080FB006100600088
:1051F0000004E0000400320010C0B30086F1020099
:1052000000000000030037000040EB0086F10200C0
:1052100000000000B0602300104078000080FB0018
:105220000000D10080407800B06023000148780081
:10523000C0602300104078008040E800C060230078
:1052400001487800C060230010407800E34F500010
:10525000E3FF360016F102000000000016F1020024
:10526000000000008EDF02000000000010B081008E
:105270000000E80010B0890011B0810040B081004A
:10528000808F5000CEFF390090FD3700ECDF020028
:10529000000000000080FB0040B089000000EB002F
:1052A00010B089001600370022C0B30060B920009A
:1052B000A10B2000510207008402070022C0B300A6
:1052C00060BB2D00A10B20004C02070022C0B300E0
:1052D000603D2D00A10B2000480207007B02070063
:1052E00022C0B30060BB2000A10B200043020700D6
:1052F0007602070010B081000000E80010B08900BD
:1053000011B0810040B08100808F5000E6FF39006D
:105310006EFD3700ECDF0200000000000080FB00A3
:1053200030B08900ECDF0200000000000080FB00CC
:1053300020B089006067230010407800E24F5000E1
:1053400007003A0030B081006500B90080007800A5
:1053500020B081000080400040B089001C00370070
:105360006067230010407800E14F500008003A00C9
:1053700030B08100000040008000780020B0810043
:10538000008040000000400040B08900100037005D
:105390006067230010407800E34F500008003A0097
:1053A00030B08100000040008000780020B0810013
:1053B000008040000000400040B089000400370039
:1053C0000040EB008EDF0200000000003FFD3700D0
:1053D0000000EB0010B0890009003700817F8100D8
:1053E00010B0810000844000ECDF020000000000EB
:1053F000004C780010B081000000E80010B0890077
:1054000011B0810040B08100808F5000F3FF39005F
:1054100020B081000000E0000300320010C0B300A3
:105420008EDF0200000000000000EB0010B08900D9
:1054300075003700817F810010B08100008040003E
:1054400010407800E14F500045003A0060672300AB
:1054500010407800E34F500015003A00817F810032
:1054600010B08100008040006300400010417800CF
:10547000817F810010B08100008040000080E80042
:1054800090417800817F810010B081000080400051
:105490000000E80010407800834078001501070004
:1054A00010B081006400400010B089005600370041
:1054B0006067230010407800E14F500015003A006B
:1054C000817F810010B081000080400063004000B7
:1054D00010417800817F810010B081000080400081
:1054E0000080E80090417800817F810010B0810049
:1054F000008040000000E800104078008340780001
:105500004101070010B081006400400010B0890024
:105510003D0037006067230010407800E24F5000E4
:1055200039003A00817F810010B081000080400086
:105530006400400010417800817F810010B081003C
:10554000008040000000E8008240780080010700F1
:1055500010B081006500400010B089002A003700BB
:10556000817F810010B081000080400010407800F1
:10557000E24F500024003A0060672300104078009A
:10558000E34F50000A003A00817F810010B0810093
:10559000008040000000E80010407800BA000700DA
:1055A00010B081000080E80010B0890016003700BC
:1055B0006067230010407800E14F50000A003A0075
:1055C000817F810010B08100008040000000E80071
:1055D00010407800EB00070010B081000080E80068
:1055E00010B0890008003700606723001040780081
:1055F000E24F500004003A00B401070010B08100EF
:105600000000E80010B0890011B0810040B08100B6
:10561000808F500087FF390020B081000000E0003B
:10562000AAFC3A0010C0B3008EDF020000000000A8
:10563000A6FC37000040EB008EDF020000000000F7
:10564000A2FC3700E060230010407800940A0200BA
:105650000100000010C0B3008EDF02000000000057
:105660009AFC3700E060230010407800120B020023
:10567000010000008EDF02000000000093FC3700F4
:10568000E06023009040780030C0B30080C060002C
:10569000E060230001487800E0602300904078003B
:1056A000C05C230001487800C05C23009040780073
:1056B000A06023001040780062EF020000000000AC
:1056C00010C0B300F2F102000000000010C0B300EF
:1056D0008EDF0200000000007CFC3700E15D23004B
:1056E000114078000040A10080487800E06023006D
:1056F000104078000080FB004300DE000000A200A4
:10570000610060000004E00004003200E15D23005D
:10571000114078000040A00080487800A16023007C
:1057200020C0B30080487800E0602300104078007B
:105730000080FB004200DE00610060000004E00029
:1057400003003200A160230030C0B300804878001D
:10575000E15D2300114078000030A100804878000E
:10576000E0602300104078000080FB000000D100C2
:10577000610060000004E00004003200E15D2300ED
:10578000114078000030A00080487800C05C230001
:1057900090407800A06023001040780062EF020083
:1057A0000000000010C0B300F2F102000000000091
:1057B00010C0B3008EDF02000000000043FC370081
:1057C000E0602300104078000080FB00000F7800AC
:1057D000000F20009E017800808F510005003200EC
:1057E000100F20009E007800808F500004003200CF
:1057F00009003700F40B02000100000033FC370001
:10580000CE0B02000100000010C0B3008EDF0200CA
:10581000000000002DFC3700E060230010407800FD
:105820000080FB006F00600000B0890000B08100C4
